:020000040800F2
:100000000050002089010008D10100080000000014
:10001000D1010008D1010008D10100080000000052
:10002000000000000000000000000000D1010008F6
:10003000D101000800000000D1010008D101000832
:10004000D1010008D1010008D1010008D101000848
:10005000D1010008D1010008D1010008D101000838
:10006000D1010008D1010008D1010008D101000828
:10007000D1010008D1010008D1010008D101000818
:10008000D1010008D1010008D1010008D101000808
:10009000D1010008D1010008D1010008D1010008F8
:1000A000D1010008D1010008D1010008D1010008E8
:1000B000D1010008D1010008D1010008D1010008D8
:1000C000D1010008D1010008D1010008D1010008C8
:1000D000D1010008D1010008D1010008D1010008B8
:1000E000D1010008D1010008D1010008D1010008A8
:1000F000D1010008D1010008D1010008D101000898
:10010000D1010008D1010008D1010008D101000887
:10011000D1010008D1010008D1010008D101000877
:10012000D1010008D1010008D1010008D101000867
:10013000D1010008D1010008D1010008D101000857
:10014000D1010008D1010008D1010008C116000842
:10015000D1010008D1010008D1010008D101000837
:10016000D1010008D1010008D1010008D101000827
:10017000D1010008D1010008D1010008D101000817
:10018000D1010008D1010008684620F007018D4622
:1001900001B50A4A0A4B0B4903E052F8040B43F835
:1001A000040B8B42F9D3084B0849002201E043F8C5
:1001B000042B8B42FBD300F00DF8FEE7A03A0008B9
:1001C000000000203800002038000020381C0020EB
:1001D000FEE70000F7B5002000F0A0FF002001F0CE
:1001E0001DF9012001F0A0F8684601F0B8FECD48E5
:1001F00001238DF8043000251F33CB4E8DF80550B8
:100200008DF8065069460383009301F061FE4FF4B8
:100210000053338330466946009301F059FE0823AA
:10022000338330466946009301F052FEBF4E731986
:1002300070599B88694603830835009301F048FE96
:10024000302DF4D1B74F8026B74D7E8338466946AE
:10025000009601F03DFE48F2000169834FF400432F
:1002600028466946009301F033FE20236B8328461D
:100270006946009301F02CFEAA4B20225A834FF4CA
:10028000005708226F8301206A8301F0E7F8A5492F
:1002900020230B8308232F8301202B8301F0DEF81A
:1002A00016F1FF36A04CE7D1A14D04214FF40062B6
:1002B0004FF4805361836A834FF480616383994B69
:1002C000698348F200024FF480715A8301206183F0
:1002D00001F0C4F804224FF400634FF480512283EC
:1002E0002B834FF4806221838E492A8348F20003D6
:1002F0004FF480720B830120228301F0AFF80123B9
:100300008DF8073002AD1F3345F8083D8548694632
:100310008DF8046001F0DCFD20466946009701F08D
:10032000D7FD082100912046694601F0D1FD7F4CA0
:10033000A3199B88A05969460836009301F0C8FDAF
:10034000302EF5D1774C802320466946009301F08A
:10035000BFFD4FF4004374486946009301F0B8FDB7
:10036000202369467048009301F0B2FD642001F03B
:1003700015F8266901F0B8F9C5B206F001061DB9F5
:10038000236913F0010F0BD03EB18020012101F051
:100390004FFE8020002101F04BFE002001F0AAF961
:1003A000002000F04FFB002000F026F965B95D4BFE
:1003B0001B6913F0010F40F0AE80A7E05D4B1B7886
:1003C000002B00F0A8803EE0102000F0E9FAA2E047
:1003D00001F016F86422B0FBF5F3B3FBF2F102FB77
:1003E0001133B0FBF7F207FB120241F288315B08D0
:1003F0008A42B0FBF5F105FB110188BFC3F132035E
:100400000446994294BF00210121012000F0AEFF73
:100410000A23B4FBF3F203FB12440CB900F034FEE0
:10042000002000F043FD00F0EBFF44F61F62904215
:10043000CED900F0EBF80028CAD126B139490B69B2
:1004400013F0010FC4D101F0B5FC0120002100F030
:100450008DFF394BDB78082B41D16FF0070001216C
:1004600001F0D8FD6FF08000012101F0E1FD4FF0B7
:10047000FF30012101F0EAFD4FF0FF30012101F0D2
:10048000F3FD4FF0FF30002101F0C4FD4FF0FF30CD
:10049000002101F0CDFD4FF0FF30002101F0D6FD2D
:1004A0004FF0FF30002101F0DFFD46B18020012137
:1004B00001F0BEFD8020002101F0BAFD08E001F04E
:1004C00013F928B11D48D0F8E0350BB102F0F5FA68
:1004D0001B4B1B6883F30888174B1B68984740F237
:1004E000F31400F083FF0120014600F03FFF00F00D
:1004F00087FFA042FBD900F079FF0120002100F026
:1005000035FF00F07DFFA042FBD9EAE70D4B1B78D9
:10051000422B3FF453AF00F069FF322542F21077CF
:1005200056E700BF000002400004024064380008A3
:10053000000C0240D33F000804400008E0150020F2
:1005400000400008D23F0008134B1A78032A0CD849
:10055000124900F07F00D1F800C04FEACC1C4CEAF1
:100560000010086013D1042212E0072A88BF4FF060
:10057000FF300FD80A4900F07F00D1F800C04FEAE1
:10058000CC1C4CEA0010086001D1082200E00132C6
:100590001A700020704700BFFC04002038000020C3
:1005A0004800002070B5134B16461A7888B08DF8B5
:1005B00000205A780D468DF801209A7804468DF86F
:1005C0000220DA781B798DF803208DF8043000F0D2
:1005D0009FFDF7238DF805006946204609228DF816
:1005E00006508DF807608DF8083000F0A1FA08B0C9
:1005F00070BD00BF9439000810B9034B187001E0BA
:100600004FF0FF30704700BFFD040020014B187809
:10061000704700BFFD040020F7B51E460D46174683
:10062000044600F06BFD00F0E1FE012E06D0022E24
:1006300018BF4FF0FF3040F08B8189E01DB1012DD4
:10064000C84B0BD105E0C74B1D70C74B1D60C74B96
:1006500091E01B78072B00F27A8197E01B78082B3A
:1006600040F0E680C04BC24D1F68C04B1E68C14BB6
:100670001A782A705A786A709A78AA70DA781B7990
:10068000EA702B7100F044FD4FEA566C6871780EE9
:100690000223E871C7F386416044AB712972C7F346
:1006A000C6234118C7F30612C9186B728918C6F31E
:1006B00086432B73C918C6F3C623C9186B73C6F3D8
:1006C0000613AB73CB1803F0FF010023AA7285F861
:1006D0000BC01A460F351846019422E010F807E0C7
:1006E0004FF0000C01334FEADE14DBB244EA420261
:1006F0004FEA4E0E062BD2B25FFA8EFE09D9C3F135
:1007000007039A40D2B25118002305F8012BC9B251
:100710001A460CF1010C5FFA8CFCBCF1080FE1D118
:100720000130B042DAD1019C1BB1891805F8012BC8
:10073000C9B249422A4601F07F0102F8011B8C49E7
:10074000F72301326B70521A204600F0F1F9FEE0F7
:1007500015B1012D5CD111E0824B1D70824B1D60E3
:10076000824B1D60844B1D70844B1D70844B1D603B
:10077000844B1D60844B1D602846E9E0794B187856
:10078000072807D87C4B1A78BA181A703846FFF732
:10079000DBFEDCE0082832D1774B1A78BA181A70E1
:1007A000774B1B68B3F5806F80F0D1806F4A704E35
:1007B0001468754A4FF0000C1168724A2546126899
:1007C0000132C7F380147F00072A44EA4101FFB2D7
:1007D00005D9F1540133AB4228BF092000220CF1A6
:1007E000010CBCF1070FEBD1DFF89CC1CCF8001075
:1007F00064490A60624A13605A4B1870A7E00928DE
:1008000004BF5E4B1F7000F0A2800C221A709EE0A5
:10081000564B1B6801935A4B019A1B68934203D2B3
:1008200020460E21012213E04E4B1B780C2B03D1E6
:1008300020460E2132460BE0504B1A784E4B1B7867
:100840005B4203F07F039A4205D020460E2103222B
:10085000FFF7A8FE7BE04D4B01221A70424B019A34
:100860001D6845EA020313F0030F63D1484B9D4214
:1008700063D900F0E7FC00F100600138854249D8F7
:1008800001F08AFA002243491346885885421BD159
:10089000414A954202D1414A00211160012098400D
:1008A0003E4A116808420CD140EA01011160394A00
:1008B0000C2101FB03230221586801F0D3FA082818
:1008C00017D12B4E002720E001330C320C2BDCD14A
:1008D000F7E7B1787378264A090441EA0321D35D2A
:1008E0001943F378043641EA036101F09DFA0828C0
:1008F00006D04FF0FF3001F065FA6FF003021EE002
:1009000001F042FA01F038FA0437019B78199F424E
:10091000DFD31EE0B5F1005F0FD300F09BFC00F1C8
:1009200000500138854208D828461149019A02F042
:100930008DFF0EE06FF0080201E06FF007025242F7
:10094000D2B220460E21FFF72DFE00F09DFB0020C5
:10095000FEBD094B20461A780F21524202F07F0259
:10096000F1E700BFFC040020380000204800002010
:100970005000002094390008400000204C00002066
:10098000F80400200005002044000020FD040020A1
:10099000FF3F000894380008004000083C00002099
:1009A00010B5114B88B01A7804468DF800205A789B
:1009B0008DF801209A788DF80220DA781B798DF86D
:1009C00003208DF8043000F0A3FB01238DF805000F
:1009D0008DF806302046F633694608228DF8073038
:1009E00000F0A6F808B010BD9439000808B5202022
:1009F000FFF7D6FF1020FFF7D3FF024B002018703F
:100A000008BD00BFFD04002008B50A4A137803F0B2
:100A10000803DBB23BB1084B1B78834203D10023B0
:100A20001370064A1370064B1B6803B198470020E9
:100A300008BD00BF2805002014050020090500207E
:100A40001805002010B504464FF0FF30002C2AD1C5
:100A5000154A10231370154A20461370144B1C605E
:100A6000144B1C60144B1C60144B1C60144B1C601A
:100A7000144B1C6000F04AFF134B144A1C70144BBB
:100A8000C00F1C70134B1C701278422A05D1124AF9
:100A9000127812F0800F08BF1A70104A00231380DA
:100AA0000F4A4042136010BD0000002001000020EA
:100AB0000C05002004050020240500201805002056
:100AC0001C0500201005002014050020D03F000860
:100AD0002805002015050020D13F0008160500203C
:100AE0002005002010F0F00F38B504460D4604D163
:100AF00001280CBF0B4B0C4B1C780C4B64F30715F7
:100B00001B681BB120462946984748B904F0F004F9
:100B1000102C18BF4FF0FF3002D1284600F06AFFBA
:100B200038BD00BF010000200000002004050020A7
:100B3000F0B585B0174603900D4600260623072220
:100B40004FF0040C40E0B91B022914D003291FD038
:100B50000129A95D18BF6CF3030406F1010618BF53
:100B600061F30F241AD1052060F3030461F30F240D
:100B70006FF3174409E0A95D63F30304013661F3E1
:100B80000F24A95D013661F317446FF31F640DE074
:100B9000A95D62F3030461F30F240136A95D0136F8
:100BA00061F31744A95D013661F31F640398214680
:100BB00001920293CDF800C0FFF794FF0028019A3C
:100BC000029BDDF800C002DBBE42BCD3002005B0B2
:100BD000F0BD000010B5F023A0B08DF80030002368
:100BE0008DF801308DF802307E338DF803303223DA
:100BF0008DF804300E4B0DF16B0C1B788DF8053021
:100C00000F238DF806306B46DA1D03E002F8014B26
:100C1000624503D011F8014B002CF7D1F72102F8FF
:100C2000011BD21A6946FFF783FF20B010BD00BF39
:100C30001505002000B5F02389B08DF800300023A1
:100C40008DF801308DF802307E338DF80330322379
:100C50008DF80430084B8DF806101B788DF80720AE
:100C60008DF805306946F72309228DF80830FFF723
:100C70005FFF09B000BD00BF15050020F0B5494E6B
:100C80008BB0337804460D461746FFF7C5FC0028A5
:100C900080F2858031780D2964D001D829B174E0C3
:100CA0000E297CD00F2970D162E01DB1012D3E4B81
:100CB00005D102E03C4B1D7071E01F706FE01B78A6
:100CC000052B28D00AD8022B18D002D8012B45D1E9
:100CD00011E0032B15D0042B40D115E0082B32D0A6
:100CE00004D8062B21D0072B38D129E0092B2DD091
:100CF0007F2B33D12FE020462C4929E020462C4978
:100D000026E020462B4923E000F096FA6D46024685
:100D1000294968460FE0684600F0A0FA00286D46B1
:100D2000BCBF2046254908DA12E000F08BFA2449BE
:100D300002466D46684600F0F3FF2046694607E02C
:100D400000F088FAF3E720461E4901E01E492046DC
:100D5000FFF740FF23E0FFF749FE20E020460E2189
:100D60000D220FE0022D1AD120460E21102209E09B
:100D7000164B15B1012D154B01D15D600FE05A687E
:100D80006AB92046FFF756FF09E00E210A462046C1
:100D9000FFF750FF0D4A00231370024A1370002022
:100DA0000BB0F0BD0905002008050020343900080B
:100DB0003B3900084C390008563900085B390008F7
:100DC0005D390008603900087239000828050020E4
:100DD000F72910B50A465CD82F4B1C7804F008039D
:100DE000DBB21BB12D49097881424FD1A0F111012D
:100DF000C9B206294AD9294908700BBB264B1B7872
:100E000003F00703042B03D82549C95C914223D181
:100E100004F00704052C03D12249097891421BD123
:100E2000013303F007021C4B052A197862F3020113
:100E300084BFCAB242F00802197088BF1A7028E055
:100E400012F0800F0ED0F72A06D104F01004E4B29D
:100E500014B10221FFF712FF0F4B00201870124B44
:100E6000187017E004F01004E4B25CB90A4B19786A
:100E700041F0100119700C4B21461A70FFF7FEFE6D
:100E8000204607E00121FFF7F9FE02E04FF0FF30B6
:100E900000E0002010BD00BF280500201405002040
:100EA000943900081505002009050020F0B501213E
:100EB00087B000250646029101952F4600E0039F6A
:100EC0007B1CDBB2039317B10C2F0BD8A2E005A853
:100ED00000F0AAFD0599C1F30314103410F10A0FB4
:100EE00013D10DE0019A2B1E18BF0123092A8CBFD4
:100EF000002303F00103002B40F0BE80029389E041
:100F00002046FFF781FD029784E00028C0F282802E
:100F1000019A67F30711531CDBB2019301F00F0331
:100F200003F1080202F00F020135062AEDB2059125
:100F300002D8204686B96DE09A1E0D2A6AD8DFE8ED
:100F400002F007070D444848696969696969690DD4
:100F5000002E5FD005992046B0475BE09DF8151044
:100F6000F729F5D8F0291CD1454A1368CBB904F00C
:100F7000F002102A02D0302A13D109E0414A13802E
:100F8000012204F00F0312FA03F33D4A138008E034
:100F90003C4A1380012204F00F0312FA03F3384A8B
:100FA00053802046FFF714FF9DF8143003F00F0321
:100FB0000F2B2FD09DF816102046FFF709FF9DF844
:100FC00017102046FFF704FF24E09DF81520F72AAC
:100FD000BED8043BDBB2EBB19DF815702046394614
:100FE0000093FFF7F5FE009B012B0ED09DF81670C5
:100FF00020463946FFF7ECFE009B022B05D09DF8FA
:10100000177020463946FFF7E3FEF72F02D11C4B3D
:10101000002119601A4B1A683AB31A490A88B2F5C6
:101020007A7F22D9198861B1002251FA02F313F0B4
:10103000010303D10132102AF7D11A461032D0B27F
:101040000DE0588858B10B4650FA03F212F0010235
:1010500003D10133102BF7D113463033D8B2FFF749
:10106000D3FC074B00221A6003E0029A002A7FF4A7
:1010700026AF002007B0F0BD00250395CAE700BFEA
:10108000200500201605002008B500F0F9FC044BEF
:101090004FF6FF711A888A4201D001321A8008BDCA
:1010A00016050020F0B5134E85B034680746ECB144
:1010B000C1F307638DF80E300F4BC1F30742C1F344
:1010C0000720002401F00F018DF80D208DF80C0091
:1010D0005A5C254608E003AB595D384601923368F7
:1010E0009847019A044301359542F4DB204605B048
:1010F000F0BD00BF0C05002024390008012817BFEF
:10110000024B4FF0FF3018700020704701000020A4
:10111000014B1878704700BF1505002013B5044631
:101120004FF0FF30002C79D11F20012100F03AFF51
:101130003B4B01949A6802F00C02082A02D1012369
:1011400001935DE01A6842F001021A609C601A681F
:1011500022F0847222F480321A60324A5A601A688D
:1011600022F480221A60DC6000941A6842F4803213
:101170001A601A6802F400320192009A0132009259
:10118000019A1AB9009AB2F5A06FF2D1244B1B68EC
:1011900013F4003318BF01230193019B012B2FD1BE
:1011A0001F4B1A6C42F080521A641F4A116841F4B6
:1011B000804111609A689A609A6842F400429A608D
:1011C0009A6842F4A0529A60184A5A601A6842F02B
:1011D00080721A601968124A11F0007FFAD0144B1D
:1011E00040F205611960936823F0030393609368EC
:1011F00043F002039360936803F00C03082BFAD1C9
:101200000C48002100F0A6FD4FF4407000F098FD5E
:101210000198012814BF4FF0FF3000201CBD00BF13
:10122000003802401030002400700040085440078D
:10123000003C024000000008014B1868704700BFE6
:10124000002004E0024B188880B28002704700BF83
:10125000227AFF1F4FF440307047000000230B4AF2
:1012600059108A18127813F0010F08BF120902F002
:101270000F02092A94BF302137218A18C254013342
:10128000182BECD10023037618467047107AFF1F05
:10129000084B1B681BB9EFF31082074B1A604FF025
:1012A000010080F31088034B00201A6801321A6095
:1012B000704700BF3405002030050020064A4FF07B
:1012C000FF3013683BB1013B13601BB9034B1B6834
:1012D00083F310880020704734050020300500207B
:1012E0000F2988BF4FF0FF3018D80D4B42B2DB6892
:1012F0005209DB43C3F30223C3F104039940094BB2
:101300000901C318C9B283F8001300F01F000123BC
:1013100013FA00F0034B43F822000020704700BF8F
:1013200000ED00E000E100E037B50446684600F05B
:1013300016FE01238DF80430013B8DF80630023390
:1013400014F0010F6D468DF8053006D04FF4805330
:1013500005486946009300F0BBFD34F00F040CBF54
:1013600020466FF001003EBD000C024010F0010F5E
:101370000BD011F0010F15BF074B074B4FF48052F4
:101380004FF4805214BF1A835A8330F00F0018BFF5
:101390006FF00100704700BF000C024030B5012122
:1013A00085B00446102000F019FE4FF6FF7302933B
:1013B00054235C430C4D013CADF804402846002406
:1013C00001A9ADF80C40ADF8064000F05BFE01212C
:1013D0000A46284600F0BFFE2846012100F0AEFE76
:1013E000204605B030BD00BF001000400348012179
:1013F00008B5416200F0C6FE002008BD00100040A4
:10140000054810B50121446A00F0B0FE002818BF5D
:101410004FF0FF34204610BD001000401FB50446B9
:101420004FF0FF30B4B90120014600F0E5FD4FF662
:10143000FF7302930848A72301A9ADF80430ADF863
:101440000C40ADF8064000F01DFE0348012100F0FD
:1014500075FE204604B010BD00000140044B5A6ADE
:1014600092B2596A891A89B28142FAD9002070472A
:101470000000014012230B8000487047E839000843
:1014800004230B8000487047E439000810B586B08B
:101490001F49122201A802F0D9F91E490122002396
:1014A00006E0203AD2B25F2A8CBF0022012201332B
:1014B0001F2BCCBF002002F0010020B111F8012F3A
:1014C000002AEED10132002B0CBF002302F00103F1
:1014D00001A903B11049114A02234FF0000C04E0A6
:1014E00002F8020C02F801CC023311F8010B0232AF
:1014F000041E18BF0124632BCCBF002404F0010498
:10150000002CEDD1064803700323437006B010BDD4
:1015100060390008DF3F0008E03F0008D21B0020D0
:10152000D01B002008B5FFF7B1FF08BD08B5FFF7D5
:10153000ADFF08BD70477047704770477047002087
:10154000704700207047000065230B8000487047FB
:10155000283A000870B58CB00BAD03220C4601AEE2
:101560000849284602F072F93046FFF777FE002856
:10157000ACBF304628460449224601F053F90248E0
:101580000CB070BD183A0008D01B00207FB5084C85
:1015900001AD0E460C222846064902F057F92846AE
:1015A0002146324601F03EF9204604B070BD00BF2E
:1015B000D01B00201B3A0008022908B503D10846B9
:1015C000002100F06FFA002008BD012908B503D101
:1015D0000846013900F05CFA002008BD10B5022170
:1015E000044601F0F4FD2046812101F0F0FD0020C9
:1015F00010BD08B5002000F08FF908BD08B5012026
:1016000000F08AF908BD0000022110B5402204460E
:101610000B4601F0B3FD812140220223204601F058
:10162000ADFD0221034A4023034801F0EFFD0020F5
:1016300010BD00BFA0150020E015002013B501204B
:10164000014600F0AFFC4FF4D853194C009303232C
:101650008DF80530013B8DF80430204600236946A3
:101660008DF806308DF8073000F032FC2046082156
:101670000A2200F07DFC204609210A2200F078FCB5
:1016800020460B210A2200F073FC0A2220460C217E
:1016900000F06EFC01214FF4804000F0ADFC802092
:1016A000012100F08DFC012000F060FB1CBD00BF9B
:1016B0000000024008B543200821FFF711FE08BDD5
:1016C00008B5024801F048FE08BD00BFE015002043
:1016D00008B580B2FFF7C2FE08BD08B54FF47A73B3
:1016E0005843FFF7F5FF08BD4FF0A0431868C0F35B
:1016F000C0407047022837B5054688BF4FF0FF301D
:101700003ED8FFF776FF4DBBFFF7EEFF30B31D4C21
:101710002046FFF793FF1C4B0121C4F8E0351B4B1B
:101720002046C4F8E4351A4BC4F8E83501F0E6F871
:10173000204601F0BBF9204601F02AFA2046FFF7C7
:10174000B9FF01210323204684F8101184F81231D7
:10175000FFF75AFFFFF752FF284611E00B4B01211C
:101760000B4A00930748084B00F0FFFD054801F0C5
:10177000E9FD3220FFF7B1FF024801F0D9FD00205A
:101780003EBD00BFE0150020B8390008FC39000854
:101790009C390008F0B52B4C85B0D4F8E035002B0F
:1017A0004DD0FFF775FD284B1B78002B45D0D4F8A2
:1017B000D853C5F38F05002D3FD0244B29B21A888A
:1017C00092B2C2F50072914237DA013D204F214CAE
:1017D000214AADB240F2FF1C57F8046B0392C6F3E6
:1017E0000310103031460193CDF808C0FFF75AFCC2
:1017F000039A019BDDF808C080B9218889B242F8BC
:1018000021602188013189B22180218889B2614516
:1018100088BF20801988013189B21980013DADB29D
:10182000691C09B20029D7DC074B00221A70054851
:101830000221074A402301F0E9FCFFF73FFD05B014
:10184000F0BD00BFE01500208015002078050020C5
:10185000A015002082150020800D0020244B10B51B
:10186000D3F8E035002B42D0FFF712FD214B1B7857
:10187000002B3AD1204B1A8892B2002A35D01F4A49
:101880001278002A31D01A881D4892B2102A98BFC7
:101890001B88184A94BF9BB2102301211170164A6D
:1018A000DFF860E0118840F2FF1CC91A89B211808C
:1018B0001BB20021144A10E01488A4B25EF8244040
:1018C00040F8044B14880134A4B214801488A4B2E4
:1018D000644501D90024148001319942ECDB9B005E
:1018E00003488121064A01F0B9FCFFF7E7FC10BD6F
:1018F000E01500207C0D0020841500208A150020B2
:10190000380500207C05002086150020002814BF23
:101910004FF0FF3000207047104A002313801188D9
:101920000F4A89B2118011880E4A89B211800E4A7D
:1019300013700E4A138011880D4A89B211801188E4
:101940000C4A89B211800C490C4A10B10120087070
:1019500001E00B7001231370002070477805002010
:10196000821500207A0500208015002084150020B3
:101970008C150020861500208A1500207C0D002083
:1019800038B5184D04462B784FF0FF304BB3164B4B
:101990001B889BB2B3F5FF7F09D9FFF75FFF2B7858
:1019A000002B14BF6FF001004FF0FF3019E0FFF77C
:1019B0006FFC0E4B0E491A8892B241F82240013258
:1019C00092B21A801A8892B2B2F5007F01D3002237
:1019D0001A80054B1A88013292B21A80FFF76EFC0A
:1019E000002038BD8A150020841500208C150020A9
:1019F0007C05002070B506460A4C42F20F7504E0E3
:101A00002388AB420CD8013323803046FFF7B8FF60
:101A100010F1020FF4D0002802DB024B00221A80E2
:101A200070BD00BF88150020124B10B51B880446FE
:101A30009BB24FF0FF30E3B1FFF72AFC0E4B0F4A89
:101A4000198889B252F8212022601A88013292B294
:101A50001A801A8892B2B2F5007F01D300221A8050
:101A6000044C2388013B9BB22380FFF727FC20888E
:101A700080B210BD780500207A050020800D00207E
:101A800008B5FFF787FEFFF7E9FE002008BD00005C
:101A900008B5034B00221A70FFF7E0FE08BD00BF37
:101AA0007C0D002008B5034B01221A70FFF772FE6F
:101AB00008BD00BF80150020002A30B5C8BF4FF018
:101AC000000C044602DC12E00CF1010C11F80C00D1
:101AD0000028F9D19445B4BFCCEB0202024613F0C2
:101AE000020F0CBF4FF0200C4FF0300C01E04FF014
:101AF000200C13F001000CD108E02CB1236883F80E
:101B000000C02368013323600130013A002AF4DC6D
:101B100008E0002006E024B125682B70236801331B
:101B20002360013011F8013B002BF4D108E02CB107
:101B3000236883F800C02368013323600130013A31
:101B4000002AF4DC30BD7FB594461C46089A099BF8
:101B50000D4649B94FF0300C8DF8051001A98DF8EC
:101B600004C0FFF7A9FF46E0BCF10A0F14BF002133
:101B70000121002C0CBF002401F001042CB1002D28
:101B800002DA6D42012400E000240A9E0DF1100EDD
:101B900000210EF8011D3A3E0BE0B5FBFCF10CFBF9
:101BA00011510929C8BF891930310EF8011DB5FB43
:101BB000FCF57146002DF0D1D4B192B113F0020FB3
:101BC0000FD058B1D0F800C04FF02D0E8CF800E0C7
:101BD000D0F800C00CF1010CC0F800C0013A01249B
:101BE00006E04FF02D0C0EF1FF310EF801CC002471
:101BF000FFF762FF001904B070BD0000F0B589B0B6
:101C000005460E46059200247DE0252B72D116F87C
:101C1000013F002B7BD0252B6CD02D2B02D1013620
:101C2000012303E0002301E043F00203374616F8E6
:101C3000012B302AF8D0002202E00A2000FB02C269
:101C400039783E46A1F1300C5FFA8CF00137092853
:101C5000F3D9732909D10599081D059009682F4802
:101C6000002908BF0146284641E064290ED10599A4
:101C70000193612300920293081D096805900A22CE
:101C800028460123FFF75FFF24183BE0782906D19F
:101C900005990193081D05900092612307E05829DA
:101CA0000AD105990193081D0590009241230293E2
:101CB0002846096810220BE075290BD1059901937C
:101CC000612300920293081D096805900A222846A4
:101CD0000023D7E7632915D10599081D09680590E8
:101CE0008DF81C1000218DF81D10284607A9FFF75C
:101CF000E3FEC9E7327825B12B681A702B680133EF
:101D00002B60013401363378002B7FF47EAF15B1A0
:101D10002B6800221A70204609B0F0BD903A0008E6
:101D20000EB40FB505AA52F8041B019001A8039246
:101D3000FFF764FF04B05DF804EB03B070470000E8
:101D400040F0BE60024B40F42020D860704700BFD6
:101D500000ED00E021F0604121F07F01024B41EAFB
:101D600000009860704700BF00ED00E0014B586133
:101D7000704700BF003C0140024B1A6842F4006209
:101D80001A607047003C0240024B1A6842F48052CD
:101D90001A607047003C0240044B1A69002ABFBF1A
:101DA000034A5A6002F188325A607047003C024090
:101DB00023016745024B1A6942F000421A617047DD
:101DC000003C0240014BD860704700BF003C02401D
:101DD0000C4BDA6812F4803F0ED1DA6812F0100F63
:101DE0000CD1DA6812F0EF0F0AD1DB6813F0020FA2
:101DF0000CBF0820072004E0012002E0052000E0DD
:101E000006207047003C024007B508238DF80730D4
:101E1000FFF7DEFF8DF807009DF80730012BF7D0A4
:101E20009DF807000EBD000070B504460E46FFF792
:101E3000EBFF082813D10A4D2B6923F440732B6163
:101E40002B6943F400732B612B6943F001032B6171
:101E50002660FFF7D9FF2B6923F001032B6170BDCA
:101E6000003C024070B504460E4651B1012908BF3E
:101E70004FF4807605D0022914BF4FF440764FF41A
:101E80000076FFF7C1FF08281FD1104D2B6923F4FE
:101E900040732B612B691E432E612B6923F0F803DD
:101EA0002B612B6943F0020343EA04042C612B6984
:101EB00043F480332B61FFF7A7FF2B6923F0020364
:101EC0002B612B6923F0F8032B6170BD003C0240AD
:101ED000F7B50B68019300231A46012404FA02FCAB
:101EE000019D0CEA0504644534D1032606FA03FC7F
:101EF00005686FEA0C0C0CEA050505600D790768AA
:101F000015FA03F6013DEDB23E43012D066013D8EC
:101F10004E7985689E400CEA05058560856846EA2D
:101F200005058560456825EA040444608C794568A8
:101F30009440A4B22C434460C4680CEA040CC0F87A
:101F40000CC091F807C0C4680CFA03FC4CEA040CFE
:101F5000C0F80CC001320233102ABED1FEBD4FF6CC
:101F6000FF7303600023037143718371C371704772
:101F700001F007039B004FF00F0C0CFA03FC12FA60
:101F800003F3C908083110B550F8214024EA0C0CBD
:101F900040F821C050F821C043EA0C0340F821303A
:101FA00010BD000019B1054B1A6B104303E0034B41
:101FB0001A6B22EA00001863704700BF0038024025
:101FC00019B1054B5A6B104303E0034B5A6B22EADD
:101FD00000005863704700BF0038024019B1054B3C
:101FE0001A6C104303E0034B1A6C22EA00001864D9
:101FF000704700BF0038024019B1054B5A6C1043BE
:1020000003E0034B5A6C22EA00005864704700BF9B
:102010000038024019B1054B1A69104303E0034B25
:102020001A6922EA00001861704700BF00380240B8
:1020300019B1054B5A69104303E0034B5A6922EA70
:1020400000005861704700BF0038024019B1054BCD
:102050001A6A104303E0034B1A6A22EA000018626E
:10206000704700BF0038024019B1054B5A6A10434F
:1020700003E0034B5A6A22EA00005862704700BF2F
:1020800000380240264ADFF89CC00388904214BF03
:1020900000220122604508BF42F0010210B59BB248
:1020A000CAB9214CB0F1804F14BF4FF0000C4FF073
:1020B000010CA04214BF64464CF001045CB91B4CF7
:1020C000DFF86CC0A04214BF00240124604508BFA3
:1020D00044F001042CB1B1F802C023F0700343EACC
:1020E0000C03144CDFF850C0041B18BF01246045DA
:1020F0000CBF002404F0010434B123F44073B1F8A0
:1021000008C09BB243EA0C0303804B68C3620B8890
:1021100003850AB18B7A03860123838210BD00BF39
:10212000000001400004014000040040000800409D
:10213000000C0040001000400014004021B1038852
:102140009BB243F0010304E0038823F001031B0466
:102150001B0C038070471AB183899BB2194303E0BB
:1021600083899BB223EA010181817047038A8289B6
:1021700011420CBF0020012019420CBF002000F0CA
:1021800001007047C94389B201827047D0F8E43535
:1021900010B51B6904469847032384F812310020C8
:1021A00010BD08B5042380F81231D0F8E435DB689F
:1021B0009847002008BD08B5D0F8E035DB6903B1C9
:1021C0009847002008BD08B5D0F8E0351B6A98474D
:1021D000002008BD08B5D0F8E0355B6A98470020BC
:1021E00008BD002110B5402204460B4600F0C6FF92
:1021F000802140220023204600F0C0FF012384F804
:102200001231D4F8E435A0785B689847002010BDFF
:1022100037B56946044600F015F99DF800106D4683
:1022200001F01F03012B07D0022B0AD073B92046FF
:10223000694600F0C7F90FE02046694600F0A8F9AA
:102240000AE02046694600F031F905E021F07F01FF
:10225000C9B2204601F024F800203EBD38B504463E
:1022600000293DD190F81131022B42D1D0F8342110
:10227000D0F820319A4211D9C178D21A0129C0F878
:10228000342104D1D0F82411CB18C0F8243192B2F3
:102290002046D4F8241100F0A5F82AE0D0F838211F
:1022A000B2FBF3F503FB152565B99A420AD3D0F8C2
:1022B0003C319A4206D229462A4600F093F8C4F8E7
:1022C0003C5116E0D4F8E035DB682BB194F81221CC
:1022D000032A01D120469847204600F0A4F808E0E0
:1022E000D0F8E0355B6923B190F81221032A00D1C0
:1022F0009847002038BD10B5044659BB90F81131FD
:10230000032B30D1D0F88C23D0F878339A4214D9EB
:10231000C178D21A0129C0F88C2304D1D0F87C13DB
:10232000C918C0F87C139A4228BF1A4692B22046B8
:10233000D4F87C1300F05FF815E0D0F8E0351B69A5
:1023400023B190F81221032A00D19847204600F0CB
:102350005BF808E0D0F8E0359B6923B190F81221D2
:10236000032A00D19847002010BDF8B50446164650
:102370001F460D46FFF762F9069B2046C4F8E43578
:102380002946C4F8E075C4F8E86500F0ABFED4F85F
:10239000E4351B6898472046FFF78CF9F8BDD0F864
:1023A000E03510B51B6804469847D4F8E4359B68BF
:1023B0009847002010BD08B5D0F8E0355B68984715
:1023C000002008BD08B58C461346C0F83821C0F877
:1023D0003421022280F811210021624600F03EFFE4
:1023E000002008BD8C4608B500211346624600F067
:1023F00035FF002008BD8C4608B500211346624613
:1024000000F004FF002008BD0021042310B50A4697
:10241000044680F811310B4600F020FF204600F002
:1024200041FE002010BD0021052310B50A460446D8
:1024300080F811310B4600F0E9FE204600F032FE34
:10244000002010BD90F8C8350B7090F8C9354B705E
:1024500090F8CB2590F8CA3503EB02234B8090F817
:10246000CD2590F8CC3503EB02238B8090F8CF2557
:1024700090F8CE3503EB02239BB2CB80C0F83C3101
:10248000012380F81131704710B591F900300446EE
:10249000002B01DBCB8813B92046802100E000210E
:1024A00000F0FEFE204600F0FDFD10BD38B50D46E3
:1024B0006B780446012B097916D033D3032B63D1F3
:1024C00090F81231022B34D0032B59D16B88FBB911
:1024D0000B1E18BF012380290CBF002303F001034A
:1024E000B3B100F0DDFE13E090F81231022B20D0E2
:1024F000032B45D16B88002B46D10B1E18BF01233F
:1025000080290CBF002303F001033BB100F0E9FE7A
:10251000D4F8E03520469B68294698472046FFF7C7
:1025200073FF31E090F81231022B02D0032B27D138
:102530000CE00B1E18BF012380290CBF002303F001
:1025400001030BB3204600F0ABFE1DE011F0800F3D
:1025500007D001F07F01282303FB010191F81A2124
:1025600004E0282303FB010191F87223074B02B119
:1025700001221A60204605490222FFF723FF03E0EB
:1025800020462946FFF780FF002038BD981500201F
:1025900038B590F812310446032B0D460CD10B7957
:1025A000012B09D8D0F8E0359B689847EB883BB9F8
:1025B0002046FFF729FF03E020462946FFF764FF86
:1025C000002038BD73B54B7804460D46092B00F248
:1025D0001C81DFE813F0D30010011A01E3001A0197
:1025E00072000A001A01C00092004B881A0A013AD0
:1025F000062A00F20A81DFE812F007001A0027001D
:102600000801080108010801D4F8E8350DF10601B8
:102610001B68A0789847EB880146402B03D094F8BC
:102620001231012B3AD10822ADF8062036E0D4F859
:10263000E0350DF106019B6AA078984702234370AC
:102640000146C4F8EC0529E0DBB2052B00F2DD8081
:10265000DFE803F003080D12171CD4F8E835A07862
:102660005B6817E0D4F8E835A0789B6812E0D4F8EE
:10267000E835A078DB680DE0D4F8E835A0781B6970
:1026800008E0D4F8E835A0785B6903E0D4F8E835D1
:10269000A0789B690DF1060198470146BDF8063008
:1026A000002B00F0B680EA88002A00F0B2809A423F
:1026B00028BF1A46ADF806205EE08B88002B40F05C
:1026C000A480CB88002B40F0A08094F812214B8886
:1026D000032A00F09A8003F07F05204684F8135106
:1026E000294600F01DFE2046FFF78EFE0DB10223A5
:1026F00000E0012384F812318BE08978464E0129ED
:10270000317000F2828094F81231022B02D0032B38
:102710007BD108E000294CD00121032384F810115B
:1027200084F8123113E041B9022384F8123184F89D
:1027300010112046FFF73FFE3BE094F810110129ED
:1027400037D02046FFF737FE317884F81011204645
:10275000FFF725FE2DE0CA88012A56D194F81231E0
:10276000022B02D0032B50D104E02C492046FFF766
:1027700029FE4EE004F588712046F8E794F81231FE
:10278000023B012B41D8D4F814312549002B0CBF52
:10279000012303230B6020460122E8E74B88012B2D
:1027A0000BD1C4F81431D4F8E03520469B68294693
:1027B00098472046FFF728FE2BE0022B29D18B8873
:1027C00013F0FF0F25D121691B0A013B4A68042B36
:1027D0000FD8DFE803F0030507090B00012306E02B
:1027E000022304E0032302E0042300E0052363F353
:1027F00006124A60DDE794F81231023B012B04D83F
:102800004B88012B05D1013BCBE720462946FFF73A
:102810003BFE00207CBD00BF941500209C150020CD
:102820009015002010B5D0B18446002300E0DBB243
:102830001CF8014B0133002CF9D15B009BB21380D3
:102840000B7003234B70013B05E0CA545A1CD2B2F3
:1028500002338C54DBB210F8012B002AF5D110BDE5
:1028600073B50024114D064601940320FEF730FF96
:10287000336801341A69AC42019215D0019A002ADA
:10288000F3DA019A42F001020192019A1A61074AB1
:10289000196912F1FF32019103D0019911F0010F72
:1028A000F6D10320FEF714FF00207CBD410D03008C
:1028B00010B5C47874B900EB820003339B10D0F8D4
:1028C000D000224604E051F804CB0132C0F800C029
:1028D0009A42F8D3002010BD0332D0F8D0C010B512
:1028E00092100846002304E0DCF80040013340F871
:1028F000044B9342F8D301EB820010BD012270B566
:102900000023827040220129C37082800CD10833D9
:102910000370042343704FF4A073C3800223037237
:10292000C1724FF0A04309E041B90C2303700623A4
:1029300043704FF4A062224BC172C280457803F508
:10294000006201350261C36001466D01002203F59A
:102950000E6403F52E6C04E0A6184E610CEB020623
:102960000E6520320431AA42F6D1014611F88CCB13
:1029700003F58062426103EB4C1403F58862C0F8F2
:10298000CC2004F5A06403F5A06202E041F8042F16
:102990002032A242FAD103EB0C3C00F1CC010CF541
:1029A000805C1A4601E041F8042F02F5805262452E
:1029B000F9D103F56063C0F80C31002070BD00BF91
:1029C0000000044038B5037A0025012B0446C26894
:1029D00026D1936B417A65F3104309B143F4801318
:1029E0009363D36804F10C006FF386136FF396536F
:1029F00043F010036FF3C3036FF3C7136FF3514337
:102A00006FF3D343D360FFF72BFFE378012B40D163
:102A1000043363F34405E36845F020059D6038E026
:102A2000D36800F10C0043F04003D360FFF718FFB8
:102A3000237A627A032B14BF4FF434134FF43C1300
:102A40000AB143F48013E26814209363FEF745FE55
:102A5000E268217AD368032908BF43F48033D36046
:102A6000237A032B15D1156B012363F39B656FF359
:102A7000D7552C3345F0805563F316451563C820B0
:102A8000FEF72BFEE36845F400051D63C820FEF742
:102A900024FEE378012B07D1E36805229D6862F3E9
:102AA000440545F020059D60002038BDC368002026
:102AB0009A6842F001029A607047C36800209A68E1
:102AC00022F001029A60704707B500230193019A32
:102AD00042F020020192019A61F38A120192019957
:102AE000C26811610749106901338B42019003D01C
:102AF000019810F0200FF6D10320FEF7E9FD002029
:102B00000EBD00BF410D030007B500230193019ADC
:102B100042F0100201920199C268116107491069DF
:102B200001338B42019003D0019810F0100FF6D1C1
:102B30000320FEF7CDFD00200EBD00BF410D0300B8
:102B4000C26808B5D36801296FF35D736FF39E7394
:102B500008BF43F0005302D009B943F0804332204C
:102B6000D360FEF7BAFD002008BDC3685B6913F0AF
:102B7000010F14BF002001207047C3685A6998698B
:102B80001040704703691A6861F301021A607047C8
:102B9000C26800239361013B5361536053610B4B47
:102BA0009361C3789169002B14BF4FF400634FF415
:102BB000016343F4701343F4405343F0080321EAE4
:102BC000030141EA0303936100207047000800807D
:102BD00038B5D0F80C3100221A60036915461A681E
:102BE000044665F3CC221A60C37A012B1AD1032163
:102BF000FFF7C8FFE36880214FF4800261F30F0202
:102C000059629A62C02262F30F0561F31F455218A0
:102C1000C3F8045162F30F056FF31F45C3F8085161
:102C2000C3F80C5110212046FFF74EFF2046FFF756
:102C30006BFF226900234FF0FF31136104F1140090
:102C400053619E4691614FF0FF0CD36112E050F842
:102C5000042F01331168C1F3076101F08001C9B28B
:102C6000002914BF4FF0904100211160C2F810E01C
:102C7000C2F808C062789342E9D3002304F15000FF
:102C80009E464FF0FF0C12E050F8042F01331168FC
:102C9000C1F3076101F08001C9B2002914BF4FF0F0
:102CA000904100211160C2F810E0C2F808C06278BB
:102CB0009342E9D32269136943F480731361E37883
:102CC000012B08D14021023361F38A0343F480339E
:102CD00061F3594313632046FFF75AFF002038BDC4
:102CE00003699B68C3F341035A1E022A04D8034AAE
:102CF000D31813F8010C00E003207047983A00083D
:102D000003698169D3F808C00A68CCF3410002283E
:102D100018BF6FF30A0202D1032060F30A020A60AF
:102D20005A68002042F480725A60704710B54C789F
:102D30000022012C0B7808D100EB830C14FA03F36A
:102D4000DCF818C063F30F0208E0012400EB830CE9
:102D500014FA03F3DCF854C063F31F42DCF80030CC
:102D6000C3F3072404F08004E4B274B98C6864F3FC
:102D70000A03CC78C98864F3934361F3995343F011
:102D8000805343F40043CCF8003003690020D96934
:102D90000A43DA6110BD10B54C784FF0000C012CDD
:102DA00062460B7807D100EB830114FA03F38969BB
:102DB00063F30F0207E0012400EB830114FA03F32D
:102DC000496D63F31F4203696FF3CF3CC1F800C044
:102DD000D969002021EA0202DA6110BD38B54D78C8
:102DE0000B78012D4C6955D100EB8303D3F818C043
:102DF000DCF80030DCF8102024B964F3120265F32B
:102E0000DC420DE08D6864F312026419013CB4FBEE
:102E1000F5F5CC7865F3DC42012C08BF64F35E72F3
:102E2000CCF81020C278012A08D10A78D1F810C055
:102E300000EB82029269C2F814C00FE0CA78012A3E
:102E40000CD04A6952B191F800C0012505FA0CFC7A
:102E50000269546B4CEA040CC2F834C0CA78012AE7
:102E600008D10269926812F4807F0CBF43F00053CE
:102E700043F080530A7843F0044300EB82029269E6
:102E80001360CB78012B3ED10A788B8AC968FFF793
:102E90000FFD38E000EB83035D6DD1F808C02B68AF
:102EA0002A6934B96CF312024FF0010C6CF3DC4266
:102EB0000BE06444013CB4FBFCF4A405A40D0CFB42
:102EC00004FC64F3DC426CF312022A61C278012A2A
:102ED00001BF0A78D1F810C000EB8202526D08BF22
:102EE000C2F814C0CA78012A06D14A7912B143F057
:102EF000005301E043F080530A7843F0044300EBB1
:102F00008200426D1360002038BD73B54D784C6966
:102F1000012D45D1D0F818C0DCF80030DCF81020C5
:102F2000009254B99DF8002064F306028DF8002049
:102F30009DF8022065F3C40210E08D689DF8002022
:102F4000AC4286BF4D6165F3060264F306028DF85C
:102F500000209DF80220012464F3C4028DF80220B1
:102F6000009A43F00443CCF81020C278012A01BF34
:102F70000A780C6900EB8202926908BF5461CCF8B0
:102F80000030C378002B45D14B69002B42D00A7822
:102F9000012111FA02F20369586B02435A6339E0C6
:102FA0000B7800EB8303D3F854C0DCF80030DCF876
:102FB00010500095EAB2C5F307468D684CB965F329
:102FC00006028DF80020012262F3C4068DF802602B
:102FD0000AE065F306024D618DF8002035460122B6
:102FE00062F3C4058DF80250009A43F00443CCF814
:102FF0001020C278012A01BF0A78D1F810C000EB76
:103000008202526D08BFC2F814C00A7800EB820039
:10301000426D136000207CBD4B78012B0B780CD1E6
:1030200000EB830082691368C3F3076101F080013C
:10303000C9B231B143F0804303E000EB8300426D3D
:10304000136843F400131360002070474B78012B82
:103050000B78C9780BBF00EB830000EB830083691A
:10306000436D02391A68C9B26FF35552012998BFEE
:1030700042F080521A600020704703699A69D8694B
:103080001040000C704700EB81014B6D02699B689A
:1030900050691840704703699869DB69184080B22D
:1030A0007047000082B000230093C0338DF80330D6
:1030B0000122002362F3C4038DF8023018238DF837
:1030C0000030436D009A1A61C278012A01BF00F5F1
:1030D000B96058611A68024A08BF1A6002B07047A6
:1030E0000080008038B50446FFF708FC012000216D
:1030F00084F81201054684F8131194F801C02346A0
:10310000224608464FF0400E0EE082F8F010A2F87A
:10311000F61082F8F15082F8F300C2F8F8E0C2F835
:10312000FC00C2F80401013128326145EDD30022D0
:10313000114640200EE083F84823A3F84E2383F87D
:10314000491383F84B13C3F85003C3F85413C3F85F
:103150005C13013228336245EDD32046FFF7ADFC06
:103160002046FFF72FFC00212046FFF7E9FC204610
:10317000FFF72EFD2046FFF799FC38BD10B5CCB205
:1031800014F0800F14BF4FF0280E4FF0280E8C461D
:1031900001F07F0115BF0EFB01F10EFB01F101F5FE
:1031A0008C7101F55C7141180CF07F0CE40981F819
:1031B00000C04C708A60CB700CB1A1F806C0022B25
:1031C00001D100230B71FFF7B1FD002010BDCAB281
:1031D00012F0800F14BF4FF0280C4FF0280C08B5E8
:1031E00001F07F0315BF0CFB03F30CFB03F303F5A6
:1031F0008C7303F55C73C318D20901F07F01197059
:103200005A701946FFF7C7FD002008BD08B54FF0FA
:10321000280C01F07F0E0CFB0EFC0CF55C71844455
:10322000CCF8843300238CF870E38CF87133CCF83D
:103230008833C3784118012B08BFCCF8802328239A
:1032400003FB0E0E9EF87033CCF87C2313B9FFF706
:103250005CFE01E0FFF7C2FD002008BD10B54FF095
:10326000280C01F07F040CFB04FC0CF58C718444E9
:103270004FF0010ECCF82421CCF82821002241186F
:103280008CF819E18CF81841CCF83021CCF82C31AD
:1032900014B9FFF73AFE01E0FFF7A0FD002010BDD2
:1032A000CAB212F0800F08B508D001F07F034FF0CA
:1032B000280C0CFB03F303F58C7303E028234B432A
:1032C00003F55C73C3184FF0010CD20901F07F01C4
:1032D000197083F802C05A701946FFF79DFE00204E
:1032E00008BDCAB212F0800F10B508D001F07F03FC
:1032F0004FF0280C0CFB03F303F58C7303E0282339
:103300004B4303F55C73C3180024D20901F07F011D
:1033100019709C705A701946FFF798FE204610BD30
:103320000369002261F30A1219680A431A607047A0
:1033300008B5036903205A686FF341025A60FEF72B
:10334000CCF908BD08B5036903205A6842F00202AF
:103350005A60FEF7C2F908BDF0B587B00446FFF722
:1033600004FC002800F06C822046FFF706FC029067
:10337000002800F06482C0F3074000F00800C0B2EB
:10338000002864D02046FFF778FE039000202746EF
:103390002646049057E0039911F0010F48D0049B92
:1033A0002046DAB211460192FFF76DFE10F0010FD0
:1033B0000546019A21D0736D01259D60E178A942EF
:1033C00007D11B69D7F87813C3F31203CB1AC7F8D8
:1033D0008833DFF870C42046DCF8003011461B68E3
:1033E0009847E378012B08D1049830B994F811314B
:1033F000052B02D12046FFF755FE05F00203DBB294
:1034000013B1736D02259D6005F00403DBB213B1A7
:10341000736D04259D6005F00805EDB245B1DFF838
:10342000241420460B689B689847736D08229A60A5
:10343000049BDDF80CC001334FEA5C0C0493CDF81B
:103440000CC00436283703980028A4D10130029913
:10345000C1F3074303F00403DBB2002B00F0C68086
:103460002046FFF718FE00220490254627460392C7
:103470002646B5E0049B13F0010F00F0A6803369E7
:10348000DDF80CC019695C6B5FFA8CFC24FA0CF453
:1034900006EB8C029269E401926804F0FF040C438D
:1034A000144014F0010FCDF814C01DD0DDF80CC08D
:1034B000012000FA0CF15A6B044622EA01025A6319
:1034C000AB6905999860DF48036830465B689847A8
:1034D000F378A34208D1039931B996F81131042B3E
:1034E00002D13046FFF7DEFD04F00403DBB213B176
:1034F000AB6904249C6004F00803DBB213B1AB6930
:1035000008249C6004F01003DBB213B1AB691024F3
:103510009C6004F02003DBB213B1AB6920249C60F3
:1035200004F04003DBB213B1AB6940249C6004F0AB
:103530000203DBB213B1AB6902249C6024F07F0468
:1035400014F0FF0F41D0D7F83031D7F82CC1C3EBBE
:103550000C0CD7F820319C4528BF9C460CF1030C7D
:10356000AB694FEA9C0C64469B69B4461EE0D7F8F1
:1035700020219E1B964228BF1646B3B26046D7F85C
:103580002411059ACDF804C0FFF792F9D7F8243139
:10359000F41C9B19C7F82431D7F83031DDF804C08A
:1035A0009E19AB69C7F830619B69A4089BB2A3421E
:1035B00007D9D7F83061D7F82C319E4201D2002BC1
:1035C000D5D1AB69802266469A60039BDDF810C0B6
:1035D00001334FEA5C0C0393CDF810C00435283753
:1035E000049800287FF446AF34460130029901F078
:1035F0000203DBB213B1E36802225A61029AC2F3FA
:10360000076303F08003DBB2CBB1A37A43B1D4F8F4
:103610000C31D4F80C216FF341036FF300031360F6
:10362000236920465A6822F001025A60854B1B68C4
:103630009B699847E3684FF000425A610120DDF82A
:1036400008C0CCF3072303F00803DBB2FBB17D4BCA
:1036500020461B685B6998472369E2684FF4006164
:103660009B685161A27A8AB113F0010F0ED0D4F891
:103670000C311A6842F001021A601A6842F0030223
:103680001A60714B1A6942F006021A610120029910
:1036900001F00803DBB243B16A4B20461B68DB68CC
:1036A0009847E36808225A610120029A02F0100349
:1036B000DBB2002B3AD0E3689A6922F010029A61DB
:1036C0001D6AC5F34343022B05F00F0602D0062BFB
:1036D00026D115E047F6F07305EA030303B3282368
:1036E00003FB0646C5F30A152046D6F87C132A4686
:1036F000FFF7F2F8D6F87C335B19C6F87C330AE0A2
:1037000004F5B96120460822FFF7E6F8282303FBF9
:103710000646C5F30A15D6F88833ED18C6F888535F
:10372000E36801209A6942F010029A61DDF808C04E
:10373000CCF3072303F01003DBB2002B36D0236950
:1037400000255A68294622F001025A602046FFF7F8
:10375000BBF904F114022B46FF2105E052F8040FD7
:1037600001338160D06B816060788342F6D3236936
:1037700001264FF0FF3266F30F059A6166F31F458D
:103780001032DD615A6120321A611A6820466FF3E7
:103790000A121A60FFF786FCE3684FF480525A6100
:1037A000284B20461B681B69984730460299C1F395
:1037B000072303F02003DBB2EBB12046FFF7A0FAAA
:1037C000E3682046DD68FFF78BFA032806D1002363
:1037D0004FF40072A370A280093304E00123A370A8
:1037E0004023A380052363F38D25E3684FF4005243
:1037F000DD6001205A61DDF808C0CCF3074303F017
:103800001003DBB24BB10F4B20461B68DB699847B6
:10381000E3684FF480125A6101200299C1F3074313
:1038200003F02003DBB25BB1064B20461B681B6A2A
:103830009847E3684FF400125A61012000E00298B3
:1038400007B0F0BD0400002000ED00E0002305E01B
:1038500011F803C0013A00F803C00133002AF7D180
:10386000704700000004024004000000000C024009
:10387000000800000004024000100000000C02409C
:10388000000400000000024000800000000402402C
:1038900000010000FFFFFFFF00000000000000002B
:1038A0000040000808000000000000000080000840
:1038B000100000000000000000C000081800000018
:1038C00000000000000001082000000000000000CF
:1038D00000000208280000000000000000000408AA
:1038E0003000000000000000000006083800000062
:1038F0000000000000000808400000000000000078
:1039000000000A08480000000000000000000C0849
:10391000500000000000000000000E0858000000E9
:10392000000000000000020303010203030303037D
:10393000020203014D494F5333320053544D333289
:103940004634444953434F564552590053544D331E
:1039500032463478780025303878003F00256400FE
:103960004D494F53333220426F6F746C6F61646501
:103970007200286329203230313220542E204B6CC3
:103980006F7365002025303258002020200025303C
:1039900038582000F000007E320000007514000846
:1039A000811400088D1500088D14000855150008B5
:1039B000251500082D15000809160008DD1500085A
:1039C0003F1500080000000043150008CB15000853
:1039D000B915000800000000000000000000000011
:1039E0004915000804030904120100020000004008
:1039F000C016FE0310100102030100003515000877
:103A000037150008FD1500083B1500083D15000896
:103A100039150008F31500083432006D69646962D5
:103A20006F782E6F72670000090265000201008046
:103A3000320904000000010100020924010001090B
:103A40000001010904010002010300020724010032
:103A500001410006240201010006240202020009BD
:103A600024030103010201000924030204010101EE
:103A700000090502024000000000052501010109BE
:103A8000058102400000000005250101030000003F
:103A9000286E756C6C290000020102000000000015
:103AA0001010000008000020F72200085D22000826
:103AB00011220008B7210008E3210008A321000813
:103AC0008D210008C7210008D52100080000000052
:103AD0000000000000000000FFFFFFFFFFFFFFFFEE
:103AE000FFFFFFFFFFFFFFFFFFFFFFFFFFFFFFFFE6
:103AF000FFFFFFFFFFFFFFFFFFFFFFFFFFFFFFFFD6
:103B0000FFFFFFFFFFFFFFFFFFFFFFFFFFFFFFFFC5
:103B1000FFFFFFFFFFFFFFFFFFFFFFFFFFFFFFFFB5
:1040000000000220415800088B580008B14D0008FC
:104010008B5800088B5800088B58000800000000DF
:10402000000000000000000000000000F95400083B
:104030008B580008000000006D550008A9550008C5
:104040008B5800088B5800088B5800088B580008C4
:104050008B5800088B5800088B5800088B580008B4
:104060008B5800088B5800088B5800088B580008A4
:104070008B58000809800008E97F00088B58000869
:104080002D8500088B5800088B5800088B580008B5
:104090008B5800088B5800088B5800088B58000874
:1040A0008B5800088B5800088B5800088B58000864
:1040B000258B0008498B00088B5800088B58000896
:1040C0008B58000831970008F59800088B580008B5
:1040D0008B5800088B58000875960008D196000888
:1040E0008B5800088B5800088B5800088B58000824
:1040F0008B5800088B5800088B5800088B58000814
:104100008B5800088B5800086D8B00088B580008EE
:104110008B5800088B5800088B5800088B580008F3
:104120008B5800088B580008C97F00088B5800087E
:104130008B5800088B5800088B5800088B580008D3
:104140008B5800088B5800088B580008B98E00085F
:104150008B5800088B5800088B5800088B580008B3
:104160008B5800088B5800088B5800088B580008A3
:104170008B5800088B5800088B5800088B58000893
:084180008B5800088B58000861
:10418800F7B500F0D5FF019001A8012101F0E6F88C
:104198003F4B40491F78404B00221E880846134673
:1041A8003E4D21E0072B23D830F902EBBEF1000F7A
:1041B80019DA3B4C04F803C015F902C0394C0CFB62
:1041C80006FC24F813C00133BEF1FF3F02BFDFF83D
:1041D800D8C00EF1010E4FF6FE74DBB204BF4CF8E6
:1041E80022E020F8024C01325FFA82FCBC45D9D3A8
:1041F8002E4A1278D2F1010238BF0022072B98BF4D
:1042080042F00102002A3FD0214A24481678224A67
:104218001588002234E0072B36D831F802EB0FFA64
:104228008EF7002F2BDD1E4F1E4C07F803C010F829
:1042380002C00EF1FF3E4FFA8CF76F431FFA8EFE55
:1042480024F8137001331EF0070F08BF184F21F828
:1042580002EC08BF17F802E0DBB204BFCEEB0C0C8F
:1042680000F802C010F902C0BCF1000FDFBF4FF028
:10427800000C4FF0000E00F802C021F802EC0132E9
:104288005FFA82FCB445C6D30A4A13707CE700BFC4
:10429800A4560020204B0020020000204C420020A1
:1042A800C44C00208C420020C44B0020CC4C002081
:1042B8000C420020C04B0020F8B5134F05460E46AF
:1042C80007EB4517114802F041FA3146384609F024
:1042D800E3FB0446384609F05BFC002C04DA21466F
:1042E8000B4802F033FA0CE00A4B002243F8252071
:1042F800BB68094A094842F825302946324602F087
:1043080025FA2046F8BD00BF2043002004DF00083E
:1043180014DF0008C44B0020E84000203BDF000801
:10432800F7B5144B054653F822600C46760A0196F9
:10433800009209F09DFB019B0746B3FBF0F61F2E88
:10434800009A88BF4FF0FF3012D80B4B06EB421291
:1043580053F8220009F092FB019B294607FB163609
:10436800801902F0CBFF0028ACBF20466FF0010097
:10437800FEBD00BFC44B002068110020F7B54A4BB2
:1043880003F5806200280CBF1E461646474B1B7873
:1043980033B91A46F2500433B3F5806FFAD182E08C
:1043A80004F01AFC0120014604F02EF9404A137863
:1043B8001A46002B6ED000243E4D3F4F3FE03F4A47
:1043C8004FF4007102EB44202A5DFFF7A9FF002893
:1043D80006DA2B5D002227F81320394B23F8142026
:1043E8002B5D384951F8232002F5007241F823204B
:1043F800354951F823108A4202D3002227F81320A6
:1044080004F0F4FB2D2804F1010417D9284D0A22E1
:104418002B78B0FBF2F102FB110200932B482346E4
:1044280002F094F92C70224B294A93F800E0234CAF
:10443800012302EB4E0E47F6FF7C27E0E4B21C4A4C
:104448001378A342BBD8EEE70F7811F8015C01F5A9
:10445800007105EB072530F9027F2DB207FB052215
:104468007045F1D1D2136245C8BF47F6FF7203DC2D
:1044780018498A42B8BF0A46120442EA124246F86C
:10448800042B023340F20122934208D01048E1186D
:104498000022E5E7F2500433B3F5806FFAD101202A
:1044A800002104F0B1F8FEBD68310020E841002089
:1044B800C04B0020C44C0020204B00206801002085
:1044C8008C420020C44B0020E84000206FDF000829
:1044D8008A4200200080FFFFF0B5684B9DB07F2224
:1044E80016AC1A801AAD06466549204609F031FC1B
:1044F80032462846634905F077FB2946204609F0ED
:104508000EFC0120014604F07FF85F4B00251D706A
:104518005E4B01221A7021465D4802F017F95D488A
:10452800214609F0B9FAA84203DA5B4802F00EF90D
:104538009DE006AEB31C594F2C46049330463F21EC
:1045480009F074FB002836D000211022049800F0EE
:10455800C7FCDFF84CC1002145F80C000A22701D89
:1045680000F0BEFC4F4A00211055F01D0A2200F051
:10457800B7FCDFF834C1C3B20CF8043013B1434AB6
:104588000021117006F10C011E223846039309F030
:10459800EFFB039B434A0093135DDFF804C10193CB
:1045A8003A4655F80C304148214602F0CFF8364BD0
:1045B8001A7801321A7001341E370435402CBDD1E7
:1045C800344809F0E5FA00244BE0344B1E2101FB86
:1045D80004312046FFF770FE054618B1344802F052
:1045E800B5F838E009F044FA324B334A400203EB9D
:1045F800C413059004932E4602EB4417DFF8BCC0A1
:104608005CF824309D4226D2384609F089FA002801
:1046180021DB284609F0D8FA0028034605DB0DF10E
:104628006F00012109F0E0FA03463846039309F0C8
:10463800AFFA039B002B0EDB049B3A69314643F823
:10464800042F1F480493013602F080F8DDF814C0E7
:10465800202E6544D2D11B4B002223F814200134AC
:10466800E4B2DFF824C09CF80030A342ADD80120A2
:10467800002103F0C9FF1DB0F0BD00BF02000020FB
:1046880008000020ADDF0008A4560020CC4C002014
:10469800B0DF0008EC410020C5DF000868390020C1
:1046A800A8560020A0420020E0420020DFDF0008DA
:1046B8002CE000086411002020430020E84000207E
:1046C80045E00008204B002010B5002420460134A6
:1046D8000421E4B203F0F8FF082CF7D103F0F7FF48
:1046E800C0B27F2812D0BF2808BF204619D0DF28C3
:1046F8000ED0EF280ED0F7280ED0FB280ED0FD28BC
:104708000ED0FE2814BF012002200AE0092008E08C
:10471800072006E0062004E0052002E0042000E06F
:10472800032010BDF7B500F003FD02AC114F124E87
:10473800124D44F8040D2046642100F00FFE104A83
:104748001378002BF7D0FFF7BFFF3B780146834271
:10475800F1D0387030700B4801F0F8FF00230A4898
:104768002B7001F0F3FF3078FFF7B6FE01232B70B2
:10477800E1E700BF0400002005000020E841002018
:104788009C420020F9E0000855E00008F0B52249F5
:1047980089B0224801F0DAFF21481F4909F07CF965
:1047A8000028A4BF01AE1F4F03DA1F4801F0CEFF57
:1047B80030E03046192109F039FA40B31B49304638
:1047C80009F0EAFA1A490546002009F0E5FA044614
:1047D80029462246174801F0B9FF1749284609F02B
:1047E800ADFA014620B920460A2200F079FB38705C
:1047F8001249284609F0A2FA01460028D9D12046D4
:104808000A2200F06DFB0E4B01381870D1E70448FE
:1048180009F0BEF909B0F0BD84E000086DE00008B9
:10482800A04B00209C4200208FE000086AEB0008A3
:1048380087E20008ABE00008C7E00008CEE0000807
:1048480000000020F8B5DFF8FCC0C1F303249CF891
:1048580000C0C1F307420CF1FF3C080E6445D3B217
:104868006ED101F00F0CACF10804E4B2012C4AD867
:10487800C1F3072101F0F001902900D148B9324A6B
:1048880000211578314ADFF8C8C0177831480A4640
:1048980035E02D4A304915782E4C0022DFF8BCC08F
:1048A8002F4F2E460BE051F8045FAB4201BF4FF08B
:1048B800FF3524F812503D5C0CF802500132D5B295
:1048C800B542F0D33CE0274EB45CB4B95CF8224062
:1048D800A34212D127B9244CA65C0EB1445E14B988
:1048E8000026465209E01D4C4652A456F6080136E9
:1048F80094FBF6F61D4C0136A65401320231D4B2AF
:10490800AC42E0D31CE0BCF10C0F11D1184C194695
:104918002270184D184801F019FF00232B70174812
:1049280001F014FF2078FFF7D7FD01232B7007E073
:10493800134B144A01EA0303934204BF124B188035
:10494800F8BD00BF00000020A4560020CC4C002079
:10495800A8560020204B0020A45600204C420020DE
:1049680084DE0008A0420020E04200200C42002023
:1049780005000020E8410020DAE0000855E00008C2
:104988000F00FF000B00070002000020704770476F
:104998007047000008B54FF40071024A024803F05E
:1049A800A3FD08BD85430008683100201FB54FF0FE
:1049B800FF3003F0E3FD2D4B01221A702C4801F063
:1049C800C5FE2C4801F0C2FE2B4801F0BFFE0020B6
:1049D80009F02CF8002802DA284801F0B7FE002474
:1049E800002002F043FC002806DC0134B4F57A7F8D
:1049F800F6D1234801F0AAFEFFF7C8FE214B1B7829
:104A080033B1214801F0A2FEFFF75EFE1F4B18707C
:104A18001E4B00241878FFF75FFD1D4801F096FE35
:104A28001C4B01221A700020FFF7B4FF1A4801F04E
:104A38008DFE642004F0A8F8032300931749234649
:104A48004FF48072164801940294039400F078FAA7
:104A58000223009313494FF48072234612480194AD
:104A68000294039400F06CFA1FBD00BFA857002001
:104A78000DE100082EE1000857E100086EE100088A
:104A880089E100089C420020ABE1000805000020F5
:104A9800BEE10008E8410020D4E10008E5E1000893
:104AA80089410008F0E100082D4700087047704769
:104AB800704708B501F084F8FFF769FF08BD0000EA
:104AC80013B500F035FB02AC44F8040D0121204673
:104AD80000F044FC00F02CFB019A431F9A4238BFB7
:104AE800019002F043F8024801F07EFEEEE700BFB5
:104AF8004D48000813B500F01BFB02AC44F8040D48
:104B08000121204600F02AFC00F012FB019A431F05
:104B18009A4238BF0190064800F0E6FF054801F0C8
:104B280095F9054804F09DF802F0A7F8E8E700BFFA
:104B380099490008B74A0008B94A000830B500206A
:104B480085B002F03DFD002004F05EF8002003F07F
:104B58000BFD002003F076F8002000F0EFFE0020A7
:104B680000F084FF002000F0EFFF002000F0FAFFC3
:104B7800002002F05BFA002004F072F8002002F036
:104B880052FA002004F0AEF9002001F0ABFA002040
:104B980002F03AF8002002F03DF8002001F0BEF9DA
:104BA800002003F0EBFA09F083F8FFF7FFFE01F0AD
:104BB8005DFA4FF4FA644FF47A7004F045F814F192
:104BC800FF34F8D1032523460C494FF480720C4872
:104BD800009501940294039400F0B2F909494FF446
:104BE800807223460848009501940294039400F0CB
:104BF800A7F900F071FA204605B030BD05E20008BB
:104C0800FD4A000800E20008C94A000808B5FFF795
:104C1800BDFE024800F0EEFE08BD00BFBB4A00081A
:104C280008B5FFF743FF08BD70B50024642642F2BB
:104C380010750134B4FBF6F306FB13430BB901F00E
:104C480095FF084801F0D0FDB4FBF5F305FB1343CD
:104C5800002BEED103F01CFDC143012003F0D4FC6E
:104C6800E7E700BF4D48000810B5036888B0079310
:104C78004368374C069383680593C36804930369B4
:104C880003934369029383690193C36920460093A0
:104C980001F05CFD2F4801F059FD204601F056FD5A
:104CA80007992D4801F052FD06992C4801F04EFD58
:104CB80005992B4801F04AFD04992A4801F046FD60
:104CC8000399294801F042FD0299284801F03EFD68
:104CD8000199274801F03AFD0099264801F036FD70
:104CE800254B2648196801F031FD254B25481968E0
:104CF80001F02CFD244B2548196801F027FD244BB1
:104D08002448196801F022FD234B2448196801F052
:104D18001DFD6FF07F4001F0DCF9002001F0DDF9A6
:104D2800002001F0BBF801F05FF90020014601F016
:104D3800BBF81B4801F08CF90121002001F0B4F800
:104D48000199184801F0B2F9FFF76EFF08B010BDDD
:104D580061E2000875E2000889E2000894E20008B0
:104D68009FE20008AAE20008B5E20008C1E20008D4
:104D7800CCE20008D7E2000838ED00E0E3E20008E2
:104D880028ED00E0F0E200082CED00E0FDE200086C
:104D980030ED00E00AE300083CED00E017E300080E
:104DA80024E3000835E300081EF0040F0CBFEFF3FE
:104DB8000880EFF30980FFF757BF7047F0B587B059
:104DC8000492464A0F4612680846039210F8012BCF
:104DD800039C014604EB020C9CF8015015F00805F1
:104DE800F4D12D2A03D111F8012B012503E02B2A38
:104DF80008BF11F8012BD3F1010038BF0020102B98
:104E080014BF044640F00104BCB1302A10D191F817
:104E180000C0BCF1780F14BF00240124BCF1580F66
:104E280008BF44F001041CB14A781023023104E0A1
:104E380018B1302A14BF0A230823002D0CBF6FF0C5
:104E480000404FF00040B0FBF3FC03FB1C000024C3
:104E5800059001952046039EB5186D7815F0040F4E
:104E680001D0303A08E015F0030F22D015F0010FF9
:104E78000CBF57253725521B9A421ADA604594BF52
:104E88000025012555EAD4740ED1059D604514BF4F
:104E980000240124AA42D4BF002404F001041CB950
:104EA80003FB0020013401E04FF0FF3411F8012B1F
:104EB800D1E7B4F1FF3F019D06D1002D0CBF6FF083
:104EC80000404FF0004001E005B14042049E1EB191
:104ED80004B14F1E049B1F6007B0F0BD6C0000209A
:104EE80008B58C4686461346002071466246FFF791
:104EF80065FF08BD0D4B10B51A68044650600C4A92
:104F08001268904206D20B4A10681968043100F002
:104F1800AAFA0AE0084A10681968043100F0A3FAEE
:104F2800064B1A68944238BF1C6010BD884D00209B
:104F3800A04D0020A44D0020E84C002018000020BF
:104F4800F0B587B0039048200491144605930C9E51
:104F58000E9F00F0E7FB0546002800F09B801FB974
:104F6800A00000F0DFFB07462F631FB9284600F0BA
:104F7800A3FB8FE0A2003846A52108F0C8FE2B6BE2
:104F880004991022671E05F1340003EB870708F027
:104F9800EFFE002385F843302C1D042E34BF334622
:104FA8000423EB626B642046019300F04CFA05F190
:104FB800180000F048FA019B27F00707C3F1050322
:104FC800AB612D616D6238460399059A00F080FA4D
:104FD8000D9B286003B11D6000F0AAFA304A1368DF
:104FE800013313602F4B1F68002F28D11D601368F1
:104FF800012B2CD12C4A133303FB072001370292D3
:10500800019300F015FA052F029A019BF4D1274B62
:10501800274F1846019300F00BFA384600F008FABB
:10502800244800F005FA244800F002FA234800F06A
:10503800FFF9019B224A1360224B1F6007E0224AB6
:10504800126822B91A68D26AB24298BF1D601F4A14
:10505800EB6A11688B4288BF13601D4A11680131E1
:1050680011601C4A11688B4288BF13600E4A1420D5
:1050780000FB0320214600F0E9F900F067FA124B23
:105088001B6853B1074B1B68DB6AB34205D200F0BB
:105098003FFA02E04FF0FF3000E0012007B0F0BD1A
:1050A800C84D0020884D00201C4D0020B04D002028
:1050B800084D00208C4D0020F44C0020D44C0020DA
:1050C800E84C0020A44D0020EC4C0020CC4D0020E2
:1050D800AC4D0020A84D002030B5002485B00C4808
:1050E8000C494FF48072234600940194029403946F
:1050F800FFF726FF0128054607D100F011FA064BF5
:105108001D60064B1C6000F067FA05B030BD00BF9B
:10511800FD52000842E30008EC4C0020A04D00209E
:10512800024B1A6801321A60704700BF804D002098
:1051380010B500F0FDF9034B1C6800F007FA204693
:1051480010BD00BFA04D00202F4BF7B51B68002BEA
:105158004ED12E4B1A6801321A601B68ABB92C4B22
:105168002C4A19681068186011602B4A11680131BF
:1051780011601A681168294A11B94FF0FF3303E02A
:105188001B68DB68DB685B681360204F234B3A6859
:105198001B689A4232D31E4D214C224E2B681B6845
:1051A80013B94FF0FF3206E02B68DB68DB6839681B
:1051B8005A68914202D2194B1A601FE01A1D104614
:1051C8000192009300F069F9009B9A6A22B103F1F9
:1051D800180000F062F9009BD86A23680199984288
:1051E80088BF2060142303FB006000F02FF9D5E787
:1051F8000D4B1A6801321A60FFF708FD0A4B1B684D
:105208000BB9FFF703FDFEBD804D0020A04D002027
:10521800E84C0020A44D0020844D002018000020F8
:10522800A84D00201C4D0020D04C0020F7B500F000
:105238007FF9284B1A68013A1A601D68002D43D17E
:10524800254B1C68002C40D0244F254E1DE0FB68E0
:10525800DC6804F1180000F020F9211D08460191CE
:1052680000F01BF9E06A3368019998421D4B88BF2A
:105278003060142202FB003000F0E8F81A4A136884
:10528800E26ADB6A9A4228BF01253B68002BDED11F
:10529800164C23682BB908E0FFF756FF2368013B3B
:1052A80023602368002BF7D107E0012D05D0104AB1
:1052B8001268012A18BF1C4607D10D4B00221A603C
:1052C80000F026F9012400E0002400F03FF9204610
:1052D800FEBD00BF804D0020C84D00208C4D002031
:1052E800A84D00201C4D0020884D0020D04C0020E7
:1052F800C44D0020F8B5154C154F164E1AE0FFF7AF
:105308000FFF3D68FFF792FFA5B100F011F9FB68A8
:10531800DD68281D00F0C1F83368013B336023685D
:10532800013B236000F012F9286B00F0C5F928460C
:1053380000F0C2F92368002BE1D1074A1368012B5A
:1053480001D900F0E5F8FFF76BFCF3E7F04C00201B
:10535800F44C0020C84D00201C4D002038B50C46E8
:105368000546FFF7DDFE124A2B681168E4189942DA
:1053780002D29C4208D201E09C4207D313689C42A7
:1053880094BF0023012302E0002300E001232C60E6
:105398003BB1084B1868043000F07FF82046FFF74F
:1053A800A9FDFFF743FF08B900F0B2F838BD00BF08
:1053B800A04D0020884D0020184B10B51B6833B154
:1053C8000122174B28E018680138186002E0154BD5
:1053D80015491422D3F800C0134802FB0CFC51F8FD
:1053E8000C40002CEFD00F4B4FF0140C19680CFB3D
:1053F80001FC00EB0C035A680CF1080C526860447D
:1054080082425A6004BF52685A60074B142202FB5A
:1054180001314B68DA68054B1A6010BD804D0020D9
:10542800C44D0020A84D00201C4D0020884D0020B0
:1054380000F108034FF0FF3282604360C3600361EC
:1054480000230360704700230361704743685A686C
:105458008B604A605A689160596003684160013303
:105468000861036070470A68B2F1FF3F0CBF036927
:1054780000F1080301D106E05B68D3F804C0DCF84A
:1054880000C09445F8D95A68086191604A6059602B
:105498008B600368013303607047436882689A60D1
:1054A8008268536003695968814208BF5A600022C4
:1054B80002611A68013A1A60186870470348006860
:1054C800006880F3088862B600DF00BF08ED00E0DE
:1054D800031F4FF0807C40F804CC181F43F8041CCD
:1054E800002140F8041C40F8182CA3F13C00704738
:1054F800064B19680868B0E8F00F80F309884FF088
:10550800000080F311884EF00D0E7047884D002082
:10551800024B4FF080521A60704700BF04ED00E064
:10552800EFF311804FF0BF0181F31188704700201D
:1055380008B5FFF7F5FF024B1A6801321A6008BD7B
:105548001C00002080F311887047000008B5044B48
:1055580018680138186008B9FFF7F4FF08BD00BFE4
:105568001C000020EFF309800C4B1A6820E9F00FAB
:1055780010602DE908404FF0BF0080F31188FFF755
:105588001BFF4FF0000080F31188BDE80840196840
:105598000868B0E8F00F80F309887047884D00204C
:1055A80008B5064B4FF080521A60FFF7B9FFFFF7B6
:1055B800CBFD0020FFF7C6FF08BD00BF04ED00E0EB
:1055C800034A044B1A600722043B1A60704700BF65
:1055D8003F90020014E000E0094B10B51A6800245F
:1055E80042F47F021A601A6842F07F421A60FFF79D
:1055F800E7FF044B1C60FFF761FF204610BD00BFAA
:1056080020ED00E01C000020F0B50C2404FB00FC99
:1056180009180B4B04FB01F533F80C605F1926F4ED
:1056280000465E53788033F80C0089B24004400C81
:1056380004FB0034618042EA010123F80C10F0BD3C
:10564800B85700200C2110B548430A4B1A18B2F875
:1056580006C0948801FB0C3CACF80440B2F804C0C6
:10566800D28801FB0C31CA801A5A22F400421A521D
:1056780010BD00BFB8570020F8B50C2505FB00F693
:105688000C4C0746A05B05FB00F3E35E002B0FDA2A
:10569800FFF7D8FFA35B6B43E35A5B045B0C05FB86
:1056A80003435F80A35B5D43635B23F40043A35321
:1056B800F8BD00BFB857002070B5064600282ED0A8
:1056C800174C0C25361BFFF72BFDB6FBF5F6B6B2CB
:1056D8003046FFF7D1FF05FB06F3E2185088684310
:1056E800215E00290BDAE15A6FEA41416FEA514124
:1056F8002152E35A528805FB034462800DE0A188D9
:1057080005FB014591800021EE80A680D180E25AF8
:105718006FEA42426FEA5242E252FFF787FD70BDDC
:10572800B8570020F7B5064600287FD0FFF7F8FCE9
:10573800082E07D9A6F109010C23B1FBF3F10231B8
:1057480089B200E001213A4847F6FF7384880025B2
:1057580022464FF00C0E18E030F80C506D04C4EBE4
:105768005545ADB28D4234BF4FF0000C4FF0010CDF
:105778009D422CBF4FF0000C0CF0010CBCF1000F47
:1057880018BF224618BF2B4634460EFB04FC00EB1C
:105798000C06B688002EDFD147F6FF70834218BF8B
:1057A8001D4618BF14460C226243214B9A5A5204D4
:1057B800560C82B18D4203D12046FFF743FF2EE0FD
:1057C8006D1AADB2204629464FF400422C19FFF756
:1057D8001BFFA4B223E06218B2F5557F06DB224610
:1057E800144800F0B3FFFFF721FD1FE01CB90122A8
:1057F8001A809A8001340C2202FB04F30C4E6518BF
:10580800F118C888AFB202FB006002FB056587800B
:105818002846019308F070FA019B6C80F752FFF755
:1058280005FD034B0C2606FB043604363046FEBD48
:10583800B85700206CE40008684620F007018D4640
:1058480001B50A4A0A4B0B4903E052F8040B43F826
:10585800040B8B42F9D3084B0849002201E043F8B6
:10586800042B8B42FBD3FFF769F9FEE7D0F9000858
:10587800000000206801002068010020B089002095
:105888007047FEE7254B70B5002101241C700A46BD
:10589800204602F0C3F821460022204602F0BEF856
:1058A80000212246204602F0B9F821462246204629
:1058B80002F0B4F81A4B1B4893F800C01A490023A9
:1058C8001A4A0AE0C55CCC5CD65C86EA040445EA60
:1058D8000404C454D45CCC5401336345F2DB144B48
:1058E8001B6803B19847134B1B78ABB1124B1A785E
:1058F80092B1013A1A700A4B0B4993F800C0002381
:10590800084A184606E0CC5CD55C85EA0404CC5409
:10591800D05401336345F6DB70BD00BFD64D00207F
:10592800D54D0020B47F0020E47F0020D47F0020E4
:10593800D04D0020D44D0020D74D002038B5002888
:1059480032D11B4B102218601A4B1B4DDFF86CE04C
:10595800DFF86CC01B491A700346FF222B540EF85F
:1059680000200CF800200B54013000241028F4D13A
:10597800154B01201C70154B21461C70024602F085
:105988004DF801200246014602F048F802210120A4
:1059980001F0FAFE06220120032102F0BBF80C4BAD
:1059A80001221A70204601E04FF0FF3038BD00BFD9
:1059B800D04D0020D54D0020C47F0020E47F00207A
:1059C800D47F0020B47F0020D44D0020D74D002084
:1059D800D64D0020014B1878704700BFD54D0020E8
:1059E800024B00201A78024B1A707047D44D0020E1
:1059F800D74D002037B5174D2B7823B3164B1A789F
:105A080022B300241C70154B214618602246012041
:105A180002F004F801200146224601F0FFFF0120B0
:105A28002146024601F0FAFF01200146024601F034
:105A3800F5FF0B4A2B78009201200A490A4A02F026
:105A480035FA204604E04FF0FF3001E06FF0010026
:105A58003EBD00BFD54D0020D64D0020D04D0020C2
:105A68008D580008C47F0020D47F002060B9DFF87B
:105A780020C0084AFF2103460CF8001013540130D7
:105A88001028F9D1002001E04FF0FF30704700BF27
:105A9800E47F0020B47F002010B50446FFF79AFF8A
:105AA800844236BF024B4FF0FF30185D10BD00BF77
:105AB800E47F002070B504460E46FFF78BFF844252
:105AC8000CD201F015FE074B1D5D1A5D06EA0505AF
:105AD80022EA06061E5501F021FE00E000252846B0
:105AE80070BD00BFB47F0020F7B50190FFF772FFCB
:105AF800064620B3019A12B300241CE02046FF2179
:105B0800FFF7D8FF0746A8B10025E30057FA05F2CA
:105B180012F0010F0BD00B4AE818115D00932941D0
:105B2800019A01F001019047FFF75AFF009B0135E8
:105B3800082DEBD10134B442E0DB002001E04FF046
:105B4800FF30FEBDE47F002038B9054A03461354F0
:105B580001301028FBD1002001E04FF0FF307047E2
:105B6800C47F002010B520BB134C1449024604F82A
:105B7800202011F8303043F00F036FF3041301F8BD
:105B8800303001EBC00393F803C001300CF0F00C87
:105B98006FF3071C83F803C093F805C040286FF320
:105BA800030C5A709A701A7183F805C0DFD100206F
:105BB80001E04FF0FF3010BDF87F0020F880002092
:105BC800F7B59F4E9F4D002416F82430002B00F0A7
:105BD800318105EBC4039A780AB1013A9A7006EB51
:105BE80084039F780FB35B7803215B09994015F80C
:105BF80034200193134662F38303013F924AFFB2B4
:105C080005F83430D35DC9B219420ED03846FFF7D3
:105C180051FF50B13846FFF73FFF019B184115F877
:105C2800343060F3010305F8343015F83410C1F34B
:105C3800810201F003039A4200F0FC8001F00F0298
:105C4800012A16F8243002D113F0100F08E0072AB1
:105C580002D113F0200F03E00E2A02D113F0400FF7
:105C680006D1082A14BF0020012010EAD31068D0FA
:105C780001F01001C9B229B905EBC4029278E02AF3
:105C880000F2D880FF2B0BD105EBC40315F83420A4
:105C9800DB7802F00F0203F00F039A4200F0CA808B
:105CA80015F8343043F0100305F8343005EBC4031D
:105CB8001A799978891A142901DD14329A7006EB39
:105CC80084035A7812F0030316D0022B4FEAC40358
:105CD80026D1EB189978C2F38202C2F1070251FA71
:105CE80002F293F9011008BF01228A1A6FF04501E8
:105CF8008A42B8BF0A4616E005EBC4035979C2F3D5
:105D08008202D24301F00F01521802D559780139A5
:105D1800597005EBC403597962F30301597103E023
:105D2800EB185A78013A5A7005EBC4039A781A713D
:105D38004FF0FF329A7015F83410DA7861F30302E5
:105D480077E0022A02D113F0010F0DE00B2A02D1ED
:105D580013F0020F08E00D2A02D113F0040F03E03C
:105D6800042A67D113F0080F64D001F01001C9B2FA
:105D780021B105EBC4029278E02A5BD8FF2B09D148
:105D880015F8343005EBC402D27803F00F03B3EBF7
:105D9800121F4FD015F834306FF3041305F8343060
:105DA80005EBC4031A799978891A142901DD14328C
:105DB8009A7006EB84035A7812F0030314D0022B6E
:105DC8004FEAC40325D1EB189978C2F38202C2F1D5
:105DD800070251FA02F293F9011008BF0122521882
:105DE800462AA8BF462217E005EBC4035979C2F337
:105DF800820201F00F018A1801320F2A02DD597858
:105E08000131597005EBC403597962F303015971E3
:105E180003E0EB185A7801325A7005EBC4039A78FC
:105E28004FF0FF311A71997015F83410DA7861F370
:105E38000712DA700134402C7FF4C6AE0020FEBD94
:105E4800F87F0020F8800020B47F0020F7B50546D1
:105E58004FF0FF30BDB100240B4F264601F048FC3F
:105E680007EBC40393F9011039B15E70019101F099
:105E780055FC20460199A84701E001F04FFC013488
:105E8800402CEBD10020FEBDF8800020024B93F996
:105E98000000C00F704700BFFC820020014B187043
:105EA80000207047E44D002008B50B4B18800B4BC1
:105EB80019800B4B9A8812B1D2B29B7901E0082362
:105EC80006224243DFF81CC04B43ACF80020064AC8
:105ED800138006F0F5FC08BD068300200C83002023
:105EE800D84D00200E830020F882002008B5034B0F
:105EF8001880034B198006F077FC08BD0E8300203C
:105F0800F8820020044A0023C15C99540133042B11
:105F1800FAD10020704700BF0883002007B5002889
:105F280039D11E4B1E4A9C4607CAACE80300ACF8A0
:105F380000201C4A1278422A0ED11B4A12781A7085
:105F48001A4A12785A701A4A12789A70194A1278AC
:105F58009A80194A1278DA80184B00229A80184BD6
:105F680002A81B6840F8043DFFF7CCFF4CF2503004
:105F780002F06AFE002006F0E5F900280DDB06F0C5
:105F8800A5FB00200146FFF78FFF00200146FFF721
:105F9800ADFF002001E04FF0FF300EBDFC82002075
:105FA80000E50008C03F0008C13F0008C23F0008E4
:105FB800C33F0008C43F0008C53F0008D84D002073
:105FC8000CE500088278074B043282181A600278C0
:105FD8009A804278DA80C27800201A8101229A7267
:105FE800704700BFD84D002008B506F06FFB08BD0C
:105FF8001FB5144B844693F90030002B17DA124B67
:106008004FF0FF309A88D2B10DF1040E93E80700E3
:106018008EE80700DA881989D2084A430CFB020C7B
:10602800CDF804C09EE8070006F078FC01E006F011
:10603800ABF8002803DB054B1A8801321A8005B03B
:1060480000BD00BFFC820020D84D00200683002040
:1060580038B50546002402E0FFF7CAFF044315F8E7
:10606800010B0028F8D1204638BD000038B50C4B8C
:1060780000241C7021462046FFF716FF05460948F4
:10608800FFF7E6FF012140EA05052046FFF70CFF70
:1060980005430548FFF7DCFF45EA000038BD00BFAF
:1060A800E44D00200DE100082EE100080FB410B502
:1060B80092B014AA52F8041B01AC2046119203F0C6
:1060C800A2FD2046FFF7C4FF12B0BDE8104004B09F
:1060D800704708B506F01CFC08BD08B506F01BFCA7
:1060E80008BD000038B504464FF0FF30002C39D108
:1060F8001D4A102313701D4A204613701C4B1C6048
:106108001C4B1C601C4B1C601C4B1C601C4B1C60FB
:106118001C4B1C6002F0F4FFC50F204600F0CEFDBA
:106128000028B8BF45F00205002000F071FF164AAC
:106138000028B8BF45F0040500231370134A1370F4
:10614800134A1370134B1B78422B05D1124B1B7843
:1061580013F0800F08BF1370104A00231380104AF1
:106168006842136038BD00BF2000002022000020D4
:10617800F04D0020E84D0020104E0020144E002065
:10618800084E0020F44D0020F84D0020004E00205D
:10619800F94D0020D03F0008D13F0008FA4D0020FB
:1061A8000C4E002010F0F00F70B505460C4604D1D7
:1061B80001280CBF164B174B1D78174B05F00F061F
:1061C8001B682BB166F30714284621469847E8B99F
:1061D80005F0F005202D0CD0302D11D0102D18BF52
:1061E8004FF0FF3012D166F30714204602F0FAFF91
:1061F8000CE066F307143046214600F019FE05E06E
:1062080066F307143046214600F007FF70BD00BF53
:106218002200002020000020E84D0020F0B585B0C5
:10622800174603900D460026062307224FF0040C5C
:1062380040E0B91B022914D003291FD00129A95D08
:1062480018BF6CF3030406F1010618BF61F30F24AD
:106258001AD1052060F3030461F30F246FF3174488
:1062680009E0A95D63F30304013661F30F24A95D16
:10627800013661F317446FF31F640DE0A95D62F303
:10628800030461F30F240136A95D013661F3174455
:10629800A95D013661F31F640398214601920293B8
:1062A800CDF800C0FFF77EFF0028019A029BDDF8B9
:1062B80000C002DBBE42BCD3002005B0F0BD000028
:1062C80010B5F023A0B08DF8003000238DF8013010
:1062D8008DF802307E338DF8033032238DF8043088
:1062E8000E4B0DF16B0C1B788DF805300F238DF8D4
:1062F80006306B46DA1D03E002F8014B624503D015
:1063080011F8014B002CF7D1F72102F8011BD21A22
:106318006946FFF783FF20B010BD00BFF94D00208C
:1063280000B5F02389B08DF8003000238DF80130D6
:106338008DF802307E338DF8033032238DF8043027
:10634800084B8DF806101B788DF807208DF805305E
:106358006946F72309228DF80830FFF75FFF09B077
:1063680000BD00BFF94D0020F7B5174600250422EF
:1063780062F303056FF00F0262F30F256FF3174501
:106388006FF31F650B46294604460193FFF70AFF82
:106398007E2262F30F25322262F317450C4A064625
:1063A8001278204662F31F652946FFF7FBFE0D228F
:1063B800019B62F30F2563F3174567F31F6540EAF6
:1063C800060629462046FFF7EDFE46EA0000FEBD18
:1063D800F94D0020F0B585B003900B461646002A0B
:1063E80035D000250F462E464FF0040C2DE0595DA0
:1063F8006CF3030431B101F07F0161F30F24797864
:1064080019B909E061F30F2406E001F07F0161F397
:106418001744B97819B907E06FF3174404E001F09D
:106428007F0161F31F6401E06FF31F640398214645
:1064380000920193CDF808C0FFF7B4FEDDF808C05C
:10644800019B009A0643033503379542CFD3304664
:1064580005B0F0BD08B50021052363F303016FF013
:10646800080363F30F216FF317416FF31F61FFF701
:1064780099FE08BDF8B5054607F072FC0A4E0746B6
:10648800402130782A78FFF76FFF012F044605D99D
:106498003078691C7A1EFFF79DFF0443024B187879
:1064A800FFF7D8FF2043F8BD2200002030B50B4687
:1064B8005E498BB0097804460D295ED001D839B100
:1064C800A6E00E2900F0AE800F2940F0A18093E0ED
:1064D8001BB1012B564B02D156E0554AA1E01B785F
:1064E800052B25D00AD8022B17D002D8012B40D172
:1064F80011E0032B13D0042B3BD112E0082B2FD033
:1065080004D8062B1ED0072B33D11EE0092B29D027
:106518007F2B2ED12AE0474925E0474923E0474908
:1065280021E000F0E1FF6D4602464549684612E069
:10653800684600F0EBFF00286D46BCBF2046414985
:106548000BDA10E000F0D6FF01E000F0DBFF3E4977
:1065580002466D46684603F047FB2046694602E05E
:106568003A4900E03A49FFF7ABFE5BE000F06CFF08
:1065780058E020460E210D2247E01BB1012B354D76
:1065880018D103E0334BFF221A704BE02B78FF2B16
:1065980008BF2A7046D013B1012B43D101E02E4B1E
:1065A80000E02E4B1B68002B3CD02D490878114683
:1065B800984737E02A78B2B90F21FFF7B1FE2B7858
:1065C800002B2FD1244B1B68002B2BD1254B012CE2
:1065D8001D78254818BF1C70FFF74CFF012D1CBF04
:1065E800204B1D701EE0012A02D11C4B1B68CBB941
:1065F80020460E21102208E01C4A13B1012B1B4A29
:1066080001D153600EE0526862B9FFF789FE09E0D4
:106618000E210A462046FFF783FE144A0023137012
:10662800024A137000200BB030BD00BFEC4D0020B3
:10663800FC4D002030E5000837E5000848E5000873
:106648003DE3000852E50008ADDF00080DE1000851
:106658002EE1000821000020084E0020F44D002003
:10666800F84D00202200002054E50008004E0020CC
:10667800F72910B50A465CD82F4B1C7804F008039C
:10668800DBB21BB12D49097881424FD1A0F111012C
:10669800C9B206294AD9294908700BBB264B1B7871
:1066A80003F00703042B03D82549C95C914223D181
:1066B80004F00704052C03D12249097891421BD123
:1066C800013303F007021C4B052A197862F3020113
:1066D80084BFCAB242F00802197088BF1A7028E055
:1066E80012F0800F0ED0F72A06D104F01004E4B29D
:1066F80014B10221FFF7DAFE0F4B00201870124B7D
:10670800187017E004F01004E4B25CB90A4B197869
:1067180041F0100119700C4B21461A70FFF7C6FEA4
:10672800204607E00121FFF7C1FE02E04FF0FF30ED
:1067380000E0002010BD00BF004E0020F84D0020F2
:1067480040E60008F94D0020EC4D00200FB430B5AC
:10675800A3B0269D284607F003FB642888BF0E488F
:1067680013D801AC27AA29462046219203F04BFAF8
:10677800204607F0F5FA201804E0237803F07F0399
:1067880004F8013B8442F8D101A8FFF773FE23B057
:10679800BDE8304004B07047A2E5000810B50D4AC6
:1067A8000446137803F00803DBB23BB10A4B1B78AD
:1067B800834203D100231370084A1370084B1B68E7
:1067C8000BB12046984721460648FFF7BFFF002037
:1067D80010BD00BF004E0020F84D0020EC4D0020F9
:1067E800144E0020F5E50008F0B5002289B001211B
:1067F8000546049101920392134600E0059B5A1C3A
:10680800D2B205920C2B58D8DFE803F0070F151BFE
:1068180021272D33393F454B510007A802F0FCFCD6
:10682800079CC4F30314103458E0002007A900F0B3
:106838000BFB202452E0012007A900F005FB2124CE
:106848004CE0022007A900F0FFFA222446E00320CA
:1068580007A900F0F9FA232440E0002007A900F076
:10686800DFFB30243AE0012007A900F0D9FB3124EE
:1068780034E0022007A900F0D3FB32242EE00320E5
:1068880007A900F0CDFB332428E0042007A900F075
:10689800C7FB342422E0052007A900F0C1FB3524FA
:1068A8001CE0062007A900F0BBFB362416E00720F1
:1068B80007A900F0B5FB372410E0019A0399131ECD
:1068C80018BF012309298CBF002303F00103002B03
:1068D80000F03F8100220192059208E110F10A0FB1
:1068E80004D12046FFF75AFF002332E10028C0F206
:1068F800FE800199039A4B1CDBB207990193531C44
:10690800DBB26FF30711039301F00F0303F10802E1
:1069180002F00F02062A079104D82046002D40F005
:10692800E580E4E09A1E0D2A00F2E180DFE812F02B
:106938007A007A000E0076007D007D00DF00DF001F
:10694800DF00DF00DF00DF00DF000E009DF81D1014
:10695800F72967D8F0291CD1804A1368CBB904F00D
:10696800F002102A02D0302A13D109E07C4A1380A1
:10697800012204F00F0312FA03F3784A138008E0A7
:10698800774A1380012204F00F0312FA03F3734AC3
:1069980053802046FFF76CFE9DF81C3003F00F0370
:1069A8000F2B09D09DF81E102046FFF761FE9DF8B9
:1069B8001F102046FFF75CFE6A490B7803F00803B6
:1069C800DBB2002B40F09380674A1668DEB19DF871
:1069D8001D102046B0479DF81C30C6B203F00F03C7
:1069E8000F2B10D0604A9DF81E1013682046984758
:1069F8005D4A07469DF81F101368204698470743CD
:106A080047EA0606F6B22B1E18BF0123002E14BF54
:106A1800002603F00106002E69D065E09DF81D20D0
:106A2800F72A02D9002D5FD161E0043BDBB2029363
:106A3800002B00F090809DF81D6020463146FFF73E
:106A480017FE48490B7803F00803DBB23BB9464A06
:106A580017682FB120463146B847C7B200E0002773
:106A6800029B012B2CD09DF81E6020463146FFF773
:106A7800FFFD3C490B7803F00803DBB243B93A4AFF
:106A880013682BB120463146984740EA0707FFB202
:106A9800029B022B14D09DF81F6020463146FFF759
:106AA800E7FD30490B7803F00803DBB243B92E4AFF
:106AB80013682BB120463146984740EA0707FFB2D2
:106AC800F72E02D1254B00211960264A137803F0CE
:106AD8000803DBB25BB92B1E18BF0123002F14BFBC
:106AE800002703F0010717B107992046A8471B4B59
:106AF8001A683AB31A4A1288B2F57A7F22D91988E5
:106B080061B1002251FA02F313F0010303D10132FB
:106B1800102AF7D11A461032D0B20DE0588858B171
:106B28000B4650FA03F212F0010203D10133102B85
:106B3800F7D113463033D8B2FFF730FE074B0022A7
:106B48001A6003E0049B002B7FF458AE002009B0C4
:106B5800F0BD0493CBE7029FB7E700BF0C4E0020BF
:106B6800FA4D0020004E0020104E002010B502F013
:106B78007FFB044600F0CAF840EA040400F04BFA30
:106B8800054B4FF6FF711A8844EA00008A4201D08B
:106B980001321A8010BD00BFFA4D002008B5034B22
:106BA8001B680BB1984700E0184608BDF04D00205F
:106BB800F0B5134E85B034680746ECB1C1F30763EE
:106BC8008DF80E300F4BC1F30742C1F307200024A4
:106BD80001F00F018DF80D208DF80C005A5C254648
:106BE80008E003AB595D3846019233689847019A2B
:106BF800044301359542F4DB204605B0F0BD00BFE3
:106C0800F04D002020E50008002814BF4FF0FF30A9
:106C18000020704738B9054B054A186010231370D7
:106C2800044A137001E04FF0FF307047184E0020FF
:106C3800230000202400002010F0F00F08B504D134
:106C480001280CBF064B074B18780309022B18BF05
:106C58004FF0FF3003D100F00F0002F0F9FC08BD3F
:106C6800240000202300002007B502AB03F8011D13
:106C780019460122FFF7E0FF0EBD002300E013468E
:106C88005A1C042BD2B2FAD900207047012810B53B
:106C9800044688BF4FF0FF300BD800F029FD054BA4
:106CA800FF221A55044B002223F8142000F036FD69
:106CB800002010BD1C4E00203C4E002010B504469C
:106CC8004FF0FF30ECB90F4BFF221C601C715C7158
:106CD8009C71DC711C81DC601C745C749C74DC74B9
:106CE8009C82094B20461A70FFF7D0FF0120FFF75E
:106CF800CDFF204602F004FB0028B4BF4FF0FF3060
:106D0800002010BD204E0020384E002008B500F0AD
:106D1800EFFC124B4FF6FF711A888A4201D00132FC
:106D28001A800F4B4FF6FF711A898A4201D001323F
:106D38001A810A4B4FF6FF715A888A4201D00132F4
:106D48005A80074B4FF6FF719A8A8A4201D0013266
:106D58009A8200F0E3FC002008BD00BF3C4E0020F2
:106D6800204E0020F7B50128C1F3072601F00F03D4
:106D7800C1F307420446F7B2C1F3076144D846E0BD
:106D880026488DF8046030F814C08DF80520BCF54D
:106D98007A7F8DF8061003D92046FFF777FF22E0A7
:106DA800DFF87CC09CF800C04CFA04FC1CF0010F12
:106DB80019D0072B17DD0E2BCCBF00230123012D83
:106DC80094BF002303F001036BB1164B1B5DBB425C
:106DD80006D1013D8DF804208DF80510EDB202E0D2
:106DE800002320F81430F72F98BF0E4B204698BF89
:106DF8001E5501A92A4602F02BFC023002289CBF2E
:106E0800094B53F8200001D94FF0FF30FEBD074869
:106E1800C55C2846002DB3D1F8E700BF3C4E0020E2
:106E2800384E00201C4E002048E6000820E50008E7
:106E380038B505460C4628462146FFF793FF10F162
:106E4800020FF8D038BD00000128F8B504460E46F8
:106E580088BF4FF0FF3000F2D280ABE0C0B210F034
:106E6800800F55D0F72808D9336843F00F033360F3
:106E780000237070B370F370C2E0C0F30213FB5CC0
:106E880028716B71002B3BD15E4900F00F028A5CC0
:106E9800F0286A7103D101226870EA7131E0F7289D
:106EA80021D1EA791AB1012A2A7810D108E02B7881
:106EB800052161F303032B706870AA70EA700CE077
:106EC800062161F303022A70A870EB7005E01346EF
:106ED800072262F303032B70E8702B6833600023EA
:106EE800EB7101330DE062B92B78052161F30303DF
:106EF8002B706870AA70EA702B683360012300E079
:106F080000236A79AA7100222A81002B57D077E0E2
:106F18002B79F02B17D1EB790133DBB2012BEB7115
:106F280002D0022B04D101E0687048E0A87046E066
:106F38002B78042262F30303E8702B702B6833600C
:106F48000023EB715CE0AB7923B96A792B81013AB4
:106F5800AA7101E0013BAB716B79012B03D1013BB5
:106F6800A870EB7004E0AB790BB1A87000E0E87092
:106F7800AB7923BB2B7903F0F002F02A02D01A096F
:106F88002B780BE06B791BB1012B2B7805D102E034
:106F98002B78052202E0022200E0032262F30303B9
:106FA8002B700C236343184AD11808794870D358BA
:106FB800336025E0144B0C2505FB0435134F2046A0
:106FC80002F054FA0028BFF649AF00200C235C43B6
:106FD8000D490B199A796AB11A89B2F57A7F09D9DC
:106FE80000220A511A715A719A71DA711A816FF076
:106FF800090004E000280CBF4FF0FF300020F8BD66
:107008000120E3E710E50008204E002038E60008DC
:107018004FF0FF307047002070474FF0FF30704747
:107028004FF0FF3070474FF0FF3070474FF0FF30A0
:10703800704710B504464FF0FF304CB92146204642
:1070480000F0A2FB20460321072200F063FD204642
:1070580010BD10F0800FF8B504460D46164609D04D
:1070680077200021FF22FFF7F4FF0128074675DC8F
:1070780004F07F0400200246014600F0CFFC002007
:10708800214600F023FD290E002000F01FFDC5F366
:107098000741002000F01AFDC5F30721002000F089
:1070A80015FDE9B2002000F011FD0020314600F086
:1070B8000DFD4D2C11D1FF21002000F007FDFF210F
:1070C800002000F003FD0020FF2100F0FFFC074630
:1070D800FF2814BF002501250DE000250020FF2111
:1070E80000F0F4FCFF28074604D10135082DF5D13E
:1070F800012500E00025482C14BF002301237A2C29
:1071080014BF1C4643F00104C4B1BDB9FF210020DF
:1071180000F0DCFCFF210606002000F0D7FCFF2170
:107128000746002000F0D2FCFF210446002000F0B2
:10713800CDFC46EA0747074347EA04270020FF211A
:1071480000F0C4FC55B100200146012200F066FCA5
:107158000020FF2100F0BAFC4FF0FF373846F8BD99
:10716800002070B50146012200F058FC00200321E0
:10717800072200F0CFFC00240020FF21013400F09A
:10718800A5FC0A2CF8D100200146024600F046FC76
:107198004FF47A7001F058FD402000219522FFF746
:1071A80058FF0028044654DB2F4C0025482087222E
:1071B80025704FF4D571FFF74CFFB0F5D57F19D185
:1071C800E9204FF08041FF22FFF743FF044620B13A
:1071D8000135B5F5804FF3D139E0FF227A202146F9
:1071E800FFF737FF204B10F0804F0CBF04220C2212
:1071F8001A7029E0E920FF222946FFF72AFF012813
:1072080001DC022300E00123174E237000253378A8
:10721800022B03D1E9200021FF2202E041200021B6
:10722800F922FFF716FF0028044604DB03D00135D6
:10723800B5F5804FEBD15020F9224FF40071FFF7DC
:1072480008FFB5F5804F02D0074B1B780BB96FF0DC
:10725800010400200122014600F0E0FB0020FF218C
:1072680000F034FC204670BD404E002038B504467E
:1072780078B103210122002000F04CFC00200146D7
:10728800024600F0CBFB4D200021AF22FFF7E1FEC4
:1072980025E00321072200F03DFC2046214601227B
:1072A80000F0BCFB0A24013C0020FF21E4B200F0FE
:1072B8000DFC002CF7D121462246204600F0AEFBFB
:1072C800402095222146FFF7C4FE0028054607DB2B
:1072D80021460122204600F0A1FBFFF741FF0546A9
:1072E80000200122014600F099FB0020FF2100F058
:1072F800EDFBD5F1010038BF002038BD73B5244B34
:1073080004461B780E4613F0080F08BF44020321F9
:107318000122002000F0FEFB5120FF222146FFF74A
:1073280098FE0028054603D0B8BF6FF0FF0523E09C
:1073380004460020FF2100F0C9FBC0B2FF2806D197
:107348000134B4F5803FF4D16FF4807514E0002463
:1073580032464FF4007321462046009400F0A6FD03
:10736800FF21204600F0B2FBFF21204600F0AEFBD3
:107378002046FF2100F0AAFB00200122014600F070
:107388004DFB0020FF2100F0A1FB28467CBD00BF7B
:10739800404E002037B52A4B04461B780D4613F0A3
:1073A800080F08BF440203210122002000F0B2FBAD
:1073B80058202146FF22FFF74CFE0028044603D040
:1073C800B8BF6FF0FF042FE0FE2100F07FFB2246DC
:1073D8004FF4007320462946009400F067FDFF2112
:1073E800204600F073FBFF21204600F06FFB20468B
:1073F800FF2100F06BFB00F00F00052818BF6FF4A9
:10740800807411D125460020FF2100F05FFB10F0A9
:10741800FF0F05D10135B5F5001FF4D1094C03E084
:107428000020FF2100F052FB00200122014600F05D
:10743800F5FA0020FF2100F049FB20463EBD00BFC1
:10744800404E0020FEFEFFFF08B5FEF771F86FF012
:107458007F40FEF73EFE0020FEF73FFE0020FEF7CD
:107468001DFDFEF7C1FD00200146FEF71DFD1B486E
:10747800FEF7EEFD00F03CF900214FF0FF3001F07F
:10748800C3F86FF00100012102F0B2FE6FF0800036
:10749800012102F0BBFE4FF0FF30012102F0C4FED3
:1074A8004FF0FF30012102F0CDFE4FF0FF300021F8
:1074B80002F09EFE4FF0FF30002102F0A7FE4FF0D1
:1074C800FF30002102F0B0FE4FF0FF30002102F043
:1074D800B9FE034A034BDA60FEE700BF54E6000832
:1074E8000100FA0500ED00E0014B1868704700BF85
:1074F800002004E0024B188880B28002704700BF69
:10750800227AFF1F4FF440307047000000230B4AD7
:1075180059108A18127813F0010F08BF120902F0E7
:107528000F02092A94BF302137218A18C254013327
:10753800182BECD10023037618467047107AFF1FEA
:1075480030B587B06B4683E80300044601214FF04D
:10755800805002F031FE012002F09CFD174802F035
:10756800F1FD02AD012002F005FE284602F084FE7E
:1075780063230393284641F2873305AD049302F051
:10758800ABFE284602F036FF4FF46162B4FBF2F31B
:1075980002FB13428DF814303C23B2FBF3F28DF852
:1075A8001520B4FBF3F203FB1244002029468DF8A2
:1075B800164002F0D7FE002007B030BD00031000CF
:1075C8001FB504464FF0FF30002C40F082801F208A
:1075D800012102F0D5FD404B03949A6802F00C0299
:1075E800082A02D1012303935DE01A6842F00102E0
:1075F8001A609C601A6822F0847222F480321A6041
:10760800364A5A601A6822F480221A60DC600294B2
:107618001A6842F480321A601A6802F4003203923F
:10762800029A01320292039A1AB9029AB2F5A06F2D
:10763800F2D1294B1B6813F4003318BF01230393BD
:10764800039B012B2FD1244B1A6C42F080521A64F1
:10765800234A116841F4804111609A689A609A68D7
:1076680042F400429A609A6842F4A0529A601D4A15
:107678005A601A6842F080721A601968164A11F046
:10768800007FFAD0184B40F205611960936823F027
:1076980003039360936843F002039360936803F0D5
:1076A8000C03082BFAD10021104802F0BFFA4FF45E
:1076B800407002F0B1FA0023009301936B4693E8FF
:1076C8000300FFF73DFF0398012814BF4FF0FF3078
:1076D800002004B010BD00BF003802401030002464
:1076E8000070004008544007003C02400040000879
:1076F800084B1B681BB9EFF31082074B1A604FF059
:10770800010080F31088034B00201A6801321A60C8
:10771800704700BF484E0020444E0020064A4FF0F4
:10772800FF3013683BB1013B13601BB9034B1B6867
:1077380083F3108800207047484E0020444E0020F4
:107748000F2988BF4FF0FF3018D80D4B42B2DB68C5
:107758005209DB43C3F30223C3F104039940094BE5
:107768000901C318C9B283F8001300F01F000123F0
:1077780013FA00F0034B43F822000020704700BFC3
:1077880000ED00E000E100E0F7B505460C4668466C
:1077980002F035FB072C00F23781DFE804F00A0815
:1077A80006040C12181D002417E0002410E0002421
:1077B80008E0002400E0012402238DF805300023AE
:1077C8000FE0012402238DF80530013B09E0012474
:1077D80000238DF8053004E0012400238DF80530DE
:1077E8000133012D8DF8063042D006D3022D18BF83
:1077F8006FF0010440F00A819EE005210A468448A2
:1078080002F00AFB82480621052202F005FB8048A7
:107818000721052202F000FB002C40F0F580202310
:1078280002AD022745F8083D794869468DF804708D
:1078380002F09EFA8023764869460093012602F0FA
:1078480097FA04237348694600938DF8046002F0A0
:107858008FFA4FF4006370486946009302F088FA83
:1078680040238DF804708DF8076000936848C7E0DE
:1078780068480C21052202F0CFFA66480D2105223E
:1078880002F0CAFA63480E21052202F0C5FA6148DF
:107898000F21052202F0C0FA6E462CB302244FF4E1
:1078A80000535C48694600938DF8044002F060FA82
:1078B8004FF4004357486946009302F059FA4FF4D1
:1078C80080535448694600938DF8044002F050FAFA
:1078D8004FF4806350486946009302F049FA8DF8E6
:1078E80004404FF480435EE04FF4005302274948B8
:1078F800694600938DF8047002F03AFA4FF4004399
:1079080044486946009302F033FA4FF480534148E3
:10791800694600938DF8045002F02AFA4FF4806308
:107928003D486946009302F023FA8DF804708DF8FB
:1079380007504FF4804361E035480F21062202F0DA
:107948006BFA34480321062202F066FA3148042112
:10795800062202F061FA2F480521062202F05CFA9D
:107968006E463CB308232B48694600938DF80450B3
:1079780002F0FEF9202327486946009302F0F8F93F
:107988004FF400432248694600938DF8045002F0F2
:10799800EFF94FF480731F486946009302F0E8F945
:1079A8008DF8045010231B4869460093002402F008
:1079B800DFF92BE008231748694600938DF8045037
:1079C80002F0D6F92023134869460093012702F0F4
:1079D800CFF94FF400430E48694600938DF80470C0
:1079E80002F0C6F94FF480730A486946009302F022
:1079F800BFF98DF804508DF80770102305480093DF
:107A0800694602F0B5F901E06FF002042046FEBDB8
:107A18000000024000040240000C024001281AD075
:107A280005D3022818BF6FF0010146D128E011B133
:107A3800012940D106E012B1214B042228E0204B55
:107A4800042135E01F4B4FF40061002A30D01D4B54
:107A58004FF4006229E011B101292CD108E01AB1D4
:107A6800174B4FF4805213E0154B4FF480511FE031
:107A7800144B4FF48061DAB1124B4FF4806214E07A
:107A880011B1012917D109E022B10F4B48F20002C8
:107A98001A8312E00C4B48F2000109E0084B4FF43E
:107AA80080712AB1064B4FF480721A83002104E0DA
:107AB8005983114601E06FF002010846704700BF84
:107AC80000040240000C024000000240012809D0D6
:107AD80038BF0D4B07D3022818BF6FF0010012D131
:107AE8000A4B00E00A4B99811A8802F4827222B18B
:107AF8001A8912F0800FFBD103E01A8912F0010FE6
:107B0800FBD0988980B2704700300140003C0040AB
:107B18000038004070B5002386B0ADF804304FF44B
:107B28008273ADF806300023ADF808304FF40073C7
:107B3800ADF80E300023ADF8123007230446ADF837
:107B4800143007296FD8DFE801F009121923040D52
:107B5800141E0023ADF80630ADF80E300023ADF842
:107B68000A3019E00023ADF80630ADF80E300023D6
:107B78000FE00023ADF80630ADF80E300223ADF863
:107B88000A30002308E00023ADF80630ADF80E30C7
:107B98000223ADF80A300123072AADF80C3045D886
:107BA800012C22D005D3022C18BF6FF0010041D15F
:107BB8001DE0BDF80630002B38D01F4C02F007023C
:107BC800D200204601A92588ADF8102002F018FC43
:107BD800BDF80630ADB2B3F5827F2AD12088454082
:107BE80015F0030026D0002019E0144D00E0144DD4
:107BF80002F00702013AD200284601A92E88ADF802
:107C0800102002F0FDFBBDF80630B6B2B3F5827F56
:107C18000FD12888464016F003000BD02046FF21DC
:107C2800FFF754FF05E06FF0030003E06FF0020078
:107C380000E0002006B070BD003001400038004070
:107C4800003C0040F0B5044693B04FF0FF30002CE4
:107C580040F00F8103AD884F284602F033F8012227
:107C680021463C602046FFF7D9FE01210A462046FE
:107C7800FFF7D4FE02212046FFF786FD01214FF4CD
:107C8800805002F0A7FA01214FF4001002F078FAB0
:107C980001214FF4800002F073FA7848214602F07F
:107CA80022F8774B4FF480664FF0C0620493734814
:107CB8004FF4803329460D93009303920192059463
:107CC80006940794089409960A940B940C9401F06E
:107CD800B9FF6C48214602F006F8019A4FF0400CB3
:107CE80068482946CDF818C0CDF804C00392059419
:107CF8000794099601F0A6FF0121634802F02BFCC6
:107D080001220321604802F040FC05213A20FFF7D8
:107D180017FD032106222046FFF7FCFE012021461D
:107D280002467C60FFF77AFE012002460146FFF713
:107D380075FE01200221FFF727FD01214FF4804045
:107D480002F03AFA01214FF4001002F019FA012169
:107D58004FF4800002F014FA4C48214601F0C3FFAA
:107D6800009B4B4A494829460D9304920394059475
:107D780006940794089409960A940B940C9401F0BD
:107D880061FF4448214601F0AEFFDDF804C04148D8
:107D98002946CDF818C0039405940794099601F074
:107DA80051FF01213C4802F0D6FB012203213A4849
:107DB80002F0EBFB05210E20FFF7C2FC032106228F
:107DC8000120FFF7A7FE012202202146BC60FFF731
:107DD80025FE01210A460220FFF720FE0220014667
:107DE800FFF7D2FC4FF40040012102F0E5F94FF40F
:107DF8000010012102F0C4F94FF48000012102F0C3
:107E0800BFF92648214601F06EFF009B244A23480B
:107E180029460D93049203940594069407940894B4
:107E280009960A940B940C9401F00CFF1D48214606
:107E380001F059FFDDF804C01A482946CDF818C0EA
:107E4800039405940794099601F0FCFE1648012155
:107E580002F081FB01221448032102F096FB052160
:107E68000D20FFF76DFC022003210622FFF752FECA
:107E7800204613B0F0BD00BF4C4E002040640240C5
:107E88000C30014058640240003001405860024004
:107E98000C380040706002400038004040600240EA
:107EA8000C3C004088600240003C0040F7B50128C7
:107EB80001919C4613D005D3022818BF6FF001002A
:107EC8005ED106E02F494FF0F2562F4C2F4D304B24
:107ED8000BE02C492F4E304C304D314B05E0314EE4
:107EE800314C324D324B4FF0F2516768002F45D17B
:107EF8009B892368DFF8BCE0089F23F001034EF854
:107F0800207023601AB1E26043F4806305E02A4AD6
:107F1800FF201070E26023F48063C4F804C02F6867
:107F2800019A27F0010743F001032F601AB1EA60B4
:107F380047F4806705E0214AFF201070EA6027F4C3
:107F48008067C5F804C02046009301F0D7FE284694
:107F5800314601F0D3FE089A47F00107009B2AB189
:107F680043F01003236000202F6009E023F0100382
:107F780023602F6060680028FCD101E06FF00200E8
:107F8800FEBD00BF00003910406402405864024042
:107F980000300140400E00204060024088600240EE
:107FA800003C0040390000205860024070600240E8
:107FB800003800404C4E0020594E0020584E0020FA
:107FC80008B50448044901F099FE044B1B6803B145
:107FD800984708BD40640240000039104C4E00200C
:107FE80008B505484FF0F25101F088FE034B5B6875
:107FF80003B1984708BD00BF586002404C4E0020AE
:1080080008B50448044901F079FE044B9B6803B1A4
:10801800984708BD40600240000039104C4E0020CF
:1080280070B504460D461C484FF4003102F013F8B1
:108038000028F8D11848012101F0B9FF164817495E
:1080480002F009F80028F9D013489421002201F021
:10805800C8FF1148124901F0E9FF0028F9D00026AD
:108068000CE014F8011B0C4801F0D0FF0136F6B201
:1080780009480C4901F0DAFF0028F9D0AE42F0D3E4
:108088000548094901F0E7FF0028F9D00248012115
:1080980001F09AFF70BD00BF0054004001000010BD
:1080A80082000700800007000400001010B52D486A
:1080B8004FF4003101F0CFFF0028F8D12948012101
:1080C80001F075FF2748284901F0C5FF0028F9D0BD
:1080D80024489421002201F084FF2248234901F01A
:1080E800A5FF0028F9D01F48322101F08FFF1D4855
:1080F8001F4901F09BFF0028F9D01A48012101F01F
:1081080063FF4FF40031174801F0A5FF014600282E
:10811800F7D1144801F06DFF1248012101F047FF23
:108128001048114901F097FF0028F9D00D48942113
:10813800012201F056FF0B480E4901F077FF002895
:10814800F9D008480C4901F071FF0028F9D005481A
:1081580001F05EFF01210446024801F035FF204688
:1081680010BD00BF0054004001000010820007004D
:10817800800007000200030040000300F0B5054638
:10818800A1B04FF0FF30002D40F098811CAF384669
:10819800022401F034FE10223946C9481C928DF899
:1081A80075408DF874408DF8765001F0E1FD062297
:1081B8000421C34801F030FE4FF4806C3946C148B1
:1081C800CDF870C0CDF804C001F0D2FD06220A2116
:1081D800BC4801F021FE4FF480533946B9481C933E
:1081E80001F0C6FD06220C21B64801F015FE8023D9
:1081F8003946B4481C9301F0BBFD07210622B1485B
:1082080001F00AFE012640223946AF488DF8766013
:108218001C928DF874408DF877508DF8754001F0F8
:10822800A7FD04220621A84801F0F6FD4FF40073CB
:108238003946A5481C93029301F09AFD09210422AE
:10824800A14801F0E9FD10223946A0481C928DF89A
:1082580074608DF8765001F08BFD9C48102101F078
:10826800D9FD31464FF4004001F0A6FF304601F039
:1082780017FF18A90846039102F064F9029B4AF611
:108288004442934803991A92ADF86630ADF86030CD
:10829800ADF86250ADF86450ADF86C5002F0DEF8FD
:1082A80031468B4802F064F931464FF4001001F072
:1082B80067FF05AB1846029301F004FD854829467F
:1082C80001F011FD8348844901F018FD834A029B9F
:1082D80006924022089202F5F8620C9202F5C0520A
:1082E800DDF804C00D92A2F5F85219460E927948AD
:1082F80002F57F42CDF82CC00F9205950A9501F042
:10830800A1FC18213246734801F012FD324670482C
:10831800214602F03AF905211020FFF711FA3146FB
:108328004FF4001001F048FF6D4801F08FFD14ABC9
:108338001846029301F020FE6A4ADDF804C0149240
:108348003322ADF858204FF480423146ADF85C2016
:1083580063484BF6FF72ADF85AC0ADF85620ADF839
:10836800545001F017FE029B5D48194601F09AFD32
:108378001021564801F04CFD4FF47A7000F064FC6F
:108388008DF879601EAE0D22304621468DF8782092
:108398000392FFF745FE9923304621468DF8793040
:1083A8008DF87850FFF73CFE472321468DF878304A
:1083B80030466FF07F038DF87930FFF731FEFFF715
:1083C80075FE60F07F00322321468DF87900304633
:1083D8008DF878300293FFF723FEFFF767FE029BC4
:1083E80000F07F008DF87900214630468DF878300E
:1083F800FFF716FE304621468DF878508DF87950F3
:10840800FFF70EFE04238DF878303046AB33214653
:108418008DF87930FFF704FE039A70233046214621
:108428008DF878208DF87930FFF7FAFD05238DF85F
:10843800783030467C3321468DF87930FFF7F0FDEF
:1084480006238DF878303046013321468DF879308F
:10845800FFF7E6FD0A23304621468DF8783002936F
:108468008DF87950FFF7DCFD2722304621468DF83C
:1084780078208DF87950FFF7D3FD029B9A22304679
:1084880003218DF878208DF879308DF87A30FFF750
:10849800C7FD1F238DF8783030460F2321468DF80D
:1084A8007930FFF7BDFD9E23304621468DF8784090
:1084B8008DF879302F46FFF7B3FD284621B0F0BD7F
:1084C800000002400008024000040240000C024084
:1084D800003C004088600240400E00200C3C0040F8
:1084E80000540040A0860100F8B50B4E05460C4626
:1084F80030460021174601F0F6FB3046074901F0E7
:10850800FDFB074B64001F603046F5600121746075
:1085180001F0E9FB0020F8BD88600240400E002011
:108528005C4E00200C4A08B551680C4B01EA030365
:108538002BB10A4B0020D360094B1B689847064AA9
:10854800084B516801EA03032BB1064B0120D360A5
:10855800034B1B68984708BD0060024000040020D8
:108568005C4E00200008002010B9034B188001E081
:108578004FF0FF30704700BF604E002037B504460B
:10858800684601F03CFC01238DF80430013B8DF86E
:108598000630023314F0010F6D468DF8053006D011
:1085A8004FF4805317486946009301F0E1FB14F03B
:1085B800020F08D002A94FF4005341F8083D1148B2
:1085C800694601F0D5FB14F0040F08D002A94FF456
:1085D800804341F8083D0B48694601F0C9FB14F097
:1085E800080F08D002A94FF4004341F8083D054898
:1085F800694601F0BDFB34F00F040CBF20466FF054
:1086080001003EBD000C024010F0010F0BD011F02C
:10861800010F15BF1D4B1D4B4FF480524FF4805274
:1086280014BF1A835A8310F0020F0BD011F0020FF7
:1086380015BF164B154B4FF400524FF4005214BFA0
:108648001A835A8310F0040F0BD011F0040F15BFD2
:108658000E4B0E4B4FF480424FF4804214BF1A83E6
:108668005A8310F0080F0BD011F0080F15BF074BF5
:10867800064B48F2000248F2000214BF1A835A83DC
:1086880030F00F0018BF6FF001007047000C024077
:108698000C4B58695B69C0F3003013F4005F094B59
:1086A80018BF40F002005B6913F4804F054B18BFF8
:1086B80040F004005B6913F4004F18BF40F0080055
:1086C800704700BF000C02404FF0FF3070474FF07A
:1086D800FF3070474FF0FF3070474FF0FF30704762
:1086E8004FF0FF3070470000F0B50128034685B011
:1086F80088BF4FF0FF3052D802AE30460193294C64
:1087080001F07DFB284A402108274FF4006061836F
:10871800678350834FF4807050834FF40070508308
:10872800012500220291204631468DF80E208DF851
:108738000C508DF80D5001F01BFB20463146029776
:1087480001F016FB019B0BB18DF80E5004AC4FF4F1
:10875800807544F8085D1548214601F009FB124868
:108768002146029501F004FB4FF400730E482146A0
:10877800029301F0FDFA4FF400630B48214602937F
:1087880001F0F6FA012300258DF80F3005487F33F4
:1087980021468DF80C50029301F0EAFA284605B0FC
:1087A800F0BD00BF000C024000080240000002407B
:1087B80010F0800F15BF534B524B4FF480724FF49B
:1087C800807214BF1A835A834F4B402210F0400F17
:1087D8005A835A831A831A831A830DBF494BA3F508
:1087E80040634FF480724FF4807214BF1A835A8327
:1087F800454B402210F0200F5A835A831A831A835C
:108808001A830DBF3F4BA3F540634FF480724FF4BA
:10881800807214BF1A835A833B4B402210F0100F0A
:108828005A835A831A831A831A830DBF354BA3F5CB
:1088380040634FF480724FF4807214BF1A835A83D6
:10884800314B402210F0080F5A835A831A831A8337
:108858001A830DBF2B4BA3F540634FF480724FF47E
:10886800807214BF1A835A83274B402210F0040FDA
:108878005A835A831A831A831A830DBF214BA3F58F
:1088880040634FF480724FF4807214BF1A835A8386
:108898001D4B402210F0020F5A835A831A831A8301
:1088A8001A830DBF174BA3F540634FF480724FF442
:1088B800807214BF1A835A83134B402210F0010FA1
:1088C8005A835A831A831A831A830DBF0D4BA3F553
:1088D80040634FF480724FF4807214BF1A835A8336
:1088E800094B40225A835A831A831A831A8308220F
:1088F8001A8300201A831A831A831A831A835A83C5
:10890800704700BF00000240000C024010F0800FCA
:1089180015BF454B444B4FF400624FF4006214BF3F
:108928001A835A83404B4FF4807210F0400F5A83D9
:108938005A831A831A831A8315BF4FF400624FF4BF
:1089480000621A835A83384B4FF4807210F0200F5C
:108958005A835A831A831A831A8315BF4FF4006205
:108968004FF400621A835A832F4B4FF4807210F031
:10897800100F5A835A831A831A831A8315BF4FF428
:1089880000624FF400621A835A83274B4FF48072B7
:1089980010F0080F5A835A831A831A831A8315BF53
:1089A8004FF400624FF400621A835A831E4B4FF44F
:1089B800807210F0040F5A835A831A831A831A8319
:1089C80015BF4FF400624FF400621A835A83164BA6
:1089D8004FF4807210F0020F5A835A831A831A8355
:1089E8001A8315BF4FF400624FF400621A835A834A
:1089F8000D4B4FF4807210F0010F5A835A831A837B
:108A08001A831A8315BF4FF400624FF400621A8369
:108A18005A83054B4FF480725A8300205A831A8375
:108A28001A831A83704700BF0008024020B1054B23
:108A38004FF480721A8303E0024B4FF480725A831A
:108A4800002070470000024020B1054B4FF400623F
:108A58001A8303E0024B4FF400625A8300207047E8
:108A68000008024028B1012818BF4FF0FF3015D187
:108A780008E00B4B4FF4807271B1094B4FF48072D0
:108A88001A830BE0064B4FF4007229B1044B4FF4E4
:108A980000721A83002001E05A830846704700BF1D
:108AA80000080240024B1869C0F3C010704700BFAD
:108AB800000C024000207047F8B5054600200C461F
:108AC800FFF7B4FF0120FFF7BFFF01212846FFF79A
:108AD800C9FF0028B8BF4FF0FF301EDB13E028465F
:108AE8000121FFF7BFFF0A270120FFF7ADFF17F1AC
:108AF800FF37F9D1FFF7D6FF394606462846FFF774
:108B0800B1FF16B1013C002CE9D10020FFF79CFF12
:108B1800002C14BF00206FF00100F8BD08B54FF01D
:108B28008040012101F0B0FD38B14FF080400121B3
:108B380001F0B6FD014B1B68984708BD644E002044
:108B480008B50648012101F09FFD30B10348012115
:108B580001F0A6FD024B5B68984708BD0004004081
:108B6800644E002008B50648012101F08DFD30B1A2
:108B78000348012101F094FD024B9B68984708BD0A
:108B8800000C0040644E002030B5012185B0044639
:108B9800102001F011FB4FF6FF73029354235C433E
:108BA8000C4D013CADF804402846002401A9ADF85D
:108BB8000C40ADF8064001F0F3FC01210A462846B6
:108BC80001F057FD2846012101F046FD204605B079
:108BD80030BD00BF001000400348012108B54162C4
:108BE80001F05EFD002008BD00100040054810B5EA
:108BF8000121446A01F048FD002818BF4FF0FF34F6
:108C0800204610BD001000401FB504464FF0FF304D
:108C1800B4B90120014601F0DDFA4FF6FF73029363
:108C28000848A72301A9ADF80430ADF80C40ADF809
:108C3800064001F0B5FC0348012101F00DFD204676
:108C480004B010BD00000140044B5A6A92B2596A40
:108C5800891A89B28142FAD9002070470000014080
:108C680070474FF0FF30704712230B800048704761
:108C7800B4E6000804230B8000487047B0E60008FB
:108C880013B507221E49684605F036F81D4901222A
:108C9800002306E0203AD2B25F2A8CBF00220122CC
:108CA80001331F2BCCBF002002F0010020B111F8C6
:108CB800012F002AEED10132002B0CBF002302F055
:108CC8000103694603B11049104A02234FF0000C12
:108CD80004E002F8020C02F801CC023311F8010B8F
:108CE8000232041E18BF0124632BCCBF002404F0F9
:108CF8000104002CEDD106480370032343701CBD0A
:108D080030E50008DF3F0008E03F00084689002002
:108D18004489002008B5FFF7B3FF08BD08B5FFF781
:108D2800AFFF08BD70477047704770477047002015
:108D3800704700207047000065230B80004870478B
:108D4800F4E6000870B58CB00BAD03220C4601AEFA
:108D58000849284604F0D0FF3046FEF7D7FB002824
:108D6800ACBF304628460449224602F075F802484E
:108D78000CB070BDE4E60008448900207FB5084CBB
:108D880001AD0E460C222846064904F0B5FF2846D8
:108D98002146324602F060F8204604B070BD00BF9C
:108DA80044890020E7E60008022908B503D10846EF
:108DB800002100F06FFA002008BD012908B503D191
:108DC8000846013900F05CFA002008BD10B5022100
:108DD800044602F016FD2046812102F012FD002013
:108DE80010BD08B5002000F091F908BD08B50120B4
:108DF80000F08CF908BD0000022110B5402204469D
:108E08000B4602F0D5FC812140220223204602F0C5
:108E1800CFFC0221034A4023034802F011FD002041
:108E280010BD00BF108300205083002013B501201F
:108E3800014601F0A5F94FF4D853194C00930323C8
:108E48008DF80530013B8DF8043020460023694633
:108E58008DF806308DF8073000F08AFF204608218B
:108E68000A2200F0D9FF204609210A2200F0D4FF87
:108E780020460B210A2200F0CFFF0A2220460C21AF
:108E880000F0CAFF01214FF4804001F0A3F98020CF
:108E9800012101F083F9012000F064FF1CBD00BF2F
:108EA8000000024008B543200821FEF749FC08BD30
:108EB80008B5024802F06AFD08BD00BF50830020D3
:108EC80008B580B2FFF7C0FE08BD08B54FF47A7345
:108ED8005843FFF7F5FF08BD4FF0A0431868C0F3EB
:108EE800C0407047022837B5054688BF4FF0FF30AD
:108EF8003ED8FFF776FF4DBBFFF7EEFF30B31D4CB2
:108F08002046FFF793FF1C4B0121C4F8E0351B4BAB
:108F18002046C4F8E4351A4BC4F8E83502F008F8DE
:108F2800204602F0DDF8204602F04CF92046FFF713
:108F3800B9FF01210323204684F8101184F8123167
:108F4800FFF75AFFFFF752FF284611E00B4B0121AC
:108F58000B4A00930748084B01F021FD054802F031
:108F68000BFD3220FFF7B1FF024802F0FBFC0020A6
:108F78003EBD00BF5083002084E60008C8E6000814
:108F880068E60008F7B5274CD4F8E035002B47D041
:108F9800FEF7AEFB244B1B78002B3FD0D4F8D853F8
:108FA800C5F38F05002D39D0204B29B21A8892B20B
:108FB800C2F14002914231DA013D1D4F1D4C1E4A5B
:108FC800ADB257F8046B0192C6F303101030314666
:108FD8000093FDF7EDFD019A009B80B9218889B2C5
:108FE80042F821602188013189B22180218889B223
:108FF8003F2988BF20801988013189B21980013D35
:10900800ADB2691C09B20029DBDC074B00221A70DB
:1090180004480221064A402302F012FCFEF77EFBB8
:10902800FEBD00BF50830020B8500020B04E002085
:1090380010830020BA500020B84F002008B5294BF3
:10904800D3F8E035002B4BD0FEF752FB264B1B78AC
:10905800002B43D1254B1A8892B2002A3ED0244ACD
:109068001278002A3AD01A88224892B2102A98BF59
:109078001B881D4A94BF9BB21023012111701B4A03
:10908800DFF874C01188C91A89B211801BB2002197
:109098001A4A1BE0B2F800E01FFA8EFE5CF82EE0D8
:1090A80040F804EBB2F800E00EF1010E1FFA8EFE54
:1090B800A2F800E0B2F800E01FFA8EFEBEF13F0F02
:1090C80084BF4FF0000EA2F800E001319942E1DBC5
:1090D8009B0004488121074A02F0DAFBFEF71EFBD9
:1090E80008BD00BF50830020B44F0020BC500020B2
:1090F800C2500020704E0020B44E0020BE50002008
:10910800002814BF4FF0FF3000207047104A00239A
:10911800138011880F4A89B2118011880E4A89B2CA
:1091280011800E4A13700E4A138011880D4A89B2B5
:10913800118011880C4A89B211800C490C4A10B16F
:109148000120087001E00B700123137000207047A4
:10915800B04E0020BA500020B24E0020B850002077
:10916800BC500020C4500020BE500020C250002037
:10917800B44F002038B5174D04462B784FF0FF3018
:109188003BB3154B1B889BB23E2B09D9FFF756FF03
:109198002B78002B14BF6FF001004FF0FF3018E060
:1091A800FEF7A6FA0D4B0E491A8892B241F82240F2
:1091B800013292B21A801A8892B23F2A01D900224B
:1091C8001A80054B1A88013292B21A80FEF7A6FA65
:1091D800002038BDC2500020BC500020C4500020E0
:1091E800B44E002070B506460A4C42F20F7504E0F2
:1091F8002388AB420CD8013323803046FFF7BAFFEF
:1092080010F1020FF4D0002802DB024B00221A8072
:1092180070BD00BFC0500020124B10B51B8804461B
:109228009BB24FF0FF30DBB1FEF762FA0E4B0F4AEC
:10923800198889B252F8212022601A88013292B224
:109248001A801A8892B23F2A01D900221A80054C46
:109258002388013B9BB22380FEF760FA208880B206
:1092680010BD00BFB04E0020B24E0020B84F002005
:1092780008B5FFF787FEFFF7E1FE002008BD0000F4
:1092880008B5034B00221A70FFF7D8FE08BD00BFCF
:10929800B44F002008B5034B01221A70FFF772FE85
:1092A80008BD00BFB850002030B50128044685B07D
:1092B8000D4688BF4FF0FF301AD84FF0000304A9BD
:1092C800ADF80430ADF80630ADF80830ADF80C3024
:1092D80041F8105D4FF00C0314BF06480648694674
:1092E800ADF80A3001F0E0F9044B002043F82450AF
:1092F80005B030BD0044004000480040DC5100206B
:10930800F0B5054685B04FF0FF30002D40F097804E
:10931800022107224B4800F07FFD0321072249481C
:1093280000F07AFD08210722474800F075FD02AEDB
:1093380007220921444800F06FFD304600F05FFD28
:1093480001240423022731463E48029301938DF8F5
:109358000D508DF80C708DF80E4000F009FD4FF49B
:1093680080723146384802928DF80C708DF80E40A4
:1093780000F0FEFC08223146324802928DF80C704B
:109388008DF80F4000F0F4FC4FF4007231462E487F
:10939800029200F0EDFC1020214600F01BFF4FF474
:1093A8006020214600F008FF47F612212846FFF703
:1093B8007BFF47F612212046FFF776FF019B262008
:1093C8001946FEF7BDF92246204840F2255101F022
:1093D800DCF9019B27201946FEF7B2F91C4840F238
:1093E8002551224601F0D1F91A481B490570037826
:1093F800DFF868E00B700B78194A8EF800301570AA
:1094080092F800C0174B83F800C01E78DFF858C0E8
:109418008CF8006045704078487049780B488EF8A1
:1094280001105570527821465A705B788CF80130DB
:1094380001F09EF90648214601F09AF9284605B040
:10944800F0BD00BF00000240000C02400044004094
:1094580000480040CC500020D4510020D0500020BB
:10946800D8510020E4510020C8500020012838B508
:10947800044688BF4FF0FF301DD80F4B6FF0010036
:109488001B5DC3B1FEF734F90C4B0D491A5D02EBB5
:1094980084128D5C1A5D0132D2B21A551A5D3F2AC8
:1094A80001D900221A55044B1A5D013AD2B21A5555
:1094B800FEF734F9284638BDCC500020D0500020A3
:1094C80054510020012838B504460D4688BF4FF096
:1094D800FF301FD8104B1B5D3F2B88BF6FF001007A
:1094E80018D8FEF705F90D4B0D491A5D02EB8412E9
:1094F8008D541A5D0132D2B21A551A5D3F2A01D92C
:1095080000221A55044B1A5D0132D2B21A55FEF7E1
:1095180005F9002038BD00BFCC500020D4510020F0
:1095280054510020012838B5044688BF4FF0FF3059
:109538001DD80F4B6FF001001B5DC3B1FEF7D8F8C3
:109548000C4B0D491A5D02EB84128D5C1A5D0132D9
:10955800D2B21A551A5D3F2A01D900221A55044B76
:109568001A5D013AD2B21A55FEF7D8F8284638BD26
:10957800D8510020C8500020D4500020F0B5012850
:10958800044687B00D46174688BF4FF0FF3052D8C3
:109598002A4E335DD3183F2BC8BF6FF001004ADC59
:1095A800FEF7A6F80022264B2648274901973CE0FB
:1095B80013F804C015F8017BDFF890E00CEB841C6D
:1095C8000EF80C7013F804C00CF1010C5FFA8CFC57
:1095D80003F804C013F804C0BCF13F0F84BF4FF078
:1095E800000C03F804C016F804C00CF1010C5FFA73
:1095F8008CFC06F804C016F804C0BCF1010F12D1A7
:10960800012C15BFB1F80CC0B0F80CC01FFA8CFCC7
:109618001FFA8CFC15BF4CF0800C4CF0800CA1F8A4
:109628000CC0A0F80CC0013292B2019FBA42BFD35D
:10963800FEF774F8002007B0F0BD00BFD851002035
:10964800E45100200048004000440040D45000206D
:1096580070B505460C461646284621463246FFF7A1
:109668008DFF10F1020FF7D070BD0000144B10B53C
:109678001A8812F0200F09D09C882020E4B22146D5
:10968800FDF78CFA10B92146FFF71CFF0C4C238814
:1096980013F0800F13D00B4B1B7853B10020FFF74A
:1096A80041FF0028A4BF80B2A08008DAFF23A3806E
:1096B80005E0A38923F080031B041B0CA38110BDC4
:1096C80000440040D8510020154B10B51A8812F0FC
:1096D800200F0AD09C882120E4B22146FDF75EFACB
:1096E80018B901302146FFF7EDFE0D4C238813F021
:1096F800800F13D00B4B5B7853B10120FFF712FF9B
:109708000028A4BF80B2A08008DAFF23A38005E068
:10971800A38923F080031B041B0CA38110BD00BF89
:1097280000480040D851002070B56A4C206800F00D
:109738008AFCB0F5403F054600F0CA80664B00EA57
:109748000303002B33D0E368002B30D0206800F0EF
:109758005FFC628A238A92B29BB29A4206D2638ADB
:10976800E2689BB2D05401339BB26382594B5A6969
:1097780012F0020F3ED1598A1A8A89B292B2013A7E
:1097880091420CDA5A6912F0040F00F0A1805B8A4A
:109798009BB2012B40F09C80002840F099804D4CF2
:1097A8000021206800F025FC2068012111E04B4BC6
:1097B80005EA0303A3B115F4802111D1454C258A8C
:1097C800ADB2012D40F08480206800F012FC2068C2
:1097D800294600F0F9FB636943F00203636177E00F
:1097E8003F4A05EA0202002A3ED03A4B5A6912F073
:1097F800020F07D05A6918686FF300025A614FF4D4
:10980800E0612FE0598A1A8A89B292B291420BD24A
:109818009968186829B15A8A92B2895C013292B261
:109828005A8200F0F3FB53E05A6912F0080F04D192
:109838001868012100F0C8FB03E01868012100F056
:10984800B6FB244B5A6942F002025A611A8A92B254
:109858002AB95969186862F30001596112E0186859
:109868004FF4806100220FE01E4E1A4C05EA0606EE
:10987800A6B1636913F0020F09D06369206862F327
:10988800000363614FF4E06100F0C5FB20E021793B
:10989800206801F0010200F0A4FB19E032462068BC
:1098A8004FF4E06100F0B7FB0F4B31461D606FF0DD
:1098B8000703A3616369206866F30003636100F02E
:1098C80098FB206800F0A4FB2068012100F07CFBD5
:1098D80070BD00BFE85100204000001002000010D9
:1098E80080000010010000104089002038B51C4D90
:1098F800286800F0A8FB1B4B044600EA030333B1B9
:109908002868194900F0C1FB6FF00503AB61174BDC
:1099180004EA03033BB1124D1549286800F0B5FB72
:109928006FF00403AB61134B04EA03035BB10C4C07
:109938001149206800F0A9FB6FF00603A3612068B5
:10994800012100F041FB064C4FF4E0612068002241
:1099580000F061FB63696FF30003636138BD00BF0A
:10996800E851002000010010000100010002001071
:1099780000020001000400100004000108B528B12D
:109988000368197003680133036003E0C9B201205A
:10999800FDF76AF908BD002AF7B58C460446154656
:1099A80010DD002200E001321CF802100029FAD173
:1099B800AA42ACBF0D46AD1A13F0020F0CBF202708
:1099C800302700E0202713F001060DD109E02046DA
:1099D8003946CDF804C0FFF7D1FFDDF804C00136E1
:1099E800013D002DF3DC00E00026634605E020463B
:1099F8000193FFF7C3FF019B013613F8011B0029F0
:109A0800F5D105E020463946FFF7B8FF0136013D9C
:109A1800002DF7DC3046FEBDF0B587B004461D4684
:109A28000C9E0D9B084651B930228DF80C208DF8FC
:109A38000D10204603A93246FFF7ADFF43E00A2A7E
:109A480014BF00210121002D0CBF002501F00105E4
:109A58002DB1002802DA4042012500E00025DDF89A
:109A680038E006A94FF0000C01F801CDAEF13A0E2E
:109A78000DE0B0FBF2FC02FB1C0CBCF1090FC8BFE7
:109A8800F4440CF1300C01F801CDB0FBF2F00F46B4
:109A98000028EED18DB15EB113F0020F08D0204638
:109AA8002D210193013EFFF769FF0125019B04E089
:109AB8002D224F1E01F8012C00252046394632463A
:109AC800FFF769FF401907B0F0BD0000F0B589B095
:109AD80006460D46059200247AE0252B72D115F82A
:109AE800013F002B77D0252B6CD02D2B02D10135CF
:109AF800012303E0002301E043F002032F4615F899
:109B0800012B302AF8D0002202E00A2000FB02C212
:109B180039783D46A1F1300C5FFA8CF001370928FD
:109B2800F3D9732909D10599081D059009682D48AD
:109B3800002908BF0146304641E064290ED1059945
:109B48000193612300920293081D096805900A2277
:109B580030460123FFF760FF241838E0782906D142
:109B680005990193081D05900092612307E0582983
:109B78000AD105990193081D05900092412302938B
:109B88003046096810220BE075290BD1059901931D
:109B9800612300920293081D096805900A22304645
:109BA8000023D7E7632912D10599081D0968059094
:109BB8008DF81C1000218DF81D10304607A9FFF7FD
:109BC800EAFEC9E729783046FFF7D8FE01340135A7
:109BD8002B78002B81D116B1336800221A702046E9
:109BE80009B0F0BD5CE700080EB40FB505AA52F83D
:109BF800041B019001A80392FFF768FF04B05DF809
:109C080004EB03B0704707B5034602A840F8043DCB
:109C1800FFF75CFF0EBD000040F0BE60024B40F451
:109C28002020D860704700BF00ED00E021F06041BF
:109C380021F07F01024B41EA00009860704700BFA5
:109C480000ED00E002681E4BD1F80CC002EA0303E5
:109C58000A684CEA0202D1F814C042EA0C02D1F8B0
:109C680018C042EA0C02D1F81CC042EA0C02D1F832
:109C780020C042EA0C02D1F824C042EA0C02D1F812
:109C880028C042EA0C02D1F834C042EA0C02D1F8EA
:109C980038C042EA0C0242EA030303604269D1F881
:109CA80030C0CB6A22F007024CEA03031343436136
:109CB8000B6943604B6883608B68C360704700BF63
:109CC8003F801CF00023036043608360C36003612E
:109CD80043618361C361036243628362C362036356
:109CE80043638363704719B1036843F0010302E0DB
:109CF800036823F00103036070470000084B094A1A
:109D0800DFF824C060458CBF10461846074B11F099
:109D1800005F01EA030314BFC3608360704700BF9C
:109D280000600240006402400F6402407D0F7D0F16
:109D380011F0800F08D01AB1436943F0800302E0A4
:109D4800436923F080034361802909D001F01E0193
:109D580012B10368194302E0036823EA01010160B4
:109D680070470000014B5861704700BF003C01403C
:109D7800F7B50B68019300231A46012404FA02FC84
:109D8800019D0CEA0504644534D1032606FA03FC58
:109D980005686FEA0C0C0CEA050505600D79076883
:109DA80015FA03F6013DEDB23E43012D066013D8C6
:109DB8004E7985689E400CEA05058560856846EA07
:109DC80005058560456825EA040444608C79456882
:109DD8009440A4B22C434460C4680CEA040CC0F854
:109DE8000CC091F807C0C4680CFA03FC4CEA040CD8
:109DF800C0F80CC001320233102ABED1FEBD4FF6A6
:109E0800FF7303600023037143718371C37170474B
:109E1800018370474183704701F007039B004FF0AF
:109E28000F0C0CFA03FC12FA03F3C908083110B539
:109E380050F8214024EA0C0C40F821C050F821C009
:109E480043EA0C0340F8213010BD000008B5124B5E
:109E5800984207D14FF40010012100F0E5F94FF4C2
:109E6800001014E00D4B984207D14FF480000121F7
:109E780000F0DAF94FF4800009E0094B984209D163
:109E88004FF40000012100F0CFF94FF40000002149
:109E980000F0CAF908BD00BF005400400058004057
:109EA800005C00407FB50446868868460D4600F091
:109EB800FDF802992E4826F03F063604B1FBF0F073
:109EC800360C80B240EA0606A68022882B6822F06B
:109ED80001021204120C2280264A93420AD85B001F
:109EE800B1FBF3F301309BB280B22084032B98BFFF
:109EF800042322E0B5F806C04BF6FF72944505D15D
:109F080003225343B1FBF3F39BB206E019225343F8
:109F1800B1FBF3F39BB243F480431A054FF49672F6
:109F280008BF43F00103504302F52F7290FBF2F093
:109F3800013080B243F400432084A38323886989D5
:109F48009BB243F0010323802388AA8823F480630B
:109F580023F00A031B0441EA02021B0C13439BB2C1
:109F680023802A89AB8942EA03039BB223817FBD00
:109F780040420F00A086010041F2883303600023AD
:109F880083804BF6FF72038143814FF48043C28084
:109F98008381704721B103889BB243F0010304E039
:109FA800038823F001031B041B0C0380704721B1B5
:109FB80003889BB243F4807304E0038823F480731E
:109FC8001B041B0C0380704721B103889BB243F428
:109FD800007304E0038823F400731B041B0C038044
:109FE800704712B141F0010101E001F0FE01018268
:109FF800704721B103889BB243F4806304E003886F
:10A0080023F480631B041B0C038070470182704794
:10A01800008AC0B270471AB183889BB2194303E023
:10A0280083889BB223EA010181807047838A008B71
:10A038009BB243EA0040084020F07F40884214BFAA
:10A04800002001207047838A008B9BB243EA0040BE
:10A0580020F07F40704782B00023019300930B0FDC
:10A0680000900193019B21F07F4113B1009B1433B1
:10A0780002E0009B090C18330093009B1B681942EF
:10A088000CBF0020012002B07047C94389B2818209
:10A0980070470000014B1860704700BF20000E4257
:10A0A800014B1860704700BF68004742214B9A680F
:10A0B80002F00C02042A08BF1F4B1ED0082A1BD12D
:10A0C80059685A6811F4800F15BF596859681A4BB6
:10A0D8001A4B02F03F02B3FBF2F3164A14BFC1F366
:10A0E8008811C1F3881152684B43C2F3014201320F
:10A0F8005200B3FBF2F300E0104B0E4903608B688B
:10A108000F4AC3F30313D35CD0F800C02CFA03F34F
:10A118004360D1F808C0CCF3822C12F80CC023FAA3
:10A128000CFCC0F808C08968C1F34231525CD340C6
:10A13800C36070470038024000127A000024F4001F
:10A148002800002000F44073B3F5407F09D1084B84
:10A1580020F07042996822F4407221F4F8110A4301
:10A168009A60034B00051A6F42EA1050186770474F
:10A1780000380240014B1860704700BF3C0E474250
:10A1880019B1054B1A6B104303E0034B1A6B22EA13
:10A1980000001863704700BF0038024019B1054B32
:10A1A8005A6B104303E0034B5A6B22EA00005863D2
:10A1B800704700BF0038024019B1054B1A6C1043B4
:10A1C80003E0034B1A6C22EA00001864704700BFD2
:10A1D8000038024019B1054B5A6C104303E0034B99
:10A1E8005A6C22EA00005864704700BF00380240E9
:10A1F80019B1054B1A69104303E0034B1A6922EAA7
:10A2080000001861704700BF0038024019B1054BC3
:10A218005A69104303E0034B5A6922EA0000586167
:10A22800704700BF0038024019B1054B1A6A104345
:10A2380003E0034B1A6A22EA00001862704700BF65
:10A248000038024019B1054B5A6A104303E0034B2A
:10A258005A6A22EA00005862704700BF003802407C
:10A26800002303E001330A38DBB2C0B20928F9D869
:10A2780040EA0310C0B27047002303607F33436095
:10A288008033836070470000002382B001930D4B38
:10A29800DA6812F0400F12D14FF0FF32DA60DA6854
:10A2A8000199013101910199B1F5803F02D012F075
:10A2B800400FF4D0034BD868C0F3801000E00120B1
:10A2C80002B0704700280040024BDA6822F0800292
:10A2D800DA6070470028004038B5104CCA23636222
:10A2E800532363620546FFF7CFFF90B1A36823F0BD
:10A2F8004003A360A2682B6842EA0303A360AB682B
:10A30800236123696A6843EA02432361FFF7DCFF9C
:10A318000120024BFF225A6238BD00BF00280040CE
:10A32800002382B001930E4BCA225A6253225A620A
:10A33800DA6822F0A002DA60DA6801990131019145
:10A348000199B1F5003F02D012F0200FF4D0044B70
:10A35800FF22D8685A62C0F3401002B0704700BFAD
:10A3680000280040F8B50C46C0B9204B08789B6817
:10A3780013F0400308BFCB70FFF772FF0746607801
:10A38800FFF76EFF0646A078FFF76AFFE57840EA18
:10A39800054545EA074545EA06250FE0134B4D7884
:10A3A8009B6813F0400308BFCB700B782D0245EA79
:10A3B80003458B781D43CB7845EA03450B4CCA23EC
:10A3C800636253236362FFF75FFF58B1084B05EAE6
:10A3D80003032360FFF778FFFFF7A2FF002814BFED
:10A3E80001200020014BFF225A62F8BD00280040DE
:10A3F8007F7F7F000023C3700370437083707047B2
:10A40800B1F802C00B8802884CEA0303B1F804C013
:10A4180002F4415243EA0C03B1F806C043EA0C03C4
:10A42800B1F808C043EA0C03B1F80AC043EA0C03C8
:10A43800B1F80CC043EA0C03B1F80EC043EA0C03B0
:10A4480042EA03039BB20380838B23F400631B045B
:10A458001B0C83830B8A038270470000838BF0B543
:10A4680023F47A6323F01F031B041B0C838302234A
:10A4780003848B68878B022BBFB23FD0DFF8BCC048
:10A488008A88DCF80840002A14BF0222012214F44A
:10A49800000F18BFDCF80840284D1CBF24F4000446
:10A4A800CCF80840D5F88440D5F884C06D68244EAF
:10A4B80005F03F05C4F38814B6FBF5F56C43CCF3FF
:10A4C800027CB4FBFCFCCC88B4F5007F08BF4FEAE3
:10A4D8001C2C02D05201BCFBF2FC0A2202FB0CFC31
:10A4E800BCFBF3F305330A229BB2B3FBF2F303F090
:10A4F80001021202C3F34F0392B200E00022A3F15B
:10A50800020C1FFA8CFCBCF1FE0F28BF002228BFEA
:10A518000223B1F806C0134343EA0C039BB2038439
:10A528000B884A8847EA030343F4006313438A8885
:10A5380013438A8913439BB28383F0BD00380240DA
:10A5480000127A0000230222038043808380C380A4
:10A5580082608381704721B103889BB243F0400336
:10A5680004E0038823F040031B041B0C038070479E
:10A5780021B1838B9BB243F4806304E0838B23F483
:10A5880080631B041B0C838370471AB183889BB2BA
:10A59800194303E083889BB223EA01018180704755
:10A5A800264ADFF89CC00388904214BF002201228B
:10A5B800604508BF42F0010210B59BB2CAB9214CF0
:10A5C800B0F1804F14BF4FF0000C4FF0010CA042C7
:10A5D80014BF64464CF001045CB91B4CDFF86CC036
:10A5E800A04214BF00240124604508BF44F00104C0
:10A5F8002CB1B1F802C023F0700343EA0C03144CE9
:10A60800DFF850C0041B18BF012460450CBF0024AC
:10A6180004F0010434B123F44073B1F808C09BB2CC
:10A6280043EA0C0303804B68C3620B8803850AB1B5
:10A638008B7A03860123838210BD00BF000001408E
:10A64800000401400004004000080040000C0040E5
:10A65800001000400014004021B103889BB243F071
:10A66800010304E0038823F001031B041B0C03808F
:10A6780070471AB183899BB2194303E083899BB25F
:10A6880023EA010181817047038A828911420CBF44
:10A698000020012019420CBF002000F00100704783
:10A6A800C94389B201827047038ACA889BB223F4DE
:10A6B8004053134330B503820D4683890989AA881C
:10A6C80023F4B05341EA0202698923F00C030A43D8
:10A6D8001B0492B21B0C42EA03038381838AAA8972
:10A6E8009BB223F44073134385B0044683826846C3
:10A6F800FFF7DCFC1C4B1D4A9C4214BF00230123BE
:10A70800944208BF43F001030BB1039B00E0029B96
:10A71800A28912B2002A2A6803DA19215943520081
:10A7280002E01921594392006423B1FBF2F1B1FB15
:10A73800F3F21201100903FB1011A08900B20028DE
:10A7480006DAC9003231B1FBF3F303F0070305E081
:10A7580009013231B1FBF3F303F00F0343EA0202BC
:10A7680092B2228105B030BD0010014000140140B2
:10A7780021B183899BB243F4005304E0838923F415
:10A7880000531B041B0C83817047C1F342134FF025
:10A79800010C01F01F0163450CFA01F101D10C30E5
:10A7A80004E0022B01D1103000E014301AB1036824
:10A7B80043EA010102E0036823EA010101607047EE
:10A7C800D0F8E43510B51B6904469847032384F88C
:10A7D8001231002010BD08B5042380F81231D0F8DA
:10A7E800E435DB689847002008BD08B5D0F8E035A7
:10A7F800DB6903B19847002008BD08B5D0F8E035FB
:10A808001B6A9847002008BD08B5D0F8E0355B6A98
:10A818009847002008BD002110B5402204460B4689
:10A8280000F0C6FF802140220023204600F0C0FF30
:10A83800012384F81231D4F8E435A0785B6898478E
:10A84800002010BD37B56946044600F015F99DF89B
:10A8580000106D4601F01F03012B07D0022B0AD010
:10A8680073B92046694600F0C7F90FE020466946EB
:10A8780000F0A8F90AE02046694600F031F905E041
:10A8880021F07F01C9B2204601F024F800203EBD26
:10A8980038B5044600293DD190F81131022B42D138
:10A8A800D0F83421D0F820319A4211D9C178D21A7F
:10A8B8000129C0F8342104D1D0F82411CB18C0F8EC
:10A8C800243192B22046D4F8241100F0A5F82AE0E9
:10A8D800D0F83821B2FBF3F503FB152565B99A4288
:10A8E8000AD3D0F83C319A4206D229462A4600F0CB
:10A8F80093F8C4F83C5116E0D4F8E035DB682BB186
:10A9080094F81221032A01D120469847204600F0E6
:10A91800A4F808E0D0F8E0355B6923B190F812217B
:10A92800032A00D19847002038BD10B5044659BB0A
:10A9380090F81131032B30D1D0F88C23D0F878332C
:10A948009A4214D9C178D21A0129C0F88C2304D1AB
:10A95800D0F87C13C918C0F87C139A4228BF1A464D
:10A9680092B22046D4F87C1300F05FF815E0D0F8D6
:10A97800E0351B6923B190F81221032A00D19847CA
:10A98800204600F05BF808E0D0F8E0359B6923B179
:10A9980090F81221032A00D19847002010BDF8B57D
:10A9A800044616461F460D46FEF740FA069B20460B
:10A9B800C4F8E4352946C4F8E075C4F8E86500F041
:10A9C800ABFED4F8E4351B6898472046FEF76AFAD0
:10A9D800F8BDD0F8E03510B51B6804469847D4F8A0
:10A9E800E4359B689847002010BD08B5D0F8E035DD
:10A9F8005B689847002008BD08B58C461346C0F828
:10AA08003821C0F83421022280F811210021624641
:10AA180000F03EFF002008BD8C4608B50021134613
:10AA2800624600F035FF002008BD8C4608B50021BD
:10AA38001346624600F004FF002008BD00210423ED
:10AA480010B50A46044680F811310B4600F020FF85
:10AA5800204600F041FE002010BD0021052310B55E
:10AA68000A46044680F811310B4600F0E9FE2046FC
:10AA780000F032FE002010BD90F8C8350B7090F839
:10AA8800C9354B7090F8CB2590F8CA3503EB0223F3
:10AA98004B8090F8CD2590F8CC3503EB02238B80C2
:10AAA80090F8CF2590F8CE3503EB02239BB2CB80EC
:10AAB800C0F83C31012380F81131704710B591F985
:10AAC80000300446002B01DBCB8813B920468021D7
:10AAD80000E0002100F0FEFE204600F0FDFD10BD64
:10AAE80038B50D466B780446012B097916D033D357
:10AAF800032B63D190F81231022B34D0032B59D198
:10AB08006B88FBB90B1E18BF012380290CBF0023DB
:10AB180003F00103B3B100F0DDFE13E090F8123149
:10AB2800022B20D0032B45D16B88002B46D10B1E5E
:10AB380018BF012380290CBF002303F001033BB198
:10AB480000F0E9FED4F8E03520469B68294698478E
:10AB58002046FFF773FF31E090F81231022B02D044
:10AB6800032B27D10CE00B1E18BF012380290CBF33
:10AB7800002303F001030BB3204600F0ABFE1DE0F9
:10AB880011F0800F07D001F07F01282303FB01019A
:10AB980091F81A2104E0282303FB010191F872239C
:10ABA800074B02B101221A60204605490222FFF72D
:10ABB80023FF03E020462946FFF780FF002038BD29
:10ABC8001452002038B590F812310446032B0D4674
:10ABD8000CD10B79012B09D8D0F8E0359B68984740
:10ABE800EB883BB92046FFF729FF03E020462946BA
:10ABF800FFF764FF002038BD73B54B7804460D4657
:10AC0800092B00F21C81DFE813F0D30010011A01B0
:10AC1800E3001A0172000A001A01C00092004B8872
:10AC28001A0A013A062A00F20A81DFE812F0070040
:10AC38001A0027000801080108010801D4F8E835BE
:10AC48000DF106011B68A0789847EB880146402B58
:10AC580003D094F81231012B3AD10822ADF806201E
:10AC680036E0D4F8E0350DF106019B6AA0789847E4
:10AC7800022343700146C4F8EC0529E0DBB2052B3A
:10AC880000F2DD80DFE803F003080D12171CD4F88A
:10AC9800E835A0785B6817E0D4F8E835A0789B68B9
:10ACA80012E0D4F8E835A078DB680DE0D4F8E83590
:10ACB800A0781B6908E0D4F8E835A0785B6903E060
:10ACC800D4F8E835A0789B690DF10601984701464C
:10ACD800BDF80630002B00F0B680EA88002A00F0A4
:10ACE800B2809A4228BF1A46ADF806205EE08B88EB
:10ACF800002B40F0A480CB88002B40F0A08094F873
:10AD080012214B88032A00F09A8003F07F05204621
:10AD180084F81351294600F01DFE2046FFF78EFEE9
:10AD28000DB1022300E0012384F812318BE0897809
:10AD3800464E0129317000F2828094F81231022BBC
:10AD480002D0032B7BD108E000294CD0012103233A
:10AD580084F8101184F8123113E041B9022384F801
:10AD6800123184F810112046FFF73FFE3BE094F8BB
:10AD78001011012937D02046FFF737FE317884F8C3
:10AD880010112046FFF725FE2DE0CA88012A56D16A
:10AD980094F81231022B02D0032B50D104E02C4935
:10ADA8002046FFF729FE4EE004F588712046F8E7B3
:10ADB80094F81231023B012B41D8D4F814312549BB
:10ADC800002B0CBF012303230B6020460122E8E778
:10ADD8004B88012B0BD1C4F81431D4F8E035204648
:10ADE8009B68294698472046FFF728FE2BE0022B50
:10ADF80029D18B8813F0FF0F25D121691B0A013B4C
:10AE08004A68042B0FD8DFE803F0030507090B0095
:10AE1800012306E0022304E0032302E0042300E008
:10AE2800052363F306124A60DDE794F81231023B0A
:10AE3800012B04D84B88012B05D1013BCBE72046D9
:10AE48002946FFF73BFE00207CBD00BF10520020C2
:10AE5800185200200C52002010B5D0B184460023AF
:10AE680000E0DBB21CF8014B0133002CF9D15B0088
:10AE78009BB213800B7003234B70013B05E0CA544F
:10AE88005A1CD2B202338C54DBB210F8012B002AC0
:10AE9800F5D110BD73B50024114D06460194032069
:10AEA800FEF70EF8336801341A69AC42019215D0E6
:10AEB800019A002AF3DA019A42F001020192019AFA
:10AEC8001A61074A196912F1FF32019103D00199F9
:10AED80011F0010FF6D10320FDF7F2FF00207CBD31
:10AEE800410D030010B5C47874B900EB8200033338
:10AEF8009B10D0F8D000224604E051F804CB013270
:10AF0800C0F800C09A42F8D3002010BD0332D0F830
:10AF1800D0C010B592100846002304E0DCF80040C9
:10AF2800013340F8044B9342F8D301EB820010BD83
:10AF3800012270B50023827040220129C3708280EB
:10AF48000CD108330370042343704FF4A073C380FB
:10AF580002230372C1724FF0A04309E041B90C23E8
:10AF68000370062343704FF4A062224BC172C28063
:10AF7800457803F5006201350261C36001466D0141
:10AF8800002203F50E6403F52E6C04E0A6184E614A
:10AF98000CEB02060E6520320431AA42F6D10146B6
:10AFA80011F88CCB03F58062426103EB4C1403F576
:10AFB8008862C0F8CC2004F5A06403F5A06202E022
:10AFC80041F8042F2032A242FAD103EB0C3C00F1E5
:10AFD800CC010CF5805C1A4601E041F8042F02F51B
:10AFE80080526245F9D103F56063C0F80C31002046
:10AFF80070BD00BF0000044038B5037A0025012B5E
:10B008000446C26826D1936B417A65F3104309B1AF
:10B0180043F480139363D36804F10C006FF3861331
:10B028006FF3965343F010036FF3C3036FF3C71323
:10B038006FF351436FF3D343D360FFF72BFFE378EC
:10B04800012B40D1043363F34405E36845F0200540
:10B058009D6038E0D36800F10C0043F04003D360F2
:10B06800FFF718FF237A627A032B14BF4FF43413C7
:10B078004FF43C130AB143F48013E268142093633D
:10B08800FDF723FFE268217AD368032908BF43F458
:10B098008033D360237A032B15D1156B012363F317
:10B0A8009B656FF3D7552C3345F0805563F31645F0
:10B0B8001563C820FDF709FFE36845F400051D6323
:10B0C800C820FDF702FFE378012B07D1E3680522CA
:10B0D8009D6862F3440545F020059D60002038BD59
:10B0E800C36800209A6842F001029A607047C368FA
:10B0F80000209A6822F001029A60704707B5002381
:10B108000193019A42F020020192019A61F38A1296
:10B1180001920199C26811610749106901338B4294
:10B12800019003D0019810F0200FF6D10320FDF70D
:10B13800C7FE00200EBD00BF410D030007B5002368
:10B148000193019A42F0100201920199C2681161BB
:10B158000749106901338B42019003D0019810F020
:10B16800100FF6D10320FDF7ABFE00200EBD00BF87
:10B17800410D0300C26808B5D36801296FF35D73F8
:10B188006FF39E7308BF43F0005302D009B943F030
:10B1980080433220D360FDF798FE002008BDC368C5
:10B1A8005B6913F0010F14BF002001207047C368CA
:10B1B8005A6998691040704703691A6861F3010277
:10B1C8001A607047C26800239361013B5361536062
:10B1D80053610B4B9361C3789169002B14BF4FF4F3
:10B1E80000634FF4016343F4701343F4405343F096
:10B1F800080321EA030141EA030393610020704731
:10B208000008008038B5D0F80C3100221A600369B4
:10B2180015461A68044665F3CC221A60C37A012BD6
:10B228001AD10321FFF7C8FFE36880214FF4800299
:10B2380061F30F0259629A62C02262F30F0561F34B
:10B248001F455218C3F8045162F30F056FF31F45E9
:10B25800C3F80851C3F80C5110212046FFF74EFFE0
:10B268002046FFF76BFF226900234FF0FF3113617F
:10B2780004F1140053619E4691614FF0FF0CD361B5
:10B2880012E050F8042F01331168C1F3076101F08F
:10B298008001C9B2002914BF4FF09041002111600C
:10B2A800C2F810E0C2F808C062789342E9D30023DC
:10B2B80004F150009E464FF0FF0C12E050F8042FA6
:10B2C80001331168C1F3076101F08001C9B2002997
:10B2D80014BF4FF0904100211160C2F810E0C2F88D
:10B2E80008C062789342E9D32269136943F48073F2
:10B2F8001361E378012B08D14021023361F38A03FB
:10B3080043F4803361F3594313632046FFF75AFF30
:10B31800002038BD03699B68C3F341035A1E022A03
:10B3280004D8034AD31813F8010C00E0032070472F
:10B3380064E7000803698169D3F808C00A68CCF398
:10B348004100022818BF6FF30A0202D1032060F3FC
:10B358000A020A605A68002042F480725A607047F4
:10B3680010B54C780022012C0B7808D100EB830C27
:10B3780014FA03F3DCF818C063F30F0208E00124A1
:10B3880000EB830C14FA03F3DCF854C063F31F4298
:10B39800DCF80030C3F3072404F08004E4B274B985
:10B3A8008C6864F30A03CC78C98864F3934361F327
:10B3B800995343F0805343F40043CCF800300369B9
:10B3C8000020D9690A43DA6110BD10B54C784FF0F6
:10B3D800000C012C62460B7807D100EB830114FAAC
:10B3E80003F3896963F30F0207E0012400EB83018B
:10B3F80014FA03F3496D63F31F4203696FF3CF3CFB
:10B40800C1F800C0D969002021EA0202DA6110BD42
:10B4180038B54D780B78012D4C6955D100EB830375
:10B42800D3F818C0DCF80030DCF8102024B964F335
:10B43800120265F3DC420DE08D6864F312026419B0
:10B44800013CB4FBF5F5CC7865F3DC42012C08BF70
:10B4580064F35E72CCF81020C278012A08D10A7809
:10B46800D1F810C000EB82029269C2F814C00FE054
:10B47800CA78012A0CD04A6952B191F800C0012556
:10B4880005FA0CFC0269546B4CEA040CC2F834C08F
:10B49800CA78012A08D10269926812F4807F0CBF29
:10B4A80043F0005343F080530A7843F0044300EB21
:10B4B800820292691360CB78012B3ED10A788B8A7D
:10B4C800C968FFF70FFD38E000EB83035D6DD1F825
:10B4D80008C02B682A6934B96CF312024FF0010CCA
:10B4E8006CF3DC420BE06444013CB4FBFCF4A405BF
:10B4F800A40D0CFB04FC64F3DC426CF312022A6119
:10B50800C278012A01BF0A78D1F810C000EB820284
:10B51800526D08BFC2F814C0CA78012A06D14A7908
:10B5280012B143F0005301E043F080530A7843F02E
:10B53800044300EB8200426D1360002038BD73B5F0
:10B548004D784C69012D45D1D0F818C0DCF8003091
:10B55800DCF81020009254B99DF8002064F306022C
:10B568008DF800209DF8022065F3C40210E08D6874
:10B578009DF80020AC4286BF4D6165F3060264F376
:10B5880006028DF800209DF80220012464F3C4020D
:10B598008DF80220009A43F00443CCF81020C278BA
:10B5A800012A01BF0A780C6900EB8202926908BF80
:10B5B8005461CCF80030C378002B45D14B69002B7F
:10B5C80042D00A78012111FA02F20369586B02434A
:10B5D8005A6339E00B7800EB8303D3F854C0DCF8E6
:10B5E8000030DCF810500095EAB2C5F307468D68C4
:10B5F8004CB965F306028DF80020012262F3C406F7
:10B608008DF802600AE065F306024D618DF80020AE
:10B618003546012262F3C4058DF80250009A43F0C2
:10B628000443CCF81020C278012A01BF0A78D1F867
:10B6380010C000EB8202526D08BFC2F814C00A782D
:10B6480000EB8200426D136000207CBD4B78012B1B
:10B658000B780CD100EB830082691368C3F3076190
:10B6680001F08001C9B231B143F0804303E000EB3F
:10B678008300426D136843F4001313600020704781
:10B688004B78012B0B78C9780BBF00EB830000EBDC
:10B6980083008369436D02391A68C9B26FF3555242
:10B6A800012998BF42F080521A6000207047036950
:10B6B8009A69D8691040000C704700EB81014B6D06
:10B6C80002699B6850691840704703699869DB698B
:10B6D800184080B27047000082B000230093C03346
:10B6E8008DF803300122002362F3C4038DF8023081
:10B6F80018238DF80030436D009A1A61C278012A28
:10B7080001BF00F5B96058611A68024A08BF1A609B
:10B7180002B070470080008038B50446FFF708FC87
:10B728000120002184F81201054684F8131194F8C9
:10B7380001C02346224608464FF0400E0EE082F82C
:10B74800F010A2F8F61082F8F15082F8F300C2F86F
:10B75800F8E0C2F8FC00C2F8040101312832614562
:10B76800EDD30022114640200EE083F84823A3F8C9
:10B778004E2383F8491383F84B13C3F85003C3F8D7
:10B788005413C3F85C13013228336245EDD32046C5
:10B79800FFF7ADFC2046FFF72FFC00212046FFF7FE
:10B7A800E9FC2046FFF72EFD2046FFF799FC38BD3F
:10B7B80010B5CCB214F0800F14BF4FF0280E4FF024
:10B7C800280E8C4601F07F0115BF0EFB01F10EFB20
:10B7D80001F101F58C7101F55C7141180CF07F0CD9
:10B7E800E40981F800C04C708A60CB700CB1A1F8F4
:10B7F80006C0022B01D100230B71FFF7B1FD002019
:10B8080010BDCAB212F0800F14BF4FF0280C4FF0D1
:10B81800280C08B501F07F0315BF0CFB03F30CFBE4
:10B8280003F303F58C7303F55C73C318D20901F0B5
:10B838007F0119705A701946FFF7C7FD002008BD2F
:10B8480008B54FF0280C01F07F0E0CFB0EFC0CF530
:10B858005C718444CCF8843300238CF870E38CF852
:10B868007133CCF88833C3784118012B08BFCCF862
:10B878008023282303FB0E0E9EF87033CCF87C231C
:10B8880013B9FFF75CFE01E0FFF7C2FD002008BD19
:10B8980010B54FF0280C01F07F040CFB04FC0CF5EC
:10B8A8008C7184444FF0010ECCF82421CCF8282167
:10B8B800002241188CF819E18CF81841CCF8302195
:10B8C800CCF82C3114B9FFF73AFE01E0FFF7A0FDE0
:10B8D800002010BDCAB212F0800F08B508D001F0E0
:10B8E8007F034FF0280C0CFB03F303F58C7303E084
:10B8F80028234B4303F55C73C3184FF0010CD2099E
:10B9080001F07F01197083F802C05A701946FFF7D9
:10B918009DFE002008BDCAB212F0800F10B508D0F5
:10B9280001F07F034FF0280C0CFB03F303F58C7335
:10B9380003E028234B4303F55C73C3180024D209A2
:10B9480001F07F0119709C705A701946FFF798FE34
:10B95800204610BD0369002261F30A1219680A43E0
:10B968001A60704708B5036903205A686FF34102EB
:10B978005A60FDF7AAFA08BD08B5036903205A689A
:10B9880042F002025A60FDF7A0FA08BDF0B587B090
:10B998000446FFF704FC002800F06C822046FFF7FD
:10B9A80006FC0290002800F06482C0F3074000F013
:10B9B8000800C0B2002864D02046FFF778FE039044
:10B9C800002027462646049057E0039911F0010FFE
:10B9D80048D0049B2046DAB211460192FFF76DFE6B
:10B9E80010F0010F0546019A21D0736D01259D6065
:10B9F800E178A94207D11B69D7F87813C3F312037A
:10BA0800CB1AC7F88833DFF870C42046DCF800305A
:10BA180011461B689847E378012B08D1049830B980
:10BA280094F81131052B02D12046FFF755FE05F099
:10BA38000203DBB213B1736D02259D6005F00403A8
:10BA4800DBB213B1736D04259D6005F00805EDB2F6
:10BA580045B1DFF8241420460B689B689847736D3E
:10BA680008229A60049BDDF80CC001334FEA5C0C95
:10BA78000493CDF80CC00436283703980028A4D1C5
:10BA880001300299C1F3074303F00403DBB2002B32
:10BA980000F0C6802046FFF718FE002204902546D5
:10BAA800274603922646B5E0049B13F0010F00F0E9
:10BAB800A6803369DDF80CC019695C6B5FFA8CFCF1
:10BAC80024FA0CF406EB8C029269E401926804F003
:10BAD800FF040C43144014F0010FCDF814C01DD01E
:10BAE800DDF80CC0012000FA0CF15A6B044622EA7A
:10BAF80001025A63AB6905999860DF4803683046CC
:10BB08005B689847F378A34208D1039931B996F84E
:10BB18001131042B02D13046FFF7DEFD04F0040397
:10BB2800DBB213B1AB6904249C6004F00803DBB2F8
:10BB380013B1AB6908249C6004F01003DBB213B1A5
:10BB4800AB6910249C6004F02003DBB213B1AB692D
:10BB580020249C6004F04003DBB213B1AB6940249D
:10BB68009C6004F00203DBB213B1AB6902249C6051
:10BB780024F07F0414F0FF0F41D0D7F83031D7F804
:10BB88002CC1C3EB0C0CD7F820319C4528BF9C4630
:10BB98000CF1030CAB694FEA9C0C64469B69B446F4
:10BBA8001EE0D7F820219E1B964228BF1646B3B246
:10BBB8006046D7F82411059ACDF804C0FFF792F92A
:10BBC800D7F82431F41C9B19C7F82431D7F8303141
:10BBD800DDF804C09E19AB69C7F830619B69A408F9
:10BBE8009BB2A34207D9D7F83061D7F82C319E42CF
:10BBF80001D2002BD5D1AB69802266469A60039B9F
:10BC0800DDF810C001334FEA5C0C0393CDF810C087
:10BC180004352837049800287FF446AF34460130AD
:10BC2800029901F00203DBB213B1E36802225A6100
:10BC3800029AC2F3076303F08003DBB2CBB1A37AA5
:10BC480043B1D4F80C31D4F80C216FF341036FF3EE
:10BC580000031360236920465A6822F001025A60E3
:10BC6800854B1B689B699847E3684FF000425A610F
:10BC78000120DDF808C0CCF3072303F00803DBB28A
:10BC8800FBB17D4B20461B685B6998472369E268D6
:10BC98004FF400619B685161A27A8AB113F0010FD9
:10BCA8000ED0D4F80C311A6842F001021A601A68F2
:10BCB80042F003021A60714B1A6942F006021A61D7
:10BCC8000120029901F00803DBB243B16A4B204618
:10BCD8001B68DB689847E36808225A610120029ACA
:10BCE80002F01003DBB2002B3AD0E3689A6922F025
:10BCF80010029A611D6AC5F34343022B05F00F0633
:10BD080002D0062B26D115E047F6F07305EA0303A7
:10BD180003B3282303FB0646C5F30A152046D6F8C5
:10BD28007C132A46FFF7F2F8D6F87C335B19C6F87D
:10BD38007C330AE004F5B96120460822FFF7E6F8EB
:10BD4800282303FB0646C5F30A15D6F88833ED18F1
:10BD5800C6F88853E36801209A6942F010029A6194
:10BD6800DDF808C0CCF3072303F01003DBB2002B87
:10BD780036D0236900255A68294622F001025A6004
:10BD88002046FFF7BBF904F114022B46FF2105E01A
:10BD980052F8040F01338160D06B81606078834270
:10BDA800F6D3236901264FF0FF3266F30F059A6137
:10BDB80066F31F451032DD615A6120321A611A6834
:10BDC80020466FF30A121A60FFF786FCE3684FF407
:10BDD80080525A61284B20461B681B699847304699
:10BDE8000299C1F3072303F02003DBB2EBB120462D
:10BDF800FFF7A0FAE3682046DD68FFF78BFA03280F
:10BE080006D100234FF40072A370A280093304E026
:10BE18000123A3704023A380052363F38D25E368E2
:10BE28004FF40052DD6001205A61DDF808C0CCF300
:10BE3800074303F01003DBB24BB10F4B20461B68DE
:10BE4800DB699847E3684FF480125A610120029930
:10BE5800C1F3074303F02003DBB25BB1064B204676
:10BE68001B681B6A9847E3684FF400125A61012067
:10BE780000E0029807B0F0BD3800002000ED00E0B7
:10BE880070B51D4B01461878012802D8FCF7EAFD69
:10BE980030E01A4A937852785343023B48BF6FF018
:10BEA800010027D4042B02DC0238C0B21FE03E2B6D
:10BEB800A8BF3E23DC1013F0070F18BF0134023867
:10BEC800C6100D4659B100F0070001258540EDB2B6
:10BED80005E0B4420CBF28460020FCF701FC013CF9
:10BEE800F7D200210220FCF7F8FB02200121FCF721
:10BEF800F4FB002070BD00BFE44D0020FC82002050
:10BF080038B51F4B1878012804D840F6C411FCF73F
:10BF1800D3FD33E03F282FD80020FCF787FD012010
:10BF2800FCF7C8FD0120FCF78FFD0120FFF7A8FFF3
:10BF3800002821DB40F6C4140120FFF7A1FF0025EB
:10BF480001200135FCF780FD0A2DF9D1FCF7AAFD87
:10BF580005460020FFF794FF15B114F1FF34EBD12B
:10BF68000020FCF7A7FD0020FCF76EFD002C14BF95
:10BF780000206FF0010001E04FF0FF3038BD00BF36
:10BF8800E44D002070B53B4B05469A785C783A4BF7
:10BF98005443083C382CA8BF382400B31A78FF2A29
:10BFA80065D0FF2200201A70FCF702FC042C09DC83
:10BFB800002504E0E8B20021FCF78FFB0135A5421B
:10BFC800F8DB54E0E31014F0070F18BF01331C46E8
:10BFD80002E00020FCF784FB013CFAD23FE0274A4C
:10BFE80019781278914242D001269640F6431A7089
:10BFF800F0B2FCF7DDFB042C0DDC09E005F10801CB
:10C0080036FA01F1E8B201F00101FCF766FB0135EF
:10C01800A542F3DB2BE0194BE210197814F0070F57
:10C02800174B18BF0132083901EA03030826002B11
:10C0380091FBF6F603DA013B63F0070301330125B0
:10C048009D40ED43EDB2541E06E0B4420CBF2846B5
:10C05800FF20FCF745FB013CB4F1FF3FF5D100217F
:10C068000220FCF73AFB02200121FCF736FB0020F6
:10C0780070BD00BFFC82002068000020E44D002055
:10C0880007000080F7B53C4B04461D78002D6FD1A2
:10C098003A4B1E783A4B3246D3E9000101F0F0FDE5
:10C0A8000122002302400B4052EA030160D0354BC5
:10C0B8001A787F32D3B2052B36D8012752B217FA35
:10C0C80002F212F0230306D112F018051ED112F065
:10C0D800040F11D128E0012E4AD8FFF711FF20469E
:10C0E800FCF766FB2846FCF7A1FC3846FFF7C8FEBC
:10C0F8002846FFF7C5FE3DE03846FFF743FF2846D0
:10C10800FCF794FC2046FCF701FC33E03846019329
:10C11800FFF738FF019B6FF002051846FCF786FC15
:10C128002046FCF7F3FB25E0FFF7EAFE002811DACA
:10C13800124B01201A78002101F0AEFD104C6FF06F
:10C148000105D4E9002322EA000023EA0101C4E939
:10C1580000010FE02046FCF72BFB0020FCF766FCF3
:10C168000120FFF78DFE0020FFF78AFE002501E081
:10C178004FF0FF352846FEBD1C520020E44D00203C
:10C1880020520020FC820020F7B5684B05461B783A
:10C198000193002B40F0C3806548664C0678D4E9CB
:10C1A8000001324601F06CFD02460B4601200021D9
:10C1B80002400B4052EA030100F0B1805E4F3A782A
:10C1C8007F32D3B2052B00F28780012352B213FAD3
:10C1D80002F212F0230306D112F018045CD112F017
:10C1E800040F3CD178E0012E00F29980534EBB88B1
:10C1F80032889A4280F09380514B1A88FB889A4281
:10C2080080F08D80FFF77CFE0028BCBF484802788C
:10C2180069DB2846FCF7CCFA0120FCF707FC012073
:10C22800FFF72EFE0198FFF72BFE3B78862B0DD1EA
:10C2380033883D2201339BB2B3FBF2F1338002FB1A
:10C2480011339BB2002B6DD1002022E033880133DB
:10C258009BB213F03F0F338064D1402019E0204691
:10C26800FFF790FE0120FCF7E1FB2846FCF74EFBA8
:10C27800324A138801339BB21380BA88B3FBF2F5B4
:10C2880002FB1535ADB2002D4ED11020FFF7FAFE96
:10C298002846FFF7F7FE48E018460093FFF772FEBE
:10C2A8000120FCF7C3FB2846FCF730FB2349009B21
:10C2B8000A881846013292B20A80B988B2FBF1F4B2
:10C2C80001FB1424A4B2002C2FD12046FFF7DAFE7C
:10C2D8001020FFF7D7FE27E0FFF712FE002811DA3B
:10C2E800134B144C1A780120002101F0D5FCD4E935
:10C2F800002322EA000023EA0101C4E900016FF0EB
:10C30800010012E02846FCF753FA0120FCF78EFBE7
:10C318000120FFF7B5FD0020FFF7B2FD02E04FF066
:10C32800FF3002E0002000E02046FEBD1C52002045
:10C33800E44D002020520020FC8200200E830020C3
:10C34800F8820020F0B5DC4B85B01B78002B40F05C
:10C35800AE81002840F0AB81D84B1C783F2C00F20E
:10C36800A38122460120002101F096FCD44DD5E995
:10C3780000231943D34B1043C5E900011D78A5F1EB
:10C388008103052B00F2F680DFE803F003031F7634
:10C39800760E012C00F27A810120FCF7A5F900281D
:10C3A800C0F282813F200CE0012C00F26F81012055
:10C3B800FCF79AF90028C0F27781E220FFF762FEC5
:10C3C800AF20FFF75FFEC0205EE1002C40F05E81E9
:10C3D8002046FCF789F90028C0F26681B84EFF2292
:10C3E8000023D6E9000102430B43C6E90023B54BFD
:10C3F80001279A785D785543083D042DA8BF042588
:10C408000FE0E0B20521FCF765F9D6E9002304F155
:10C41800080117FA01F10A4343EAE173C6E9002368
:10C428000134AC42EDDB4020FFF72CFEA120FFF7E2
:10C4380029FEC020FFF726FEA620FFF723FEA22034
:10C44800FFF720FE2F20FFF71DFEF820FFF71AFE4A
:10C458000020FFF717FE2720FFF714FE8120FFF7C3
:10C4680011FE1020FFF70EFEAC20FFF70BFE002098
:10C47800FFF708FEAF2007E1002C40F007812046B7
:10C48800FCF732F90028C0F20F818D4FFF220023FC
:10C49800D7E9000102430B43C7E90023894B4FF05A
:10C4A800010C9A785E785643083E042EA8BF0426ED
:10C4B80013E0E0B20521CDF804C0FCF70BF9D7E989
:10C4C8000023DDF804C004F108010CFA01F10A4365
:10C4D80043EAE173C7E900230134B442E9DB0024ED
:10C4E8004FF47A700134FCF7AFFBB4F5FA7FF7D15B
:10C4F800A820FFF7C7FD3F20FFF7C4FDD320FFF7B3
:10C50800C1FD0020FFF7BEFD4020FFF7BBFD852DD4
:10C5180004D0A020FFF7B6FDC02003E0A120FFF75C
:10C52800B1FDC820FFF7AEFDDA20FFF7ABFD122002
:10C53800FFF7A8FD8120FFF7A5FD7F20FFF7A2FDEB
:10C54800A420FFF79FFDA620FFF79CFDD520FFF74D
:10C5580099FD8020FFF796FD8D20FFF793FD1420AD
:10C56800FFF790FDAF20FFF78DFD2020FFF78AFD34
:10C57800022089E0012D01D1002000E00120FCF714
:10C58800B3F80028C0F290804E4A9378527853430B
:10C59800012B1ADD062B08DC0024E0B2052101344A
:10C5A800FCF798F8042C10D0F7E705210020FCF7D9
:10C5B80091F805210120FCF78DF805210220FCF7F0
:10C5C80089F802200121FCF788F83820FCF7F0F8F8
:10C5D8000020FCF72BFA0020FCF736FA0120FFF7C1
:10C5E8004FFC0020FFF74CFC41F28830FCF72CFB95
:10C5F8000120FFF745FC0020FFF742FC4FF4FA70DA
:10C60800FCF722FB0120FFF73BFC0020FFF738FC7A
:10C618004FF4FA70FCF718FB0820FFF733FD274B9F
:10C628001A78274BD3E9000101F02AFB01220023E5
:10C638001040194050EA010339D00C20FFF722FDC1
:10C648000620FFF71FFD0120FFF71CFD1D4B1B787F
:10C65800012B15D13920FFF715FD1D20FFF712FD1D
:10C668005020FFF70FFD6C20FFF70CFD7C20FFF733
:10C6780009FD154B04A81B6840F8043DF9F742FC76
:10C688003820FFF7FFFC0C20FFF7FCFC0B4B1A7857
:10C698000B4BD3E9000101F0F3FA10F0010F0CBFC6
:10C6A8004FF0FF30002004E06FF0010001E04FF090
:10C6B800FF3005B0F0BD00BF1C520020E44D002043
:10C6C80020520020FC82002068E70008F8B5434BA0
:10C6D8004FF0FF301D78002D7ED1414E33787F33E7
:10C6E800DAB2052A75D801225BB212FA03F313F005
:10C6F800230406D113F0180544D113F0040F20D1F8
:10C7080067E03848F9F75EFC2C460FE0A9B2002034
:10C71800F9F7CAFB0027044304E00020FFF734FDC3
:10C7280001370443B3889F42F7DB0135F388B5EB43
:10C73800D30FEBDB00200146F9F7B6FB44EA000013
:10C748004AE02848F9F73EFC2C4616E0214600202E
:10C75800F9F7AAFB05430120FFF714FC0120FCF7B9
:10C7680065F9002704E00020FCF7D0F80137FFB294
:10C77800B388BB42F7D80134E4B2F388B4EBD30FE3
:10C78800E4D31FE01748F9F71DFC254616E02146BB
:10C798000020F9F789FB05430120FFF7F3FB01208F
:10C7A800FCF744F9002704E00020FCF7AFF8013754
:10C7B800FFB2B388BB42F7D80134E4B2F388B4EBD4
:10C7C800D30FE4D300200146F9F76EFB45EA0000D9
:10C7D80002E00120FFF756FCF8BD00BF1C52002004
:10C7E800FC8200206CE70008F8B5334B04461B7840
:10C7F8000D464FF0FF30002B5CD1304B1B78813B4E
:10C80800052B55D8DFE803F003031B3E3E0D04F06B
:10C818003F0444F04000FFF735FCC5F3C205044669
:10C828000AE03D23B4FBF3F003FB1044E0B2FFF74A
:10C8380029FCC5F3C105044645F0B80033E01F4E96
:10C84800ED08B388B4FBF3F003FB1040C0F303100A
:10C8580040F01000FFF716FCB3880746B4FBF3F06E
:10C8680003FB104404F00F00FFF70CFCF38840EAC8
:10C878000704DB0895FBF3F003FB105565F04F0048
:10C88800C0B210E004F00F00FFF7FCFBC4F3031480
:10C89800064644F01000FFF7F5FBC5F3C20540EA71
:10C8A800060445F0B000FFF7EDFB44EA000001E0A4
:10C8B8006FF00200F8BD00BF1C520020FC8200206F
:10C8C80008B50E4B1B78B3B90D4B93F90030002B0C
:10C8D80006DA0C4B18880C4B1988FFF785FF0CE01B
:10C8E800032908D8094B5B5C181860F07F00C0B2B8
:10C8F800FFF7C8FB01E04FF0FF3008BD1C520020D5
:10C90800FC8200200E830020F8820020088300208B
:10C918006FF0020070476FF002007047F0B587B003
:10C9280003AB83E80700244B1C78002C3FD1F9F7B0
:10C93800ADFA00283BD0214B214A1E889288B2428A
:10C9480098BF6FF0010034D91E4FBDF812503A88D5
:10C95800ED0801921DE0BDF81420039B02FB04338F
:10C96800029344B13988154B083189B21E80398049
:10C978003046FFF739FF002306E0029AD05C0093A7
:10C98800FFF702FC009B0133BDF810209342F4DB53
:10C998000134AC42DFDB28465DB1019A094B1146F0
:10C9A8001A80064B1888FFF71FFF002001E04FF0A0
:10C9B800FF3007B0F0BD00BF1C5200200E830020DE
:10C9C800FC820020F882002010B5044680B9094B8B
:10C9D8004FF0FF3201201A60FAF748FC00280146A0
:10C9E800C8BF204605DC0448F9F7B0FE022000E085
:10C9F800012010BD2852002070EA0008003818BF36
:10CA080001207047F7B51E46C0B90D46044611E02F
:10CA1800A718294638460192FAF770FC002805F550
:10CA28000075019A05DA06483946F9F78FFE0120A4
:10CA380005E00134B442EBDB002000E00420FEBD39
:10CA4800B0EA0008F7B51E46C0B90D46044611E025
:10CA5800A718294638460192FAF79CFC002805F5E4
:10CA68000075019A05DA06483946F9F76FFE012084
:10CA780005E00134B442EBDB002000E00420FEBDF9
:10CA8800DBEA000800207047002304E011F803C027
:10CA980000F803C00133013AF8D2704701E000F80A
:10CAA800011B013AFBD27047F7B5C56A04468D42AF
:10CAB8000E462CD00379F3B100F1300301931946E7
:10CAC80040782A460123FFF7BDFF10BBA269236AFD
:10CAD8002071D3189D4238BFE7780AD30BE0A369C9
:10CAE8006078ED1801992A460123FFF7ABFF013F53
:10CAF800FFB2012FF3D8304666B1607804F13001F7
:10CB080032460123FFF77EFF18B9E66202E00020F3
:10CB180000E00120FEBD000010B504460A4640783A
:10CB280004F130010123FFF76DFF80BB94F82E322A
:10CB380094F82F2243EA0222174B12B29A4228D1C4
:10CB480094F8682094F86930120442EA036294F871
:10CB580066301A4394F8673042EA03220F4B22F0FA
:10CB68007F429A4216D094F8840094F885200004F5
:10CB780040EA026094F88220104394F8832040EA47
:10CB8800022020F07F40C01A18BF012002E00320D5
:10CB980000E0022010BD00BF55AAFFFF4641540027
:10CBA80008B560B1037853B1C3888B4207D1407888
:10CBB800FFF724FF10F0010018BF032000E0092050
:10CBC80008BD0129F7B504460D4657D9C3699942EE
:10CBD80054D20378066A022B28D0032B35D0012BB8
:10CBE8004ED101EB510706EB5721FFF75DFF0028F7
:10CBF80046D1FB0504EBD35393F83030013706EBED
:10CC0800572120460193FFF74FFF019BC0BBFF054B
:10CC180004EBD75494F8300015F0010F43EA0020D4
:10CC280001D000092EE00005000D2BE006EB1121D4
:10CC3800FFF73AFF20BB2D0604EBD55494F83100DA
:10CC480094F8303043EA00201CE006EBD111FFF7DE
:10CC58002BFFA8B96D0604EBD55494F8320094F86C
:10CC68003330000440EA036094F83030184394F8F5
:10CC7800313040EA032020F0704003E0012001E059
:10CC88004FF0FF30FEBD0129F7B504460D461646A4
:10CC98006DD9C36999426AD20378076A022B3ED0DC
:10CCA800032B4BD0012B5ED101EB510307EB532132
:10CCB8000193FFF7F9FE019B002855D1D805C00D57
:10CCC80015F001021CBF04EB000C9CF830C0F1B257
:10CCD8001EBF0CF00F0C4CEA0111C9B220185D1CE4
:10CCE800012380F83010237107EB5521204601926B
:10CCF800FFF7DAFE019AB8BBED05ED0D12B1C6F3E8
:10CD0800071608E0631993F83030C6F3032623F0BA
:10CD18000F0343EA0606651985F8306024E007EB3F
:10CD28001121FFF7C1FEF8B92D0604EBD55585F89A
:10CD38003060C6F3072685F8316015E007EBD1119E
:10CD4800FFF7B2FE80B96D0604EBD555C6F307238D
:10CD580085F8306085F83130330C360E85F832307E
:10CD680085F8336000E002200123237100E00220EF
:10CD7800FEBDF7B5C36905460E4661B9C768D7F168
:10CD8800010238BF00229F4228BF42F00102002A58
:10CD980018BF012708E00193FFF713FF0128019B43
:10CDA80035D998423DD337463C4601349C4202D39C
:10CDB800012F2ED90224284621460193FFF701FFAF
:10CDC800019B60B1B0F1FF3F14BF0022012201288E
:10CDD80008BF42F0010222BBBC42E6D11BE0284654
:10CDE80021466FF07042FFF74EFFB0B92EB12846CA
:10CDF80031462246FFF747FF78B92B69EC60B3F15B
:10CE0800FF3F0DD0013B2B6101236B7108E001202E
:10CE180007E0002005E0104603E04FF0FF3000E097
:10CE28002046FEBD0129F8B504460F4624D9C3693A
:10CE380099421AD320E020463946FFF7C2FE05463C
:10CE4800C8B1012818D0B0F1FF3F17D020463946A5
:10CE58000022FFF718FF90B92369B3F1FF3F02D012
:10CE68000133236166712F4600E00126E3699F4282
:10CE7800E1D3002003E002E0022000E00120F8BD39
:10CE8800C3690239023B99423DBF8278836A02FB3B
:10CE980001300020704770B504460D46E180816876
:10CEA80001293AD00368DA69914236D279B91A78F9
:10CEB800032A01D1596A51B90022E2601A89AA42AB
:10CEC80082BF5B6A03EB151323611BD825E09E78AC
:10CED80036010EE02068FFF774FEB0F1FF3F01460F
:10CEE80019D0012819D92368DB69984215D2AD1BDE
:10CEF800ADB2B542EED2E1602068FFF7C1FF00EBAA
:10CF080015102061236805F00F05303303EB451534
:10CF18006561002002E0012000E0022070BDF7B545
:10CF2800C68804460136B6B20F46002E69D003699A
:10CF3800002B66D016F00F0F59D1C1680133036179
:10CF4800006819B90389B34251D85AE08378013B84
:10CF580013EA16134BD1FFF734FE0128054654D9BE
:10CF6800B0F1FF3F53D02068C3699D4239D3002FE9
:10CF780047D0E168FFF7FDFE0546002843D00128A9
:10CF880043D0B0F1FF3F42D020680021FFF78CFD6D
:10CF9800074600283BD12068394630304FF40072EC
:10CFA800FFF77CFD2368294618460193FFF768FFC1
:10CFB800019BD86201230DE01371206800210193C1
:10CFC800FFF772FD019B10BB22680137D16AFFB2DF
:10CFD8000131D16222689178B942EDD8D36ADF1B5A
:10CFE800D762E56020682946FFF74AFF2061236879
:10CFF800E680303306F00F0603EB46166661002024
:10D0080006E0042004E0072002E0022000E00120FE
:10D01800FEBD0000F7B504460B780D460131202B04
:10D02800FAD02F2B14BF002201225C2B14BF134609
:10D0380042F001030026002B18BF0D46A6602B788E
:10D048001F2B05D820463146FFF725FF6661C8E04B
:10D05800A669202130460B22FFF720FD002101910F
:10D0680008200A46DDF804C015F80C300CF1010C54
:10D07800202B8CBF002701272F2B08BF47F0010763
:10D08800CDF804C0002F44D15C2B46D02E2B14BF02
:10D09800002701278142A8BF47F001077FB12E3B37
:10D0A80018BF012308280CBF184643F001000028C8
:10D0B80040F094809200D2B208210B30D2E713F0EE
:10D0C800800F04D0DFF81CC1803B1CF80330DFF868
:10D0D80018C137461CF8016F16B19E42FAD17DE09F
:10D0E800A3F1410C5FFA8CFCBCF1190F3E4698BFC6
:10D0F80042F002020AD9A3F1610C5FFA8CFCBCF180
:10D10800190F03D8203B42F00102DBB273540131FE
:10D11800A8E7202B94BF0427002700295ED0337886
:10D12800E52B01D105233370082801D19200D2B232
:10D1380002F00303012B02F00C0208BF47F01007AE
:10D14800042A08BF47F00807F77220460021FFF7B6
:10D15800A2FEE0B920682169FFF7A6FCB8B96369A7
:10D168001A789AB1DA7A12F0080F0AD1A26903F193
:10D178000B018B420BD013F8016B12F801CB6645FB
:10D18800F7D020460021FFF7CAFEE2E70420A36992
:10D19800DB7A03F00403DBB260B1042814BF002279
:10D1A8000122002B14BF002302F00103002B18BF3B
:10D1B800052016E0ABB96369DA7A12F0100F0FD0C8
:10D1C800019A597DAD181A7D42EA0122D97E9B7ECB
:10D1D80043EA012343EA0243A36039E7062000E05B
:10D1E8000520FEBD80EB00084CEB000870B500215F
:10D1F8000446FFF750FE054648BB20682169FFF743
:10D2080053FC054618BB63691B78E52B14BF002245
:10D218000122002B14BF134642F00103CBB920466C
:10D228000121FFF77CFEE6E76669294630462022A1
:10D23800FFF734FC0B223046A169FFF725FCA369F0
:10D248000122DB7A03F01803337323681A71284626
:10D2580070BD20682169FFF727FC05460028F6D134
:10D26800E2E70000F8B5036815461A78303A092A4B
:10D2780009D893F801C0BCF13A0F04D10233036016
:10D28800002A40F01C819E4B1C680C60002C00F0AA
:10D29800188123786BB16078FFF7B0FB10F0010FAD
:10D2A80007D1002D00F00F8110F0040018BF0A20EC
:10D2B80012E1002020706070FFF786FB10F0010F6C
:10D2C80040F003811DB110F0040F40F000810021EF
:10D2D8002046FFF721FC012817D194F8F231002BE2
:10D2E80000F0F98094F8F86194F8F931360446EAC8
:10D2F800036694F8F63120461E4394F8F73146EA5F
:10D3080003263146FFF708FC00E00026032800F05A
:10D31800E080002840F0DF8094F83C2094F83B300F
:10D3280043EA0223B3F5007F40F0D58094F8472004
:10D3380094F8463053EA02230DD194F8563094F805
:10D3480057201B0443EA026394F85420134394F8CB
:10D35800552043EA022394F8402094F842C094F8F8
:10D368004110A361E270534394F83F0094F83E20C3
:10D3780041EA0C2194F8445094F843C042EA002052
:10D3880094F83D7032185CEA052C2262A77021815E
:10D398000FD194F852C094F853504FEA0C4C4CEA11
:10D3A800056C94F850504CEA050C94F851504CEA2E
:10D3B800052CC0EB0C000909C01A401AB0FBF7F79E
:10D3C800023740F6F6708742E76106D900F57040EB
:10D3D800874200F28280022500E0012598186062E9
:10D3E8005218D318A3624FF0FF3323610133032D82
:10D3F80023715AD1637194F8612094F86030607891
:10D4080043EA0222B218626104F130010123FFF7F6
:10D41800F9FA002849D194F82E3294F82F2243EAD9
:10D428000222384B12B29A423FD194F8322094F833
:10D438003330120442EA036294F830301A4394F805
:10D44800313042EA0322304B9A422ED194F8162208
:10D4580094F81732120442EA036294F814321A4319
:10D4680094F8153242EA0322284B9A421DD194F8C7
:10D478001E3294F81F221B0443EA026394F81C220C
:10D48800134394F81D2243EA0223E36094F81A3206
:10D4980094F81B221B0443EA026394F818221343EE
:10D4A80094F8192243EA02232361194A2570138844
:10D4B800002001339BB2E0621380E3800CE00B2074
:10D4C8000AE00C2008E0284606E0032004E00A20D1
:10D4D80002E0012000E00D20F8BD94F85E0094F809
:10D4E8005FC0000440EA0C6094F85CC0032540EA81
:10D4F8000C0094F85DC040EA0C20606270E700BF41
:10D508003052002055AAFFFF5252614172724161A8
:10D518002C52002050B9064B1B6803B1187009B192
:10D5280000230B70024B0020196000E00B207047AD
:10D5380030520020F0B58DB0044600230CA802F04C
:10D548001F0502AE40F82C1D236005F01E0231466F
:10D55800FFF788FE002840F0998009AB3046019912
:10D568000893FFF757FD15F01C0F56D060B104283B
:10D5780040F08C803046FFF739FE002840F0868066
:10D5880045F00805079E33E015F0040F79D1079E92
:10D59800002E7AD0F37A13F0110376D115F0080F24
:10D5A80026D0327D777DF17E42EA0727B27E337539
:10D5B8007375B376F37633777377B377F377029827
:10D5C80042EA0122012352EA07470371C36A09D0DC
:10D5D80039460093FFF726FC009B002856D1029A93
:10D5E800013FD76002981946FFF75EFA00284DD12F
:10D5F80015F0080F20D00023F372FFF743FAC0F3A9
:10D608000723B073F373030C000E33747074029B1A
:10D6180001221A7145F020050EE0002836D1079E38
:10D62800002E30D0F37A13F0100F2CD115F0020F22
:10D6380002D013F0010F28D1029BDA6AA571E261CA
:10D64800079A2262327D717DF07E42EA0121B27E24
:10D6580042EA002242EA01422261B27FF17F1204CB
:10D6680042EA0162317F00200A43717F236042EA67
:10D678000122E260FF22E271DB88A060A061A38042
:10D6880004E0082002E0042000E007200DB0F0BD0F
:10D69800F0B587B004931746049A002304460E4653
:10D6A800136081880068FFF77BFA0546002840F080
:10D6B800A780A37913F0800F40F09F8013F0010F2B
:10D6C80000F09D80E268A3680296D31A9F4228BFA3
:10D6D8001F4604F1240301970393059087E0A3688C
:10D6E800DA0568D12068E179827891420DD30BB9C7
:10D6F800206902E06169FFF764FA01280BD9B0F1EB
:10D70800FF3F4ED000236061E371276861693846A6
:10D71800FFF7B6FB20B9A37963F07F03A3716CE030
:10D72800E379019AC618550A21D0BA78E9189142C6
:10D7380088BFD51AEBB2787802993246FFF762F9BA
:10D74800A37900282ED113F0400F0BD0A069801BBD
:10D75800A84207D2029B039903EB40204FF40072C2
:10D76800FFF792F9E379EB18E3716D0232E0A379E0
:10D7780013F0400F0AD0012378780399A269FFF7C4
:10D7880061F9A37970B923F04003A371A369B34287
:10D798000DD023680399587832460123FFF732F9F0
:10D7A80028B1A37963F07F03A371012528E0E37909
:10D7B800A6610133E371A168019AC905C90DC1F5D4
:10D7C8000075039BAA4238BF1546591802982A4685
:10D7D800FFF75AF9029AA36852190292049A5B1940
:10D7E800A36013685B191360019B5B1B0193019A8B
:10D7F800002A7FF474AF059D02E0022500E00725AA
:10D80800284607B0F0BDF8B504460E468188006882
:10D81800FFF7C6F90546002840F09E80A27912F06D
:10D82800800F40F09880E3689E4203D912F0020FFF
:10D8380008BF1E460022A368A260FF32E271002ED4
:10D8480059D0206887787F0273B1013B711EB1FB04
:10D85800F7F1B3FBF7F2914206D37A4202EA0303E7
:10D86800A360F61A61690CE0216949B9FFF781FAEA
:10D878000128014635D0B0F1FF3F18BF206159D0CB
:10D888006161002936D01BE0A37913F0020F05D09F
:10D898002068FFF76EFA014620B914E02068FFF708
:10D8A80090F90146B1F1FF3F44D0012919D9236805
:10D8B800DB69994215D2A3686161DB19A360F61B85
:10D8C800BE42E1D800E03E46A368C6F347279B194D
:10D8D800A360F305E771DE0D6BB12068FFF7D0FA9E
:10D8E80020B9A37963F07F03A37134E0C619013727
:10D8F800E77100E00E46A368DB0522D0A2699642D4
:10D908001FD0A37913F0400F0BD0214651F8243BC8
:10D9180058780123FFF796F8A37960B923F04003FC
:10D92800A371214651F8243B324658780123FFF76A
:10D9380069F828B1A37963F07F03A37101250BE08F
:10D94800A661A368E268934206D9E360A37943F02D
:10D958002003A37100E002252846F8BD10B586B063
:10D96800044606A840F8141D00222146FFF77AFC59
:10D9780018BB03ABA36120460199FFF74BFBB8B96D
:10D98800636973B1DA7A12F0100F15D0597D1A7DD8
:10D9980042EA0122D97E9B7E43EA012343EA0243FD
:10D9A800A36023682046DB880021A380FFF773FA71
:10D9B800042808BF052000E0052006B010BD0000BF
:10D9C80000B5124B00201870114B124989B018701D
:10D9D800FFF7A0FD014628B10F48F8F7B7FE4FF052
:10D9E800FF3010E00D4901A8FFF7B8FF014628B144
:10D9F8000B48F8F7ABFE6FF0010004E0094B012279
:10DA08001870094B1A7009B000BD00BF7E54002081
:10DA18007F5400204052002000EC000833EC00083E
:10DA280035EC0008345200207C54002008B5094B1E
:10DA380000201870084B1870084B1870084B1870A5
:10DA4800084B1860084B1860F9F7F3FA074B0522E2
:10DA58001A7008BD7E5400207F54002070540020A6
:10DA68007C54002078540020745400207D540020F9
:10DA7800014B9878704700BF40520020054B821E2A
:10DA8800D96902398A423DBF98789B6A00FB023007
:10DA9800002070474052002070B51D4B04461B788B
:10DAA8000D462BB11B48F8F751FE6FF005002EE02C
:10DAB80019480122FFF73EFD184E306068B1FFF7A4
:10DAC8007FFF0028B8BF4FF0FF3020DB12482946FF
:10DAD8000122FFF72FFD3060B8B90F4B00209A796B
:10DAE8002270DA7962709A686260DA68A2601A69EC
:10DAF800E2605A6922619A696261DA691B6AA26105
:10DB0800E361034B01221A7001E06FF0040070BD5D
:10DB18007E540020E0EC000880540020AC890020EE
:10DB280010B5174B1B782BB11648F8F70FFE6FF09E
:10DB3800050023E0144B1549DA88D1F818C08A800B
:10DB480002780B608A714278CA71426884698A6077
:10DB58008268CA60C2680A6102694A614269C0692A
:10DB680094458A61CC61086204D058782431012335
:10DB7800FEF748FF024B01221A70002010BD00BFBB
:10DB88007E5400203CED00084052002080540020C4
:10DB98000B4B9A790270DA7942709A684260DA68B7
:10DBA80082601A69C2605A6902619A694261DA69D7
:10DBB8001B6A8261C361034B00201870704700BF65
:10DBC800805400207E54002008B501460448FFF721
:10DBD8001AFE044B0028186018BF6FF00F0008BD2C
:10DBE80080540020AC89002013B50D4A03461278F2
:10DBF8000C466FF002008AB119460A4801AB22466A
:10DC0800FFF746FD084B186030B9019BA3420CBFD3
:10DC180000206FF0070001E06FF006001CBD00BF98
:10DC28007C54002080540020AC890020F8B50446BC
:10DC38000F4600250F4E14E001212046FFF7D4FFC0
:10DC4800002815DB237801350A2B14BF0022012296
:10DC58000D2B14BF134642F0010333B9BD4238BF40
:10DC68000134B268F3689A42E6D300232370284649
:10DC7800F8BD00BF8054002008B5F7F753FD08BD74
:10DC8800D0400B1CD1409C46203AD3401843524206
:10DC980063469340184370479140031C90409C464C
:10DCA800203A9340194352426346D3401943704780
:10DCB80070B50D4D0D4E0024761BB61003E055F8D7
:10DCC800043B98470134B442F9D3094D094EF7F79C
:10DCD800D7FD761BB610002403E055F8043B98479F
:10DCE8000134B442F9D370BDCCF90008CCF900086E
:10DCF800CCF90008CCF90008002305E011F803C0AE
:10DD0800013A00F803C00133002AF7D170470346EF
:10DD180002E003F8011B013A002AFAD1704710B556
:10DD280084469CF8003062460CF1010C002BF8D1B7
:10DD3800CC5CD4540133002CFAD110BD10F8013B4F
:10DD48000A461BB111F801CB6345F7D01078181AB1
:10DD580070470023CA5CC2540133002AFAD17047C5
:10DD680003461A4613F8011B0029FAD1101A704706
:10DD780010B5844607E011F8014B634603F8014BE0
:10DD8800013A9C462CB1002AF5D104E003F8014B76
:10DD9800013A002AFAD110BDF7B51F4E044637687C
:10DDA800D7F8E850002D2ED150200191FFF764FFDD
:10DDB8003368C7F8E800D3F8E82095601560556027
:10DDC800D3F8E8201561D560D3F8E820956155614E
:10DDD800D3F8E820D5629562D3F8E8205563156337
:10DDE800D3F8E820D5639563D3F8E8205564156423
:10DDF800D3F8E820D5649564D3F8E8201577D3F8EC
:10DE0800E83001995D62044B20461B68D3F8E8208E
:10DE1800012300F003F8FEBD60010020F0B510B941
:10DE28001068002829D084460D4610F8014B07E0F9
:10DE3800B44205D1002BF6D110608CF8003017E001
:10DE480015F8016B002EF3D1034614B9146020466F
:10DE580013E01F4613F8010B0D461C4615F8016B1D
:10DE6800864207D110B100233B7000E004461460DD
:0CDE7800604602E0002EF1D1EBE7F0BDA7
:10DE8400000305070A0C0F11131517191C1E202275
:10DE9400242527292B2D2E3032333537383A3B3D74
:10DEA4003E3F414244454647494A4B4C4E4F5051F0
:10DEB40052535455565758595A5B5C5D5D5E5E5FCC
:10DEC400606162636465656667676869696A6B6BEC
:10DED4006C6D6D6E6E6F6F7070717172727373743E
:10DEE40074757576767677777878787979797A7AB9
:10DEF4007A7B7B7B7C7C7C7D7D7D7E7E7E7F7F7F51
:10DF040046696C656E616D652069732025732E000A
:10DF14005B4150505D206661696C656420746F20BC
:10DF24006F70656E2066696C652C207374617475FE
:10DF3400733A2025640A005B4150505D2053616DA3
:10DF4400706C65206E6F2025642066696C656E6157
:10DF54006D65202573206F70656E6564206F662083
:10DF64006C656E6774682025750A004162616E6491
:10DF74006F6E696E6720444D4120726F7574696ECF
:10DF8400652061667465722025642E2564206D7396
:10DF94002C20616674657220256420766F69636540
:10DFA40073206F7574206F66202564004F70656E52
:10DFB400696E672062616E6B2066696C65202573EB
:10DFC400004661696C656420746F206F70656E2013
:10DFD40062616E6B2066696C652E0053616D706CB6
:10DFE40065206E6F2025642C2066696C656E616DFA
:10DFF400652069733A2025732C206D696469206E4D
:10E004006F74652076616C75653D307825782C20B9
:10E0140064656361792076616C75652025642C20C4
:10E02400686F6C643D2564004F70656E2073616D8C
:10E03400706C652066696C65206661696C65642E28
:10E0440000436C75737465722025643A202564203E
:10E05400004F70656E696E67206E65772073616D21
:10E06400706C652062616E6B004F70656E696E67DF
:10E0740020636F6E6669672066696C65202573008E
:10E08400706C617965722E636667004661696C65C0
:10E094006420746F206F70656E20636F6E666967AD
:10E0A4002066696C652E00466F756E64207061721F
:10E0B400616D20257320616E642076616C75652026
:10E0C4002573006C65655F6877006D6964696368D2
:10E0D400616E6E656C004D4944492050726F6772E1
:10E0E400616D204368616E6765207265636569765A
:10E0F4006564202D204368616E67696E67206261E4
:10E104006E6B20746F202564005344206361726435
:10E1140020706F6C7970686F6E69632073616D70C5
:10E124006C6520706C617965720028432920323057
:10E134003131204C204F27446F6E6E656C6C206C1F
:10E14400656540626173736D616B65722E636F2EDA
:10E15400756B00496E697469616C6973696E6720D7
:10E16400534420636172642E2E004572726F7220D4
:10E17400696E697469616C6973696E6720534420C0
:10E184006361726400534420436172642065727257
:10E194006F723A20636F6E6E656374696F6E20668A
:10E1A40061696C6564210052656164696E67204A27
:10E1B40031302073776974636800496E69746961EA
:10E1C4006C6973696E672073796E74682E2E2E00E5
:10E1D40053796E746820696E697420646F6E652E5D
:10E1E40000564F4943455F5343414E0042414E4B15
:10E1F4005357495443485F5343414E004D494449A2
:10E204005F486F6F6B7300464154414C3A2046722D
:10E21400656552544F5320004D616C6C6F6320450B
:10E2240072726F722121212000464154414C3A20E0
:10E234004672656552544F53204D616C6C6F632078
:10E244004572726F722121210A00476F6F646279EF
:10E25400652100476F6F64627965210A003D3D3D89
:10E264003D3D3D3D3D3D3D3D3D3D3D3D3D3D3D0A0D
:10E27400002121212048415244204641554C54203C
:10E284002121210A005230203D20253038780A000F
:10E294005231203D20253038780A005232203D206A
:10E2A400253038780A005233203D20253038780A4A
:10E2B40000523132203D20253038780A004C52205B
:10E2C4003D20253038780A005043203D2025303841
:10E2D400780A00505352203D20253038780A0042F5
:10E2E400464152203D20253038780A004346535297
:10E2F400203D20253038780A0048465352203D20DE
:10E30400253038780A0044465352203D20253038C1
:10E31400780A0041465352203D20253038780A00BF
:10E3240021212048415244204641554C542021216A
:10E334000061742050433D307825303878004944DA
:10E344004C45000A0A44756D70696E6720746865EF
:10E3540020756D6D5F686561702E2E2E0A007C300D
:10E3640078253038787C42202535647C4E4220253F
:10E3740035647C5042202535647C5A202535647CE4
:10E384004E46202535647C5046202535647C0A00A1
:10E394007C3078253038787C42202535647C4E42A8
:10E3A400202535647C5042202535647C5A2025354F
:10E3B400647C0A00546F74616C20456E74726965E4
:10E3C4007320253564202020205573656420456E14
:10E3D4007472696573202535642020202046726597
:10E3E4006520456E7472696573202535640A00548E
:10E3F4006F74616C20426C6F636B732020253564ED
:10E40400202020205573656420426C6F636B732059
:10E4140020253564202020204672656520426C6FDB
:10E42400636B7320202535640A0053697A65206F75
:10E434006620756D6D5F6865617020697320256461
:10E444002062797465732C20757365643A202564A1
:10E454002062797465732C20667265653A202564A0
:10E464002062797465730A0043616E277420616CBD
:10E474006C6F636174652025356420626C6F636B17
:10E4840073206174202535640A00434C43440043DF
:10E494004C43445F444F4700474C43445F43555308
:10E4A400544F4D00474C43445F4B53303130380098
:10E4B400474C43445F4B53303130385F494E5643E9
:10E4C4005300474C43445F444F4700474C43445F29
:10E4D4005353443133303600474C43445F53534421
:10E4E400313330365F524F544154454400474C4316
:10E4F400445F5345443135323000000000020100CE
:10E504001400020001000000004014540101020143
:10E5140000000000000000000000000000000203F2
:10E524000301020303030303020203014D494F5392
:10E5340033320053544D33324634444953434F56D7
:10E544004552590053544D333246347878003F00D5
:10E554005B4D494F5333325F4D4944495F535953DF
:10E5640045585F436D645F44656275675D20636F02
:10E574006D6D616E642068616E646C6572206E6F8F
:10E584007420696D706C656D656E74656420627964
:10E59400206170706C69636174696F6E0A0028454C
:10E5A40052524F523A20737472696E6720706173CD
:10E5B40073656420746F204D494F5333325F4D4966
:10E5C40044495F53656E6444656275674D65737352
:10E5D4006167652829206973206C6F6E67657220F6
:10E5E4007468616E20313030206368617273210A6F
:10E5F400005B4D494F5333325F4D4944495F526587
:10E6040063656976655F48616E646C65725D20540C
:10E61400696D656F7574206F6E20706F7274203031
:10E6240078253032780A00202530325800253038D9
:10E63400582000000202020201010200F000007EE4
:10E6440032000000FEFFFFFFFFFFFFFF000000009D
:10E65400426F6F746C6F61646572204D6F646520E6
:10E6640000000000718C00087D8C0008858D000876
:10E67400898C00084D8D00081D8D0008258D00082B
:10E68400018E0008D58D0008378D000800000000B9
:10E694003B8D0008C38D0008B18D00080000000008
:10E6A4000000000000000000418D0008040309047C
:10E6B4001201000200000040C016FE030001010226
:10E6C400030100002D8D00082F8D0008F58D000832
:10E6D400338D0008358D0008318D0008EB8D00085E
:10E6E4003432006D696469626F782E6F726700005E
:10E6F40009026500020100803209040000000101E2
:10E7040000020924010001090001010904010002B9
:10E714000103000207240100014100062402010153
:10E72400000624020202000924030103010201007D
:10E73400092403020401010100090502024000004A
:10E7440000000525010101090581024000000000C7
:10E754000525010103000000286E756C6C2900007A
:10E7640002010200001020300608000600808080AC
:10E77400808000C0C0C0C0C000E0E0E0E0E000F085
:10E78400F0F0F0F000F8F8F8F8F800FCFCFCFCFC01
:10E7940000FEFEFEFEFE00FFFFFFFFFF00183C7EB2
:10E7A400FF0000FF7E3C1800000000000000000095
:10E7B4000000000000000000000000000000000055
:10E7C4000000000000000000000000000000000045
:10E7D4000000000000000000000000000000000035
:10E7E4000000000000000000000000000000000025
:10E7F4000000000000000000000000000000000015
:10E804000000000000000000000000000000000004
:10E8140000000000000000000000000000000000F4
:10E8240000000000000000000000000000000000E4
:10E8340000000000004F0000000007000700001463
:10E844007F147F1400242A7F2A1200231308646291
:10E8540000364955225000000503000000001C2228
:10E864004100000041221C000014083E0814000866
:10E87400083E080800000050300000080808080896
:10E88400000030300000002010080402003E51490E
:10E89400453E0000427F400000426151494600214C
:10E8A40041454B31001814127F1000274545453966
:10E8B400003C4A49493000017109050300364949C1
:10E8C400493600064949291E00000036360000007A
:10E8D40000563600000814224100001414141414C5
:10E8E400000041221408000201510906003249794E
:10E8F400413E007E1111117E007F49494936003E98
:10E9040041414122007F4141221C007F4949494144
:10E91400007F09090901003E4149497A007F08083E
:10E92400087F0000417F4100002040413F01007FFB
:10E9340008142241007F40404040007F020C027FC7
:10E94400007F0408107F003E4141413E007F0909D9
:10E954000906003E4151215E007F091929460046FF
:10E96400494949310001017F0101003F4040403FD6
:10E97400001F2040201F003F4038403F0063140820
:10E9840014630007087008070061514945430000FB
:10E994007F414100000204081020000041417F0033
:10E9A4000004020102040040404040400000010213
:10E9B4000400002054545478007F484444380038FC
:10E9C4004444442000384444487F00385454541884
:10E9D40000087E090102000C5252523E007F0804D6
:10E9E40004780000447D4000002040443D00007F46
:10E9F400102844000000417F4000007C0418047883
:10EA0400007C08040478003844444438007C14141E
:10EA1400140800081414187C007C08040408004836
:10EA24005454542000083E484020003C4040207C80
:10EA3400001C2040201C003C4030403C0044281076
:10EA44002844000C5050503C004464544C44000092
:10EA5400083641000000007F000000000041360835
:10EA64000002010201000000000000005B64697301
:10EA74006B5F696E697469616C697A655D20657242
:10EA8400726F72207768696C6520636865636B696F
:10EA94006E6720666F72205344204361726420289D
:10EAA400737461747573202564290A005B64697347
:10EAB4006B5F726561645D206572726F7220776846
:10EAC400696C652072656164696E6720736563743F
:10EAD4006F722025640A005B6469736B5F777269E7
:10EAE40074655D206572726F72207768696C652049
:10EAF40077726974696E6720746F20736563746FCD
:10EB0400722025640A005B4745545F534543544FC4
:10EB1400525F434F554E545D20436F756E742069A8
:10EB2400732025640A005B4745545F424C4F434BB6
:10EB34005F53495A455D20426C6F636B2053697A79
:10EB4400652069732025640A0020222A2B2C5B3D52
:10EB54005D7C7F004E4F204E414D452020202046B5
:10EB640041542020202020004E4F204E414D45206E
:10EB7400202020464154333220202000809A9041A6
:10EB84008E418F804545454949498E8F9092924FD9
:10EB9400994F555559999A9B9C9D9E9F41494F5514
:10EBA400A5A5A6A7A8A9AAABAC21AEAFB0B1B2B334
:10EBB400B4B5B6B7B8B9BABBBCBDBEBFC0C1C2C399
:10EBC400C4C5C6C7C8C9CACBCCCDCECFD0D1D2D389
:10EBD400D4D5D6D7D8D9DADBDCDDDEDFE0E1E2E379
:10EBE400E4E5E6E7E8E9EAEBECEDEEEFF0F1F2F369
:10EBF400F4F5F6F7F8F9FAFBFCFDFEFF5B46494C29
:10EC0400455D204661696C656420746F206D6F7585
:10EC14006E742053442043617264202D2065727207
:10EC24006F72207374617475733A2025640A002F1F
:10EC3400005B46494C455D204661696C65642074FF
:10EC44006F206F70656E20726F6F742064697265D7
:10EC540063746F7279202D206572726F72207374E1
:10EC6400617475733A2025640A005B46494C455F1C
:10EC74005570646174654672656542797465735D47
:10EC840020665F6F70656E646972206661696C6589
:10EC940064207769746820737461747573202564C3
:10ECA400210A005B46494C455F55706461746546B2
:10ECB40072656542797465735D20665F6765746625
:10ECC400726565206661696C656420776974682083
:10ECD400737461747573202564210A005B46494C82
:10ECE400455D204641494C5552453A207472696548
:10ECF4006420746F206F70656E2066696C652027D0
:10ED040025732720666F722072656164696E672CB3
:10ED1400206275742070726576696F7573206669F8
:10ED24006C65206861736E2774206265656E20636C
:10ED34006C6F736564210A005B46494C455D20464F
:10ED440041494C5552453A20747269656420746F88
:10ED54002072656F70656E2066696C652C20627523
:10ED6400742070726576696F75732066696C6520AE
:10ED74006861736E2774206265656E20636C6F73BF
:10ED84006564210A005B46494C455D204641494C77
:10ED94005552453A20747269656420746F206F700F
:10EDA400656E2066696C65202725732720666F725F
:10EDB4002077726974696E672C2062757420707292
:10EDC4006576696F75732066696C65206861736E1A
:10EDD4002774206265656E20636C6F736564210A15
:10EDE400005B46494C455F53656E645379784475BE
:10EDF4006D705D204552524F52207768696C6520D2
:10EE040072656164696E672066696C652C20737431
:10EE1400617475733A2025640A004552524F523A80
:10EE24002052656164696E672043494420666169C4
:10EE34006C656420776974682073746174757320D9
:10EE44002564210A002D2D2D2D2D2D2D2D2D2D2D1B
:10EE54002D2D2D2D2D2D2D2D2D0A004349443A0AFB
:10EE6400002D204D616E756661637475726572491B
:10EE7400443A0A002D204F454D204170706C694979
:10EE8400443A0A002D2050726F644E616D653A2039
:10EE940025730A002D2050726F645265763A20253E
:10EEA400750A002D2050726F64534E3A2030782535
:10EEB4003038780A002D20526573657276656431A6
:10EEC4003A2025750A002D204D616E7566616374C4
:10EED400446174653A2025750A002D206D73645FC2
:10EEE4004352433A203078253032780A002D20529C
:10EEF40065736572766564323A2025750A00455259
:10EF0400524F523A2052656164696E6720435344FC
:10EF1400206661696C656420776974682073746124
:10EF2400747573202564210A002D204353445374BF
:10EF3400727563743A2025750A002D205379735332
:10EF440070656356657273696F6E3A2025750A00A1
:10EF54002D20544141433A2025750A002D204E535B
:10EF640041433A2025750A002D204D61784275737E
:10EF7400436C6B467265633A2025750A002D204365
:10EF8400617264436F6D64436C61737365733A209B
:10EF940025750A002D205264426C6F636B4C656EBC
:10EFA4003A2025750A002D2050617274426C6F63FB
:10EFB4006B526561643A2025750A002D2057724210
:10EFC4006C6F636B4D6973616C69676E3A2025756C
:10EFD4000A002D205264426C6F636B4D6973616C3F
:10EFE40069676E3A2025750A002D20445352496DF5
:10EFF400706C3A2025750A002D2044657669636596
:10F0040053697A653A2025750A002D204D6178529E
:10F014006443757272656E745644444D696E3A2049
:10F0240025750A002D204D6178526443757272650E
:10F034006E745644444D61783A2025750A002D209B
:10F044004D6178577243757272656E745644444DBF
:10F05400696E3A2025750A002D204D617857724358
:10F06400757272656E745644444D61783A20257504
:10F074000A002D2044657669636553697A654D7588
:10F084006C3A2025750A002D20457261736547721C
:10F0940053697A653A2025750A002D2045726173FB
:10F0A4006547724D756C3A2025750A002D205772FC
:10F0B40050726F74656374477253697A653A202598
:10F0C400750A002D20577250726F7465637447720D
:10F0D400456E61626C653A2025750A002D204D61EC
:10F0E4006E4465666C4543433A2025750A002D201D
:10F0F40057725370656564466163743A2025750AD6
:10F10400002D204D61785772426C6F636B4C656EB5
:10F114003A2025750A002D205772697465426C6F78
:10F12400636B50615061727469616C3A2025750A91
:10F13400002D205265736572766564333A20257517
:10F144000A002D20436F6E74656E7450726F74657F
:10F1540063744170706C693A2025750A002D20464D
:10F16400696C65466F726D617447726F756F703A42
:10F174002025750A002D20436F7079466C61673A2B
:10F184002025750A002D205065726D577250726FDC
:10F19400746563743A2025750A002D2054656D70DA
:10F1A400577250726F746563743A2025750A002D86
:10F1B4002046696C65466F726D61743A2025750A44
:10F1C400002D204543433A2025750A002D20526521
:10F1D400736572766564343A2025750A005B53447E
:10F1E400434152445F4552524F523A25645D206672
:10F1F40061696C656420746F206163636573732057
:10F20400534420636172640A005B53444341524493
:10F214005F4552524F523A25645D204446535F473E
:10F22400657450746E5374617274206661696C65A0
:10F234006420746F2066696E6420706172746974EE
:10F24400696F6E0A005B5344434152445F45525216
:10F254004F523A25645D204446535F476574566FA8
:10F264006C496E666F206661696C656420746F20FA
:10F2740066696E6420766F6C756D6520696E666F65
:10F28400726D6174696F6E0A005B5344434152446A
:10F294005F4552524F523A25645D20756E6B6E6F16
:10F2A400776E2066696C6573797374656D20286F59
:10F2B4006E6C792046415431322F31362F3332204F
:10F2C400737570706F72746564290A005B534443EC
:10F2D4004152445F4552524F523A25645D204446A0
:10F2E400535F4F70656E46696C65282E2E444653F5
:10F2F4005F524541442E2E29206661696C65642C59
:10F3040020652E672E2066696C65206E6F742066FA
:10F314006F756E640A005B5344434152445F455227
:10F32400524F523A25645D2046494C455F5265610F
:10F33400644F70656E282920686173206265656E6C
:10F344002063616C6C6564207768696C65207072F9
:10F354006576696F75732066696C65206861736E84
:10F364002774206265656E20636C6F7365640A00A0
:10F374005B5344434152445F4552524F523A2564D1
:10F384005D204446535F5265616446696C6520663E
:10F3940061696C65640A005B5344434152445F45B0
:10F3A40052524F523A25645D206C65737320627922
:10F3B4007465732072656164207468616E20657879
:10F3C4007065637465640A005B5344434152445F4F
:10F3D4004552524F523A25645D204446535F52656C
:10F3E4006164436C6F73652061626F72746564203D
:10F3F40064756520746F2070726576696F7573200B
:10F404006572726F720A005B5344434152445F4514
:10F4140052524F523A25645D2046494C455F57721B
:10F424006974654F70656E206661696C65642074EB
:10F434006F20616C6C6F63617465206D656D6F72B4
:10F444007920666F722077726974652062756666CA
:10F4540065720A005B5344434152445F4552524F24
:10F46400523A25645D204446535F4F70656E466989
:10F474006C65282E2E4446535F57524954452E2E10
:10F4840029206661696C65640A005B5344434152F8
:10F49400445F4552524F523A25645D2046494C45DB
:10F4A4005F57726974654F70656E282920686173AF
:10F4B400206265656E2063616C6C656420776869A1
:10F4C4006C652070726576696F75732066696C650A
:10F4D400206861736E2774206265656E20636C6FAB
:10F4E4007365640A005B5344434152445F4552527E
:10F4F4004F523A25645D204446535F5772697465E0
:10F5040046696C65206661696C65640A005B5344F6
:10F51400434152445F4552524F523A25645D206C38
:10F524006573732062797465732077726974746586
:10F534006E207468616E2065787065637465640A12
:10F54400005B5344434152445F4552524F523A2563
:10F55400645D204446535F5772697465436C6F73EE
:10F56400652061626F727465642064756520746FD0
:10F574002070726576696F7573206572726F720A96
:10F58400005B5344434152445F4552524F523A2523
:10F59400645D2046494C455F5365656B28292066A8
:10F5A40061696C65640A005B5344434152445F459E
:10F5B40052524F523A25645D204446535F4F706562
:10F5C4006E446972282E2E4446535F524541442EA0
:10F5D4002E29206661696C65642C20652E672E20B7
:10F5E4006469726563746F7279206E6F7420666FDC
:10F5F400756E640A005B5344434152445F45525262
:10F604004F523A25645D2046494C455F436F7079FB
:10F614002829206661696C65640A005B5344434190
:10F6240052445F4552524F523A25645D20736F75C0
:10F634007263652066696C6520646F65736E2774F8
:10F644002065786973740A005B5344434152445FF4
:10F654004552524F523A25645D2046494C455F4716
:10F664006574446972732829206F722046494C4599
:10F674005F47657446696C65732829206661696C07
:10F6840065642062656361757365206F66206D69CA
:10F694007373696E67206469726563746F72790A43
:10F6A400005B5344434152445F4552524F523A2502
:10F6B400645D2046494C455F47657446696C6573D3
:10F6C4002829206661696C656420626563617573CD
:10F6D40065206F66206D697373696E672064697253
:10F6E4006563746F72790A005B5344434152445F0B
:10F6F4004552524F523A25645D206572726F7220F2
:10F704007768696C652072656164696E67202E7321
:10F7140079782066696C650A005B5344434152441E
:10F724005F4552524F523A25645D2046494C455F2D
:10F734004D616B654469722829206661696C656452
:10F744000A005B5344434152445F4552524F523A7C
:10F7540025645D2046494C455F4C6F616453657375
:10F7640073696F6E4E616D6528290A005B534443CB
:10F774004152445F4552524F523A25645D204649F6
:10F784004C455F5570646174654672656542797471
:10F79400657328290A005B5344434152445F455230
:10F7A400524F523A25645D207365652066696C6525
:10F7B4002E6820666F722064657363726970746961
:10F7C4006F6E0A002D006D6B64697200230064651E
:10F7D4006C0072656164005B46494C455D20446F72
:10F7E400776E6C6F6164206F662025642062797483
:10F7F400657320696E2070726F6772657373202859
:10F804002564252529005B46494C455D20446F77D6
:10F814006E6C6F6164206F66202564206279746564
:10F82400732066696E69736865642E007772697403
:10F8340065007E003030303030303030005B464977
:10F844004C455D2055706C6F6164696E672025734B
:10F8540020776974682025642062797465730A00CE
:10F86400777269746564617461005B46494C455DF7
:10F874002055706C6F6164206F6620256420627966
:10F884007465732066696E69736865642E0025303B
:10F894003858005B46494C455D2055706C6F616477
:10F8A400206F6620256420627974657320696E2058
:10F8B40070726F677265737320282564252529008B
:10F8C400002020202020202020202828282828202C
:10F8D4002020202020202020202020202020202024
:10F8E400208810101010101010101010101010108C
:10F8F400100404040404040404040410101010107C
:10F904001010414141414141010101010101010145
:10F914000101010101010101010101011010101097
:10F924001010424242424242020202020202020217
:10F93400020202020202020202020202101010106B
:10F944002000000000000000000000000000000093
:10F9540000000000000000000000000000000000A3
:10F964000000000000000000000000000000000093
:10F974000000000000000000000000000000000083
:10F984000000000000000000000000000000000073
:10F994000000000000000000000000000000000063
:10F9A4000000000000000000000000000000000053
:10F9B4000000000000000000000000000000000043
:0CF9C400000000004300000000000000F4
:10F9D00001007F000101000062616E6B2E000000DB
:10F9E0000000000000000000FFFFFFFFAAAAAAAA73
:10F9F00010FF1010100000000000000001020304BE
:10FA000001020304060708093C00002033A900088E
:10FA100099A800084DA80008F3A700081FA800082F
:10FA2000DFA70008C9A7000803A8000811A800085C
:10FA30000000000000000000FE000000C4F8000804
:10FA400000000000000000000000000000000000B6
:10FA500000000000000000000000000000000000A6
:10FA6000C8F90008000000000000000000000000CD
:10FA70000000000000000000000000000000000086
:10FA80000000000000000000000000000000000076
:10FA90000000000000000000000000000000000066
:10FAA0000000000000000000000000000000000056
:10FAB0000000000000000000000000000000000046
:10FAC0000000000000000000000000000000000036
:10FAD0000000000000000000000000000000000026
:10FAE0000000000000000000000000000000000016
:10FAF0000000000000000000000000000000000006
:10FB000000000000000000000000000000000000F5
:10FB100000000000000000000000000000000000E5
:10FB200000000000000000000000000000000000D5
:08FB300070000020000000003D
:040000050800418826
:00000001FF
